Component: ARM Compiler 5.06 update 5 (build 528) Tool: armlink [4d35e2]

==============================================================================

Section Cross References

    system_stm32f4xx.o(.text) refers to system_stm32f4xx.o(.data) for SystemCoreClock
    tcp_in.o(.text) refers to tcp_out.o(.text) for tcp_rexmit_fast
    tcp_in.o(.text) refers to pbuf.o(.text) for pbuf_clen
    tcp_in.o(.text) refers to def.o(.text) for lwip_ntohs
    tcp_in.o(.text) refers to tcp.o(.text) for tcp_seg_free
    tcp_in.o(.text) refers to tcp_in.o(.data) for flags
    tcp_in.o(.text) refers to tcp.o(.data) for tcp_ticks
    tcp_in.o(.text) refers to tcp_in.o(.bss) for inseg
    tcp_in.o(.text) refers to lwip_timers.o(.text) for tcp_timer_needed
    tcp_in.o(.text) refers to ip.o(.data) for current_iphdr_src
    tcp_in.o(.text) refers to ip_addr.o(.text) for ip4_addr_isbroadcast
    tcp_in.o(.text) refers to memp.o(.text) for memp_free
    lwip_timers.o(.text) refers to memp.o(.text) for memp_malloc
    lwip_timers.o(.text) refers to tcp.o(.text) for tcp_tmr
    lwip_timers.o(.text) refers to ip_frag.o(.text) for ip_reass_tmr
    lwip_timers.o(.text) refers to etharp.o(.text) for etharp_tmr
    lwip_timers.o(.text) refers to dhcp.o(.text) for dhcp_coarse_tmr
    lwip_timers.o(.text) refers to ethernetif.o(.text) for sys_now
    lwip_timers.o(.text) refers to lwip_timers.o(.data) for next_timeout
    lwip_timers.o(.text) refers to tcp.o(.data) for tcp_active_pcbs
    memp.o(.text) refers to memp.o(.bss) for memp_memory
    memp.o(.text) refers to memp.o(.constdata) for memp_sizes
    memp.o(.data) refers to memp.o(.conststring) for .conststring
    dhcp.o(.text) refers to pbuf.o(.text) for pbuf_free
    dhcp.o(.text) refers to def.o(.text) for lwip_htonl
    dhcp.o(.text) refers to udp.o(.text) for udp_sendto_if
    dhcp.o(.text) refers to netif.o(.text) for netif_set_down
    dhcp.o(.text) refers to etharp.o(.text) for etharp_query
    dhcp.o(.text) refers to dhcp.o(.data) for xid
    dhcp.o(.text) refers to ip_addr.o(.constdata) for ip_addr_broadcast
    dhcp.o(.text) refers to dhcp.o(.bss) for dhcp_rx_options_given
    dhcp.o(.text) refers to netif.o(.data) for netif_list
    dhcp.o(.text) refers to memseta.o(.text) for __aeabi_memclr4
    dhcp.o(.text) refers to mem.o(.text) for mem_free
    udp.o(.text) refers to pbuf.o(.text) for pbuf_header
    udp.o(.text) refers to ip_addr.o(.text) for ip4_addr_isbroadcast
    udp.o(.text) refers to def.o(.text) for lwip_ntohs
    udp.o(.text) refers to icmp.o(.text) for icmp_dest_unreach
    udp.o(.text) refers to ip.o(.text) for ip_output_if
    udp.o(.text) refers to udp.o(.data) for udp_port
    udp.o(.text) refers to ip.o(.data) for current_iphdr_dest
    udp.o(.text) refers to memp.o(.text) for memp_free
    udp.o(.text) refers to memseta.o(.text) for __aeabi_memclr4
    mem.o(.text) refers to memseta.o(.text) for __aeabi_memclr
    mem.o(.text) refers to mem.o(.data) for ram
    mem.o(.text) refers to mem.o(.bss) for ram_heap
    netif.o(.text) refers to tcp.o(.text) for tcp_abort
    netif.o(.text) refers to etharp.o(.text) for etharp_cleanup_netif
    netif.o(.text) refers to dhcp.o(.text) for dhcp_network_changed
    netif.o(.text) refers to tcp.o(.data) for tcp_active_pcbs
    netif.o(.text) refers to netif.o(.data) for netif_num
    tcp.o(.text) refers to pbuf.o(.text) for pbuf_free
    tcp.o(.text) refers to memp.o(.text) for memp_free
    tcp.o(.text) refers to tcp_out.o(.text) for tcp_zero_window_probe
    tcp.o(.text) refers to tcp.o(.data) for tcp_ticks
    tcp.o(.text) refers to tcp.o(.constdata) for tcp_persist_backoff
    tcp.o(.text) refers to lwip_timers.o(.text) for tcp_timer_needed
    tcp.o(.text) refers to ip.o(.text) for ip_route
    tcp.o(.text) refers to memseta.o(.text) for __aeabi_memclr4
    tcp.o(.constdata) refers to tcp.o(.conststring) for .conststring
    tcp.o(.constdata) refers to tcp.o(.data) for tcp_listen_pcbs
    tcp_out.o(.text) refers to pbuf.o(.text) for pbuf_alloc
    tcp_out.o(.text) refers to def.o(.text) for lwip_htons
    tcp_out.o(.text) refers to memp.o(.text) for memp_malloc
    tcp_out.o(.text) refers to tcp.o(.text) for tcp_seg_free
    tcp_out.o(.text) refers to memcpya.o(.text) for __aeabi_memcpy
    tcp_out.o(.text) refers to ip.o(.text) for ip_output
    tcp_out.o(.text) refers to tcp.o(.data) for tcp_ticks
    tcp_out.o(.text) refers to tcp_in.o(.data) for tcp_input_pcb
    raw.o(.text) refers to pbuf.o(.text) for pbuf_header
    raw.o(.text) refers to ip.o(.text) for ip_route
    raw.o(.text) refers to memp.o(.text) for memp_free
    raw.o(.text) refers to memseta.o(.text) for __aeabi_memclr4
    raw.o(.text) refers to raw.o(.data) for raw_pcbs
    raw.o(.text) refers to ip.o(.data) for current_iphdr_dest
    init.o(.text) refers to mem.o(.text) for mem_init
    init.o(.text) refers to memp.o(.text) for memp_init
    init.o(.text) refers to netif.o(.text) for netif_init
    init.o(.text) refers to udp.o(.text) for udp_init
    init.o(.text) refers to tcp.o(.text) for tcp_init
    init.o(.text) refers to lwip_timers.o(.text) for sys_timeouts_init
    pbuf.o(.text) refers to memp.o(.text) for memp_free
    pbuf.o(.text) refers to mem.o(.text) for mem_free
    pbuf.o(.text) refers to memcpya.o(.text) for __aeabi_memcpy
    pbuf.o(.text) refers to strlen.o(.text) for strlen
    ip_addr.o(.text) refers to def.o(.text) for lwip_htonl
    ip_addr.o(.text) refers to ip_addr.o(.bss) for str
    inet_chksum.o(.text) refers to def.o(.text) for lwip_htons
    ip_frag.o(.text) refers to memp.o(.text) for memp_free
    ip_frag.o(.text) refers to memcpya.o(.text) for __aeabi_memcpy
    ip_frag.o(.text) refers to icmp.o(.text) for icmp_time_exceeded
    ip_frag.o(.text) refers to pbuf.o(.text) for pbuf_clen
    ip_frag.o(.text) refers to memseta.o(.text) for __aeabi_memclr4
    ip_frag.o(.text) refers to def.o(.text) for lwip_ntohs
    ip_frag.o(.text) refers to ip_frag.o(.data) for reassdatagrams
    ip_frag.o(.text) refers to inet_chksum.o(.text) for inet_chksum
    ip.o(.text) refers to pbuf.o(.text) for pbuf_free
    ip.o(.text) refers to def.o(.text) for lwip_ntohs
    ip.o(.text) refers to ip_addr.o(.text) for ip4_addr_isbroadcast
    ip.o(.text) refers to ip_frag.o(.text) for ip_reass
    ip.o(.text) refers to raw.o(.text) for raw_input
    ip.o(.text) refers to udp.o(.text) for udp_input
    ip.o(.text) refers to tcp_in.o(.text) for tcp_input
    ip.o(.text) refers to icmp.o(.text) for icmp_input
    ip.o(.text) refers to netif.o(.data) for netif_list
    ip.o(.text) refers to ip.o(.data) for current_iphdr_dest
    icmp.o(.text) refers to pbuf.o(.text) for pbuf_header
    icmp.o(.text) refers to ip_addr.o(.text) for ip4_addr_isbroadcast
    icmp.o(.text) refers to inet_chksum.o(.text) for inet_chksum_pbuf
    icmp.o(.text) refers to ip.o(.text) for ip_output_if
    icmp.o(.text) refers to memcpya.o(.text) for __aeabi_memcpy
    icmp.o(.text) refers to ip.o(.data) for current_iphdr_dest
    err.o(.text) refers to err.o(.data) for err_strerr
    err.o(.data) refers to err.o(.conststring) for .conststring
    etharp.o(.text) refers to pbuf.o(.text) for pbuf_free
    etharp.o(.text) refers to ip_addr.o(.text) for ip4_addr_isbroadcast
    etharp.o(.text) refers to etharp.o(.bss) for arp_table
    etharp.o(.text) refers to etharp.o(.constdata) for ethzero
    etharp.o(.text) refers to def.o(.text) for lwip_htons
    etharp.o(.text) refers to dhcp.o(.text) for dhcp_arp_reply
    etharp.o(.text) refers to memcmp.o(.text) for memcmp
    etharp.o(.text) refers to ip.o(.text) for ip_input
    etharp.o(.text) refers to etharp.o(.data) for etharp_cached_entry
    stm32f4xx_hal_flash_ex.o(.text) refers to stm32f4xx_hal_flash.o(.text) for FLASH_WaitForLastOperation
    stm32f4xx_hal_flash_ex.o(.text) refers to stm32f4xx_hal_flash.o(.bss) for pFlash
    stm32f4xx_hal_rcc.o(.text) refers to stm32f4xx_hal.o(.text) for HAL_GetTick
    stm32f4xx_hal_rcc.o(.text) refers to stm32f4xx_hal_gpio.o(.text) for HAL_GPIO_Init
    stm32f4xx_hal_rcc.o(.text) refers to stm32f4xx_hal_rcc.o(.constdata) for APBAHBPrescTable
    stm32f4xx_hal_rcc.o(.text) refers to system_stm32f4xx.o(.data) for SystemCoreClock
    stm32f4xx_hal_adc.o(.text) refers to stm32f4xx_hal_msp.o(.text) for HAL_ADC_MspInit
    stm32f4xx_hal_adc.o(.text) refers to stm32f4xx_hal.o(.text) for HAL_GetTick
    stm32f4xx_hal_adc.o(.text) refers to system_stm32f4xx.o(.data) for SystemCoreClock
    stm32f4xx_hal_adc.o(.text) refers to stm32f4xx_hal_adc_ex.o(.text) for HAL_ADCEx_InjectedConvCpltCallback
    stm32f4xx_hal_adc.o(.text) refers to stm32f4xx_hal_dma.o(.text) for HAL_DMA_Start_IT
    stm32f4xx_hal_flash.o(.text) refers to stm32f4xx_hal.o(.text) for HAL_GetTick
    stm32f4xx_hal_flash.o(.text) refers to stm32f4xx_hal_flash_ex.o(.text) for FLASH_Erase_Sector
    stm32f4xx_hal_flash.o(.text) refers to stm32f4xx_hal_flash.o(.bss) for pFlash
    stm32f4xx_hal.o(.text) refers to stm32f4xx_hal_rcc.o(.text) for HAL_RCC_GetHCLKFreq
    stm32f4xx_hal.o(.text) refers to stm32f4xx_hal_cortex.o(.text) for HAL_SYSTICK_Config
    stm32f4xx_hal.o(.text) refers to stm32f4xx_hal.o(.data) for uwTick
    stm32f4xx_hal_i2c.o(.text) refers to stm32f4xx_hal_rcc.o(.text) for HAL_RCC_GetPCLK1Freq
    stm32f4xx_hal_i2c.o(.text) refers to stm32f4xx_hal.o(.text) for HAL_GetTick
    stm32f4xx_hal_i2c.o(.text) refers to stm32f4xx_hal_dma.o(.text) for HAL_DMA_Start_IT
    stm32f4xx_hal_adc_ex.o(.text) refers to stm32f4xx_hal.o(.text) for HAL_GetTick
    stm32f4xx_hal_adc_ex.o(.text) refers to stm32f4xx_hal_adc.o(.text) for HAL_ADC_ErrorCallback
    stm32f4xx_hal_adc_ex.o(.text) refers to system_stm32f4xx.o(.data) for SystemCoreClock
    stm32f4xx_hal_adc_ex.o(.text) refers to stm32f4xx_hal_dma.o(.text) for HAL_DMA_Start_IT
    stm32f4xx_hal_eth.o(.text) refers to stm32f4xx_hal.o(.text) for HAL_Delay
    stm32f4xx_hal_eth.o(.text) refers to ethernetif.o(.text) for HAL_ETH_MspInit
    stm32f4xx_hal_eth.o(.text) refers to stm32f4xx_hal_rcc.o(.text) for HAL_RCC_GetHCLKFreq
    stm32f4xx_hal_dma.o(.text) refers to stm32f4xx_hal.o(.text) for HAL_GetTick
    stm32f4xx_hal_dma.o(.text) refers to stm32f4xx_hal_dma.o(.constdata) for flagBitshiftOffset
    stm32f4xx_hal_iwdg.o(.text) refers to stm32f4xx_hal.o(.text) for HAL_GetTick
    stm32f4xx_hal_rtc.o(.text) refers to stm32f4xx_hal.o(.text) for HAL_GetTick
    stm32f4xx_hal_rtc.o(.text) refers to stm32f4xx_hal_rtc_ex.o(.text) for HAL_RTCEx_AlarmBEventCallback
    stm32f4xx_hal_rtc_ex.o(.text) refers to stm32f4xx_hal_rtc.o(.text) for RTC_Bcd2ToByte
    stm32f4xx_hal_rtc_ex.o(.text) refers to stm32f4xx_hal.o(.text) for HAL_GetTick
    stm32f4xx_hal_tim.o(.text) refers to stm32f4xx_hal_dma.o(.text) for HAL_DMA_Start_IT
    stm32f4xx_hal_tim.o(.text) refers to stm32f4xx_hal_tim_ex.o(.text) for HAL_TIMEx_BreakCallback
    stm32f4xx_hal_tim_ex.o(.text) refers to stm32f4xx_hal_tim.o(.text) for TIM_Base_SetConfig
    stm32f4xx_hal_tim_ex.o(.text) refers to stm32f4xx_hal_dma.o(.text) for HAL_DMA_Start_IT
    stm32f4xx_hal_spi.o(.text) refers to stm32f4xx_hal.o(.text) for HAL_GetTick
    stm32f4xx_hal_spi.o(.text) refers to stm32f4xx_hal_dma.o(.text) for HAL_DMA_Start_IT
    startup_stm32f407xx.o(RESET) refers to startup_stm32f407xx.o(STACK) for __initial_sp
    startup_stm32f407xx.o(RESET) refers to startup_stm32f407xx.o(.text) for Reset_Handler
    startup_stm32f407xx.o(RESET) refers to stm32f4xx_it.o(.text) for NMI_Handler
    startup_stm32f407xx.o(RESET) refers to process2.o(.text) for TIM6_DAC_IRQHandler
    startup_stm32f407xx.o(.text) refers to system_stm32f4xx.o(.text) for SystemInit
    startup_stm32f407xx.o(.text) refers to entry.o(.ARM.Collect$$$$00000000) for __main
    stm32f4xx_hal_msp.o(.text) refers to stm32f4xx_hal_gpio.o(.text) for HAL_GPIO_Init
    ethernetif.o(.text) refers to stm32f4xx_hal_eth.o(.text) for HAL_ETH_Init
    ethernetif.o(.text) refers to memcpya.o(.text) for __aeabi_memcpy
    ethernetif.o(.text) refers to pbuf.o(.text) for pbuf_alloc
    ethernetif.o(.text) refers to stm32f4xx_hal.o(.text) for HAL_GetTick
    ethernetif.o(.text) refers to netif.o(.text) for netif_set_link_up
    ethernetif.o(.text) refers to ethernetif.o(.bss) for EthHandle
    ethernetif.o(.text) refers to ethernetif.o(.data) for lnetif
    ethernetif.o(.text) refers to etharp.o(.text) for etharp_output
    ethernetif.o(.text) refers to app_ethernet.o(.text) for ethernetif_notify_conn_changed
    main.o(.text) refers to netif.o(.text) for netif_add
    main.o(.text) refers to init_l.o(.text) for Init_Config
    main.o(.text) refers to init.o(.text) for lwip_init
    main.o(.text) refers to stm32f4xx_hal.o(.text) for HAL_Delay
    main.o(.text) refers to httpd.o(.text) for httpd_init
    main.o(.text) refers to telnet.o(.text) for Telnet_init
    main.o(.text) refers to app_ethernet.o(.text) for User_notification
    main.o(.text) refers to stm32f4xx_hal_pwr.o(.text) for HAL_PWR_EnableBkUpAccess
    main.o(.text) refers to stm32f4xx_hal_rcc.o(.text) for HAL_RCC_OscConfig
    main.o(.text) refers to process2.o(.text) for main2
    main.o(.text) refers to etharp.o(.text) for ethernet_input
    main.o(.text) refers to ethernetif.o(.text) for ethernetif_init
    main.o(.text) refers to main.o(.bss) for gnetif
    stm32f4xx_it.o(.text) refers to stm32f4xx_hal_tim.o(.text) for HAL_TIM_IRQHandler
    stm32f4xx_it.o(.text) refers to stm32f4xx_hal_adc_ex.o(.text) for HAL_ADCEx_InjectedGetValue
    stm32f4xx_it.o(.text) refers to rc5_ir_emul_receiver.o(.text) for RC5_Sample_Data
    stm32f4xx_it.o(.text) refers to stm32f4xx_hal_gpio.o(.text) for HAL_GPIO_EXTI_IRQHandler
    stm32f4xx_it.o(.text) refers to stm32f4xx_hal_adc.o(.text) for HAL_ADC_Stop_DMA
    stm32f4xx_it.o(.text) refers to uldiv.o(.text) for __aeabi_uldivmod
    stm32f4xx_it.o(.text) refers to dfltul.o(.text) for __aeabi_ul2d
    stm32f4xx_it.o(.text) refers to sqrt.o(i.__hardfp_sqrt) for __hardfp_sqrt
    stm32f4xx_it.o(.text) refers to dfixui.o(.text) for __aeabi_d2uiz
    stm32f4xx_it.o(.text) refers to ethernetif.o(.text) for ethernetif_set_link
    stm32f4xx_it.o(.text) refers to stm32f4xx_hal.o(.text) for HAL_IncTick
    stm32f4xx_it.o(.text) refers to process2.o(.data) for Timer_flag
    stm32f4xx_it.o(.text) refers to lab.o(.bss) for TimHandle50ms
    stm32f4xx_it.o(.text) refers to stm32f4xx_it.o(.data) for ADC_5_acc
    stm32f4xx_it.o(.text) refers to lab.o(.data) for ADC_5
    stm32f4xx_it.o(.text) refers to main.o(.bss) for gnetif
    app_ethernet.o(.text) refers to netif.o(.text) for netif_set_addr
    httpd_cgi_ssi.o(.text) refers to httpd.o(.text) for http_set_cgi_handlers
    httpd_cgi_ssi.o(.text) refers to httpd_cgi_ssi.o(.data) for CGI_TAB
    httpd_cgi_ssi.o(.text) refers to httpd_cgi_ssi.o(.constdata) for LEDS_CGI
    httpd_cgi_ssi.o(.constdata) refers to httpd_cgi_ssi.o(.conststring) for .conststring
    httpd_cgi_ssi.o(.constdata) refers to httpd_cgi_ssi.o(.text) for RC5_CGI_Handler
    httpd_cgi_ssi.o(.data) refers to httpd_cgi_ssi.o(.conststring) for .conststring
    httpd.o(.text) refers to strlen.o(.text) for strlen
    httpd.o(.text) refers to strncmp.o(.text) for strncmp
    httpd.o(.text) refers to mem.o(.text) for mem_malloc
    httpd.o(.text) refers to memseta.o(.text) for __aeabi_memclr4
    httpd.o(.text) refers to fs.o(.text) for fs_close
    httpd.o(.text) refers to tcp_out.o(.text) for tcp_write
    httpd.o(.text) refers to strcmp.o(.text) for strcmp
    httpd.o(.text) refers to memcpya.o(.text) for __aeabi_memcpy4
    httpd.o(.text) refers to httpd.o(.data) for g_pfnSSIHandler
    httpd.o(.text) refers to httpd.o(.constdata) for g_pcTagLeadIn
    httpd.o(.text) refers to strcpy.o(.text) for strcpy
    httpd.o(.text) refers to tcp.o(.text) for tcp_arg
    httpd.o(.text) refers to httpd.o(.bss) for post_buffer
    httpd.o(.text) refers to strchr.o(.text) for strchr
    httpd.o(.text) refers to strstr.o(.text) for strstr
    httpd.o(.text) refers to process2.o(.data) for First_WEB
    httpd.o(.text) refers to rc5_ir_emul_receiver.o(.text) for RC5_CGI
    httpd.o(.text) refers to pbuf.o(.text) for pbuf_free
    httpd.o(.text) refers to atoi.o(.text) for atoi
    httpd.o(.text) refers to process2.o(.text) for PrintToLCD
    httpd.o(.text) refers to process2.o(.bss) for WEB_Arr
    httpd.o(.text) refers to printfa.o(i.__0sprintf) for __2sprintf
    httpd.o(.text) refers to strcspn.o(.text) for strcspn
    httpd.o(.text) refers to httpd_cgi_ssi.o(.text) for httpd_ssi_init
    httpd.o(.text) refers to ip_addr.o(.constdata) for ip_addr_any
    httpd.o(.constdata) refers to httpd.o(.conststring) for .conststring
    httpd.o(.data) refers to httpd.o(.conststring) for .conststring
    fs.o(.text) refers to strcmp.o(.text) for strcmp
    fs.o(.text) refers to memcpya.o(.text) for __aeabi_memcpy
    fs.o(.text) refers to fs.o(.bss) for fs_memory
    fs.o(.text) refers to fs.o(.constdata) for file__style_css
    stm324xg_eval.o(.text) refers to stm32f4xx_hal_i2c.o(.text) for HAL_I2C_DeInit
    stm324xg_eval.o(.text) refers to lab.o(.bss) for hi2c1
    stm324xg_eval_eeprom.o(.text) refers to stm324xg_eval.o(.text) for EEPROM_IO_Init
    stm324xg_eval_eeprom.o(.text) refers to stm324xg_eval_eeprom.o(.data) for EEPROMDataWrite
    init_l.o(.text) refers to stm32f4xx_hal_rtc.o(.text) for HAL_RTC_Init
    init_l.o(.text) refers to stm32f4xx_hal_cortex.o(.text) for HAL_NVIC_SetPriority
    init_l.o(.text) refers to stm32f4xx_hal_dma.o(.text) for HAL_DMA_Init
    init_l.o(.text) refers to stm32f4xx_hal_adc.o(.text) for HAL_ADC_Init
    init_l.o(.text) refers to stm32f4xx_hal_adc_ex.o(.text) for HAL_ADCEx_InjectedConfigChannel
    init_l.o(.text) refers to stm32f4xx_hal_i2c.o(.text) for HAL_I2C_GetState
    init_l.o(.text) refers to onewire.o(.text) for OW_Search
    init_l.o(.text) refers to stm32f4xx_hal_tim.o(.text) for HAL_TIM_PWM_Init
    init_l.o(.text) refers to stm32f4xx_hal_tim_ex.o(.text) for HAL_TIMEx_MasterConfigSynchronization
    init_l.o(.text) refers to lab.o(.bss) for RtcHandle
    init_l.o(.text) refers to init_l.o(.data) for er
    init_l.o(.text) refers to init_l.o(.bss) for hdma_adc
    init_l.o(.text) refers to stm32f4xx_hal_gpio.o(.text) for HAL_GPIO_Init
    init_l.o(.text) refers to stm32f4xx_hal.o(.text) for HAL_Delay
    init_l.o(.text) refers to lcd_g.o(.text) for TM_ILI9341_Init
    init_l.o(.text) refers to rc5_ir_emul_receiver.o(.text) for RC5_Receiver_Init
    init_l.o(.text) refers to stm32f4xx_hal_iwdg.o(.text) for HAL_IWDG_Init
    init_l.o(.text) refers to stm32f4xx_hal_spi.o(.text) for HAL_SPI_GetState
    lab.o(.text) refers to ldiv.o(.text) for __aeabi_ldivmod
    lab.o(.text) refers to lcd_g.o(.text) for TM_ILI9341_Fill
    lab.o(.text) refers to process2.o(.text) for PrintToLCD
    lab.o(.text) refers to stm32f4xx_hal_tim.o(.text) for HAL_TIM_Base_Stop_IT
    lab.o(.text) refers to process2.o(.data) for stop_start
    lab.o(.text) refers to lab.o(.data) for time_loc
    lab.o(.text) refers to img.o(.data) for pump_image
    lab.o(.text) refers to lab.o(.bss) for SpiHandle
    lab.o(.text) refers to printfa.o(i.__0sprintf) for __2sprintf
    onewire.o(.text) refers to stm32f4xx_hal_i2c.o(.text) for HAL_I2C_Master_Transmit
    onewire.o(.text) refers to onewire.o(.bss) for OW_SEARCH_BUFFER
    process2.o(.text) refers to stm32f4xx_hal_cortex.o(.text) for HAL_NVIC_DisableIRQ
    process2.o(.text) refers to stm32f4xx_hal_gpio.o(.text) for HAL_GPIO_WritePin
    process2.o(.text) refers to lcd_g.o(.text) for TM_ILI9341_Fill
    process2.o(.text) refers to printfa.o(i.__0sprintf) for __2sprintf
    process2.o(.text) refers to f2d.o(.text) for __aeabi_f2d
    process2.o(.text) refers to lab.o(.bss) for TimHandlePWM_Motor
    process2.o(.text) refers to process2.o(.data) for OCR_Motor
    process2.o(.text) refers to lab.o(.data) for Triac_Power_Val
    process2.o(.text) refers to process2.o(.bss) for End_LCD_Print
    process2.o(.text) refers to cdcmple.o(.text) for __aeabi_cdcmple
    process2.o(.text) refers to dadd.o(.text) for __aeabi_dsub
    process2.o(.text) refers to d2f.o(.text) for __aeabi_d2f
    process2.o(.text) refers to cdrcmple.o(.text) for __aeabi_cdrcmple
    process2.o(.text) refers to lab.o(.text) for Interpolation
    process2.o(.text) refers to dfltui.o(.text) for __aeabi_ui2d
    process2.o(.text) refers to dmul.o(.text) for __aeabi_dmul
    process2.o(.text) refers to onewire.o(.text) for Read_ds18b20
    process2.o(.text) refers to process2.o(.constdata) for arr_spirt
    process2.o(.text) refers to ffltul.o(.text) for __aeabi_ul2f
    process2.o(.text) refers to memseta.o(.text) for __aeabi_memclr
    process2.o(.text) refers to memcpya.o(.text) for __aeabi_memcpy
    process2.o(.text) refers to tm_stm32f4_fonts.o(.data) for TM_Font_11x18
    process2.o(.text) refers to onewire.o(.bss) for OW_SEARCH_BUFFER
    process2.o(.text) refers to stm32f4xx_hal_iwdg.o(.text) for HAL_IWDG_Refresh
    process2.o(.text) refers to memcmp.o(.text) for memcmp
    process2.o(.text) refers to rc5_ir_emul_receiver.o(.data) for RC5_Frame
    process2.o(.text) refers to strcmp.o(.text) for strcmp
    process2.o(.text) refers to stm32f4xx_hal_rtc.o(.text) for HAL_RTC_SetTime
    process2.o(.text) refers to stm324xg_eval_eeprom.o(.text) for BSP_EEPROM_WriteBuffer
    process2.o(.text) refers to stm32f4xx_hal.o(.text) for HAL_Delay
    process2.o(.text) refers to rc5_ir_emul_receiver.o(.text) for RC5_Decode
    process2.o(.text) refers to ethernetif.o(.text) for ethernetif_input
    process2.o(.text) refers to lwip_timers.o(.text) for sys_check_timeouts
    process2.o(.text) refers to stm32f4xx_hal_tim.o(.text) for HAL_TIM_IRQHandler
    process2.o(.text) refers to main.o(.bss) for gnetif
    process2.o(.text) refers to process2.o(.conststring) for .conststring
    process2.o(.constdata) refers to process2.o(.data) for auto_menu
    process2.o(.constdata) refers to lab.o(.data) for hour
    process2.o(.data) refers to process2.o(.conststring) for .conststring
    rc5_ir_emul_receiver.o(.text) refers to stm32f4xx_hal_tim.o(.text) for HAL_TIM_Base_Init
    rc5_ir_emul_receiver.o(.text) refers to stm32f4xx_hal_rcc.o(.text) for HAL_RCC_GetPCLK1Freq
    rc5_ir_emul_receiver.o(.text) refers to stm32f4xx_hal_gpio.o(.text) for HAL_GPIO_EXTI_IRQHandler
    rc5_ir_emul_receiver.o(.text) refers to atoi.o(.text) for atoi
    rc5_ir_emul_receiver.o(.text) refers to rc5_ir_emul_receiver.o(.data) for Disable_Ext
    rc5_ir_emul_receiver.o(.text) refers to rc5_ir_emul_receiver.o(.bss) for TimHandle
    rc5_ir_emul_receiver.o(.text) refers to stm32f4xx_hal.o(.text) for HAL_Delay
    rc5_ir_emul_receiver.o(.text) refers to stm324xg_eval_eeprom.o(.text) for BSP_EEPROM_WriteBuffer
    rc5_ir_emul_receiver.o(.data) refers to rc5_ir_emul_receiver.o(.conststring) for .conststring
    telnet.o(.text) refers to memseta.o(.text) for __aeabi_memclr4
    telnet.o(.text) refers to tcp.o(.text) for tcp_recved
    telnet.o(.text) refers to pbuf.o(.text) for pbuf_free
    telnet.o(.text) refers to memcmp.o(.text) for memcmp
    telnet.o(.text) refers to process2.o(.text) for Get_Buffer_Telnet
    telnet.o(.text) refers to tcp_out.o(.text) for tcp_write
    telnet.o(.text) refers to mem.o(.text) for mem_free
    telnet.o(.text) refers to ip_addr.o(.constdata) for ip_addr_any
    lcd_g.o(.text) refers to stm32f4xx_hal_spi.o(.text) for HAL_SPI_Init
    lcd_g.o(.text) refers to stm32f4xx_hal_gpio.o(.text) for HAL_GPIO_WritePin
    lcd_g.o(.text) refers to init_l.o(.text) for SPI_Init
    lcd_g.o(.text) refers to stm32f4xx_hal.o(.text) for HAL_Delay
    lcd_g.o(.text) refers to lab.o(.bss) for SpiHandle
    lcd_g.o(.text) refers to lcd_g.o(.data) for ILI9341_x
    lcd_g.o(.text) refers to tm_stm32f4_fonts.o(.data) for UB_Font_Font_16x27
    tm_stm32f4_fonts.o(.text) refers to strlen.o(.text) for strlen
    tm_stm32f4_fonts.o(.data) refers to tm_stm32f4_fonts.o(.constdata) for TM_Font7x10
    img.o(.data) refers to img.o(.conststring) for .conststring
    sqrt.o(i.__hardfp_sqrt) refers (Special) to iusefp.o(.text) for __I$use$fp
    sqrt.o(i.__hardfp_sqrt) refers to dsqrt.o(.text) for _dsqrt
    sqrt.o(i.__hardfp_sqrt) refers to errno.o(i.__set_errno) for __set_errno
    sqrt.o(i.__softfp_sqrt) refers (Special) to iusefp.o(.text) for __I$use$fp
    sqrt.o(i.__softfp_sqrt) refers to dsqrt.o(.text) for _dsqrt
    sqrt.o(i.__softfp_sqrt) refers to errno.o(i.__set_errno) for __set_errno
    sqrt.o(i.sqrt) refers (Special) to iusefp.o(.text) for __I$use$fp
    sqrt.o(i.sqrt) refers to dsqrt.o(.text) for _dsqrt
    sqrt.o(i.sqrt) refers to errno.o(i.__set_errno) for __set_errno
    sqrt_x.o(i.____hardfp_sqrt$lsc) refers (Special) to iusefp.o(.text) for __I$use$fp
    sqrt_x.o(i.____hardfp_sqrt$lsc) refers to cdcmple.o(.text) for __aeabi_cdcmple
    sqrt_x.o(i.____hardfp_sqrt$lsc) refers to errno.o(i.__set_errno) for __set_errno
    sqrt_x.o(i.____hardfp_sqrt$lsc) refers to dsqrt.o(.text) for _dsqrt
    sqrt_x.o(i.____softfp_sqrt$lsc) refers (Special) to iusefp.o(.text) for __I$use$fp
    sqrt_x.o(i.____softfp_sqrt$lsc) refers to cdcmple.o(.text) for __aeabi_cdcmple
    sqrt_x.o(i.____softfp_sqrt$lsc) refers to errno.o(i.__set_errno) for __set_errno
    sqrt_x.o(i.____softfp_sqrt$lsc) refers to dsqrt.o(.text) for _dsqrt
    sqrt_x.o(i.__sqrt$lsc) refers (Special) to iusefp.o(.text) for __I$use$fp
    sqrt_x.o(i.__sqrt$lsc) refers to cdcmple.o(.text) for __aeabi_cdcmple
    sqrt_x.o(i.__sqrt$lsc) refers to errno.o(i.__set_errno) for __set_errno
    sqrt_x.o(i.__sqrt$lsc) refers to dsqrt.o(.text) for _dsqrt
    entry.o(.ARM.Collect$$$$00000000) refers (Special) to entry10a.o(.ARM.Collect$$$$0000000D) for __rt_final_cpp
    entry.o(.ARM.Collect$$$$00000000) refers (Special) to entry11a.o(.ARM.Collect$$$$0000000F) for __rt_final_exit
    entry.o(.ARM.Collect$$$$00000000) refers (Special) to entry7b.o(.ARM.Collect$$$$00000008) for _main_clock
    entry.o(.ARM.Collect$$$$00000000) refers (Special) to entry8b.o(.ARM.Collect$$$$0000000A) for _main_cpp_init
    entry.o(.ARM.Collect$$$$00000000) refers (Special) to entry9a.o(.ARM.Collect$$$$0000000B) for _main_init
    entry.o(.ARM.Collect$$$$00000000) refers (Special) to entry5.o(.ARM.Collect$$$$00000004) for _main_scatterload
    entry.o(.ARM.Collect$$$$00000000) refers (Special) to entry2.o(.ARM.Collect$$$$00000001) for _main_stk
    uldiv.o(.text) refers to llushr.o(.text) for __aeabi_llsr
    uldiv.o(.text) refers to llshl.o(.text) for __aeabi_llsl
    ldiv.o(.text) refers to uldiv.o(.text) for __aeabi_uldivmod
    printfb.o(i.__0fprintf$bare) refers to printfb.o(i._printf_core) for _printf_core
    printfb.o(i.__0fprintf$bare) refers to fputc.o(i.fputc) for fputc
    printfb.o(i.__0printf$bare) refers to printfb.o(i._printf_core) for _printf_core
    printfb.o(i.__0printf$bare) refers to fputc.o(i.fputc) for fputc
    printfb.o(i.__0printf$bare) refers to stdout.o(.data) for __stdout
    printfb.o(i.__0snprintf$bare) refers to printfb.o(i._printf_core) for _printf_core
    printfb.o(i.__0snprintf$bare) refers to printfb.o(i._snputc) for _snputc
    printfb.o(i.__0sprintf$bare) refers to printfb.o(i._printf_core) for _printf_core
    printfb.o(i.__0sprintf$bare) refers to printfb.o(i._sputc) for _sputc
    printfb.o(i.__0vfprintf$bare) refers to printfb.o(i._printf_core) for _printf_core
    printfb.o(i.__0vfprintf$bare) refers to fputc.o(i.fputc) for fputc
    printfb.o(i.__0vprintf$bare) refers to printfb.o(i._printf_core) for _printf_core
    printfb.o(i.__0vprintf$bare) refers to fputc.o(i.fputc) for fputc
    printfb.o(i.__0vprintf$bare) refers to stdout.o(.data) for __stdout
    printfb.o(i.__0vsnprintf$bare) refers to printfb.o(i._printf_core) for _printf_core
    printfb.o(i.__0vsnprintf$bare) refers to printfb.o(i._snputc) for _snputc
    printfb.o(i.__0vsprintf$bare) refers to printfb.o(i._printf_core) for _printf_core
    printfb.o(i.__0vsprintf$bare) refers to printfb.o(i._sputc) for _sputc
    printf0.o(i.__0fprintf$0) refers to printf0.o(i._printf_core) for _printf_core
    printf0.o(i.__0fprintf$0) refers to fputc.o(i.fputc) for fputc
    printf0.o(i.__0printf$0) refers to printf0.o(i._printf_core) for _printf_core
    printf0.o(i.__0printf$0) refers to fputc.o(i.fputc) for fputc
    printf0.o(i.__0printf$0) refers to stdout.o(.data) for __stdout
    printf0.o(i.__0snprintf$0) refers to printf0.o(i._printf_core) for _printf_core
    printf0.o(i.__0snprintf$0) refers to printf0.o(i._snputc) for _snputc
    printf0.o(i.__0sprintf$0) refers to printf0.o(i._printf_core) for _printf_core
    printf0.o(i.__0sprintf$0) refers to printf0.o(i._sputc) for _sputc
    printf0.o(i.__0vfprintf$0) refers to printf0.o(i._printf_core) for _printf_core
    printf0.o(i.__0vfprintf$0) refers to fputc.o(i.fputc) for fputc
    printf0.o(i.__0vprintf$0) refers to printf0.o(i._printf_core) for _printf_core
    printf0.o(i.__0vprintf$0) refers to fputc.o(i.fputc) for fputc
    printf0.o(i.__0vprintf$0) refers to stdout.o(.data) for __stdout
    printf0.o(i.__0vsnprintf$0) refers to printf0.o(i._printf_core) for _printf_core
    printf0.o(i.__0vsnprintf$0) refers to printf0.o(i._snputc) for _snputc
    printf0.o(i.__0vsprintf$0) refers to printf0.o(i._printf_core) for _printf_core
    printf0.o(i.__0vsprintf$0) refers to printf0.o(i._sputc) for _sputc
    printf1.o(i.__0fprintf$1) refers to printf1.o(i._printf_core) for _printf_core
    printf1.o(i.__0fprintf$1) refers to fputc.o(i.fputc) for fputc
    printf1.o(i.__0printf$1) refers to printf1.o(i._printf_core) for _printf_core
    printf1.o(i.__0printf$1) refers to fputc.o(i.fputc) for fputc
    printf1.o(i.__0printf$1) refers to stdout.o(.data) for __stdout
    printf1.o(i.__0snprintf$1) refers to printf1.o(i._printf_core) for _printf_core
    printf1.o(i.__0snprintf$1) refers to printf1.o(i._snputc) for _snputc
    printf1.o(i.__0sprintf$1) refers to printf1.o(i._printf_core) for _printf_core
    printf1.o(i.__0sprintf$1) refers to printf1.o(i._sputc) for _sputc
    printf1.o(i.__0vfprintf$1) refers to printf1.o(i._printf_core) for _printf_core
    printf1.o(i.__0vfprintf$1) refers to fputc.o(i.fputc) for fputc
    printf1.o(i.__0vprintf$1) refers to printf1.o(i._printf_core) for _printf_core
    printf1.o(i.__0vprintf$1) refers to fputc.o(i.fputc) for fputc
    printf1.o(i.__0vprintf$1) refers to stdout.o(.data) for __stdout
    printf1.o(i.__0vsnprintf$1) refers to printf1.o(i._printf_core) for _printf_core
    printf1.o(i.__0vsnprintf$1) refers to printf1.o(i._snputc) for _snputc
    printf1.o(i.__0vsprintf$1) refers to printf1.o(i._printf_core) for _printf_core
    printf1.o(i.__0vsprintf$1) refers to printf1.o(i._sputc) for _sputc
    printf1.o(i._printf_core) refers to uidiv.o(.text) for __aeabi_uidivmod
    printf2.o(i.__0fprintf$2) refers to printf2.o(i._printf_core) for _printf_core
    printf2.o(i.__0fprintf$2) refers to fputc.o(i.fputc) for fputc
    printf2.o(i.__0printf$2) refers to printf2.o(i._printf_core) for _printf_core
    printf2.o(i.__0printf$2) refers to fputc.o(i.fputc) for fputc
    printf2.o(i.__0printf$2) refers to stdout.o(.data) for __stdout
    printf2.o(i.__0snprintf$2) refers to printf2.o(i._printf_core) for _printf_core
    printf2.o(i.__0snprintf$2) refers to printf2.o(i._snputc) for _snputc
    printf2.o(i.__0sprintf$2) refers to printf2.o(i._printf_core) for _printf_core
    printf2.o(i.__0sprintf$2) refers to printf2.o(i._sputc) for _sputc
    printf2.o(i.__0vfprintf$2) refers to printf2.o(i._printf_core) for _printf_core
    printf2.o(i.__0vfprintf$2) refers to fputc.o(i.fputc) for fputc
    printf2.o(i.__0vprintf$2) refers to printf2.o(i._printf_core) for _printf_core
    printf2.o(i.__0vprintf$2) refers to fputc.o(i.fputc) for fputc
    printf2.o(i.__0vprintf$2) refers to stdout.o(.data) for __stdout
    printf2.o(i.__0vsnprintf$2) refers to printf2.o(i._printf_core) for _printf_core
    printf2.o(i.__0vsnprintf$2) refers to printf2.o(i._snputc) for _snputc
    printf2.o(i.__0vsprintf$2) refers to printf2.o(i._printf_core) for _printf_core
    printf2.o(i.__0vsprintf$2) refers to printf2.o(i._sputc) for _sputc
    printf3.o(i.__0fprintf$3) refers to printf3.o(i._printf_core) for _printf_core
    printf3.o(i.__0fprintf$3) refers to fputc.o(i.fputc) for fputc
    printf3.o(i.__0printf$3) refers to printf3.o(i._printf_core) for _printf_core
    printf3.o(i.__0printf$3) refers to fputc.o(i.fputc) for fputc
    printf3.o(i.__0printf$3) refers to stdout.o(.data) for __stdout
    printf3.o(i.__0snprintf$3) refers to printf3.o(i._printf_core) for _printf_core
    printf3.o(i.__0snprintf$3) refers to printf3.o(i._snputc) for _snputc
    printf3.o(i.__0sprintf$3) refers to printf3.o(i._printf_core) for _printf_core
    printf3.o(i.__0sprintf$3) refers to printf3.o(i._sputc) for _sputc
    printf3.o(i.__0vfprintf$3) refers to printf3.o(i._printf_core) for _printf_core
    printf3.o(i.__0vfprintf$3) refers to fputc.o(i.fputc) for fputc
    printf3.o(i.__0vprintf$3) refers to printf3.o(i._printf_core) for _printf_core
    printf3.o(i.__0vprintf$3) refers to fputc.o(i.fputc) for fputc
    printf3.o(i.__0vprintf$3) refers to stdout.o(.data) for __stdout
    printf3.o(i.__0vsnprintf$3) refers to printf3.o(i._printf_core) for _printf_core
    printf3.o(i.__0vsnprintf$3) refers to printf3.o(i._snputc) for _snputc
    printf3.o(i.__0vsprintf$3) refers to printf3.o(i._printf_core) for _printf_core
    printf3.o(i.__0vsprintf$3) refers to printf3.o(i._sputc) for _sputc
    printf3.o(i._printf_core) refers to uidiv.o(.text) for __aeabi_uidivmod
    printf4.o(i.__0fprintf$4) refers to printf4.o(i._printf_core) for _printf_core
    printf4.o(i.__0fprintf$4) refers to fputc.o(i.fputc) for fputc
    printf4.o(i.__0printf$4) refers to printf4.o(i._printf_core) for _printf_core
    printf4.o(i.__0printf$4) refers to fputc.o(i.fputc) for fputc
    printf4.o(i.__0printf$4) refers to stdout.o(.data) for __stdout
    printf4.o(i.__0snprintf$4) refers to printf4.o(i._printf_core) for _printf_core
    printf4.o(i.__0snprintf$4) refers to printf4.o(i._snputc) for _snputc
    printf4.o(i.__0sprintf$4) refers to printf4.o(i._printf_core) for _printf_core
    printf4.o(i.__0sprintf$4) refers to printf4.o(i._sputc) for _sputc
    printf4.o(i.__0vfprintf$4) refers to printf4.o(i._printf_core) for _printf_core
    printf4.o(i.__0vfprintf$4) refers to fputc.o(i.fputc) for fputc
    printf4.o(i.__0vprintf$4) refers to printf4.o(i._printf_core) for _printf_core
    printf4.o(i.__0vprintf$4) refers to fputc.o(i.fputc) for fputc
    printf4.o(i.__0vprintf$4) refers to stdout.o(.data) for __stdout
    printf4.o(i.__0vsnprintf$4) refers to printf4.o(i._printf_core) for _printf_core
    printf4.o(i.__0vsnprintf$4) refers to printf4.o(i._snputc) for _snputc
    printf4.o(i.__0vsprintf$4) refers to printf4.o(i._printf_core) for _printf_core
    printf4.o(i.__0vsprintf$4) refers to printf4.o(i._sputc) for _sputc
    printf4.o(i._printf_core) refers to uldiv.o(.text) for __aeabi_uldivmod
    printf5.o(i.__0fprintf$5) refers to printf5.o(i._printf_core) for _printf_core
    printf5.o(i.__0fprintf$5) refers to fputc.o(i.fputc) for fputc
    printf5.o(i.__0printf$5) refers to printf5.o(i._printf_core) for _printf_core
    printf5.o(i.__0printf$5) refers to fputc.o(i.fputc) for fputc
    printf5.o(i.__0printf$5) refers to stdout.o(.data) for __stdout
    printf5.o(i.__0snprintf$5) refers to printf5.o(i._printf_core) for _printf_core
    printf5.o(i.__0snprintf$5) refers to printf5.o(i._snputc) for _snputc
    printf5.o(i.__0sprintf$5) refers to printf5.o(i._printf_core) for _printf_core
    printf5.o(i.__0sprintf$5) refers to printf5.o(i._sputc) for _sputc
    printf5.o(i.__0vfprintf$5) refers to printf5.o(i._printf_core) for _printf_core
    printf5.o(i.__0vfprintf$5) refers to fputc.o(i.fputc) for fputc
    printf5.o(i.__0vprintf$5) refers to printf5.o(i._printf_core) for _printf_core
    printf5.o(i.__0vprintf$5) refers to fputc.o(i.fputc) for fputc
    printf5.o(i.__0vprintf$5) refers to stdout.o(.data) for __stdout
    printf5.o(i.__0vsnprintf$5) refers to printf5.o(i._printf_core) for _printf_core
    printf5.o(i.__0vsnprintf$5) refers to printf5.o(i._snputc) for _snputc
    printf5.o(i.__0vsprintf$5) refers to printf5.o(i._printf_core) for _printf_core
    printf5.o(i.__0vsprintf$5) refers to printf5.o(i._sputc) for _sputc
    printf5.o(i._printf_core) refers to uldiv.o(.text) for __aeabi_uldivmod
    printf6.o(i.__0fprintf$6) refers to printf6.o(i._printf_core) for _printf_core
    printf6.o(i.__0fprintf$6) refers to fputc.o(i.fputc) for fputc
    printf6.o(i.__0printf$6) refers to printf6.o(i._printf_core) for _printf_core
    printf6.o(i.__0printf$6) refers to fputc.o(i.fputc) for fputc
    printf6.o(i.__0printf$6) refers to stdout.o(.data) for __stdout
    printf6.o(i.__0snprintf$6) refers to printf6.o(i._printf_core) for _printf_core
    printf6.o(i.__0snprintf$6) refers to printf6.o(i._snputc) for _snputc
    printf6.o(i.__0sprintf$6) refers to printf6.o(i._printf_core) for _printf_core
    printf6.o(i.__0sprintf$6) refers to printf6.o(i._sputc) for _sputc
    printf6.o(i.__0vfprintf$6) refers to printf6.o(i._printf_core) for _printf_core
    printf6.o(i.__0vfprintf$6) refers to fputc.o(i.fputc) for fputc
    printf6.o(i.__0vprintf$6) refers to printf6.o(i._printf_core) for _printf_core
    printf6.o(i.__0vprintf$6) refers to fputc.o(i.fputc) for fputc
    printf6.o(i.__0vprintf$6) refers to stdout.o(.data) for __stdout
    printf6.o(i.__0vsnprintf$6) refers to printf6.o(i._printf_core) for _printf_core
    printf6.o(i.__0vsnprintf$6) refers to printf6.o(i._snputc) for _snputc
    printf6.o(i.__0vsprintf$6) refers to printf6.o(i._printf_core) for _printf_core
    printf6.o(i.__0vsprintf$6) refers to printf6.o(i._sputc) for _sputc
    printf6.o(i._printf_core) refers to printf6.o(i._printf_pre_padding) for _printf_pre_padding
    printf6.o(i._printf_core) refers to uidiv.o(.text) for __aeabi_uidivmod
    printf6.o(i._printf_core) refers to printf6.o(i._printf_post_padding) for _printf_post_padding
    printf7.o(i.__0fprintf$7) refers to printf7.o(i._printf_core) for _printf_core
    printf7.o(i.__0fprintf$7) refers to fputc.o(i.fputc) for fputc
    printf7.o(i.__0printf$7) refers to printf7.o(i._printf_core) for _printf_core
    printf7.o(i.__0printf$7) refers to fputc.o(i.fputc) for fputc
    printf7.o(i.__0printf$7) refers to stdout.o(.data) for __stdout
    printf7.o(i.__0snprintf$7) refers to printf7.o(i._printf_core) for _printf_core
    printf7.o(i.__0snprintf$7) refers to printf7.o(i._snputc) for _snputc
    printf7.o(i.__0sprintf$7) refers to printf7.o(i._printf_core) for _printf_core
    printf7.o(i.__0sprintf$7) refers to printf7.o(i._sputc) for _sputc
    printf7.o(i.__0vfprintf$7) refers to printf7.o(i._printf_core) for _printf_core
    printf7.o(i.__0vfprintf$7) refers to fputc.o(i.fputc) for fputc
    printf7.o(i.__0vprintf$7) refers to printf7.o(i._printf_core) for _printf_core
    printf7.o(i.__0vprintf$7) refers to fputc.o(i.fputc) for fputc
    printf7.o(i.__0vprintf$7) refers to stdout.o(.data) for __stdout
    printf7.o(i.__0vsnprintf$7) refers to printf7.o(i._printf_core) for _printf_core
    printf7.o(i.__0vsnprintf$7) refers to printf7.o(i._snputc) for _snputc
    printf7.o(i.__0vsprintf$7) refers to printf7.o(i._printf_core) for _printf_core
    printf7.o(i.__0vsprintf$7) refers to printf7.o(i._sputc) for _sputc
    printf7.o(i._printf_core) refers to printf7.o(i._printf_pre_padding) for _printf_pre_padding
    printf7.o(i._printf_core) refers to uldiv.o(.text) for __aeabi_uldivmod
    printf7.o(i._printf_core) refers to printf7.o(i._printf_post_padding) for _printf_post_padding
    printf8.o(i.__0fprintf$8) refers to printf8.o(i._printf_core) for _printf_core
    printf8.o(i.__0fprintf$8) refers to fputc.o(i.fputc) for fputc
    printf8.o(i.__0printf$8) refers to printf8.o(i._printf_core) for _printf_core
    printf8.o(i.__0printf$8) refers to fputc.o(i.fputc) for fputc
    printf8.o(i.__0printf$8) refers to stdout.o(.data) for __stdout
    printf8.o(i.__0snprintf$8) refers to printf8.o(i._printf_core) for _printf_core
    printf8.o(i.__0snprintf$8) refers to printf8.o(i._snputc) for _snputc
    printf8.o(i.__0sprintf$8) refers to printf8.o(i._printf_core) for _printf_core
    printf8.o(i.__0sprintf$8) refers to printf8.o(i._sputc) for _sputc
    printf8.o(i.__0vfprintf$8) refers to printf8.o(i._printf_core) for _printf_core
    printf8.o(i.__0vfprintf$8) refers to fputc.o(i.fputc) for fputc
    printf8.o(i.__0vprintf$8) refers to printf8.o(i._printf_core) for _printf_core
    printf8.o(i.__0vprintf$8) refers to fputc.o(i.fputc) for fputc
    printf8.o(i.__0vprintf$8) refers to stdout.o(.data) for __stdout
    printf8.o(i.__0vsnprintf$8) refers to printf8.o(i._printf_core) for _printf_core
    printf8.o(i.__0vsnprintf$8) refers to printf8.o(i._snputc) for _snputc
    printf8.o(i.__0vsprintf$8) refers to printf8.o(i._printf_core) for _printf_core
    printf8.o(i.__0vsprintf$8) refers to printf8.o(i._sputc) for _sputc
    printf8.o(i._printf_core) refers to printf8.o(i._printf_pre_padding) for _printf_pre_padding
    printf8.o(i._printf_core) refers to uldiv.o(.text) for __aeabi_uldivmod
    printf8.o(i._printf_core) refers to printf8.o(i._printf_post_padding) for _printf_post_padding
    printfa.o(i.__0fprintf) refers (Special) to iusefp.o(.text) for __I$use$fp
    printfa.o(i.__0fprintf) refers to printfa.o(i._printf_core) for _printf_core
    printfa.o(i.__0fprintf) refers to fputc.o(i.fputc) for fputc
    printfa.o(i.__0printf) refers (Special) to iusefp.o(.text) for __I$use$fp
    printfa.o(i.__0printf) refers to printfa.o(i._printf_core) for _printf_core
    printfa.o(i.__0printf) refers to fputc.o(i.fputc) for fputc
    printfa.o(i.__0printf) refers to stdout.o(.data) for __stdout
    printfa.o(i.__0snprintf) refers (Special) to iusefp.o(.text) for __I$use$fp
    printfa.o(i.__0snprintf) refers to printfa.o(i._printf_core) for _printf_core
    printfa.o(i.__0snprintf) refers to printfa.o(i._snputc) for _snputc
    printfa.o(i.__0sprintf) refers (Special) to iusefp.o(.text) for __I$use$fp
    printfa.o(i.__0sprintf) refers to printfa.o(i._printf_core) for _printf_core
    printfa.o(i.__0sprintf) refers to printfa.o(i._sputc) for _sputc
    printfa.o(i.__0vfprintf) refers (Special) to iusefp.o(.text) for __I$use$fp
    printfa.o(i.__0vfprintf) refers to printfa.o(i._printf_core) for _printf_core
    printfa.o(i.__0vfprintf) refers to fputc.o(i.fputc) for fputc
    printfa.o(i.__0vprintf) refers (Special) to iusefp.o(.text) for __I$use$fp
    printfa.o(i.__0vprintf) refers to printfa.o(i._printf_core) for _printf_core
    printfa.o(i.__0vprintf) refers to fputc.o(i.fputc) for fputc
    printfa.o(i.__0vprintf) refers to stdout.o(.data) for __stdout
    printfa.o(i.__0vsnprintf) refers (Special) to iusefp.o(.text) for __I$use$fp
    printfa.o(i.__0vsnprintf) refers to printfa.o(i._printf_core) for _printf_core
    printfa.o(i.__0vsnprintf) refers to printfa.o(i._snputc) for _snputc
    printfa.o(i.__0vsprintf) refers (Special) to iusefp.o(.text) for __I$use$fp
    printfa.o(i.__0vsprintf) refers to printfa.o(i._printf_core) for _printf_core
    printfa.o(i.__0vsprintf) refers to printfa.o(i._sputc) for _sputc
    printfa.o(i._fp_digits) refers (Special) to iusefp.o(.text) for __I$use$fp
    printfa.o(i._fp_digits) refers to dmul.o(.text) for __aeabi_dmul
    printfa.o(i._fp_digits) refers to ddiv.o(.text) for __aeabi_ddiv
    printfa.o(i._fp_digits) refers to cdrcmple.o(.text) for __aeabi_cdrcmple
    printfa.o(i._fp_digits) refers to dadd.o(.text) for __aeabi_dadd
    printfa.o(i._fp_digits) refers to dfixul.o(.text) for __aeabi_d2ulz
    printfa.o(i._fp_digits) refers to uldiv.o(.text) for __aeabi_uldivmod
    printfa.o(i._printf_core) refers (Special) to iusefp.o(.text) for __I$use$fp
    printfa.o(i._printf_core) refers to printfa.o(i._printf_pre_padding) for _printf_pre_padding
    printfa.o(i._printf_core) refers to uldiv.o(.text) for __aeabi_uldivmod
    printfa.o(i._printf_core) refers to printfa.o(i._printf_post_padding) for _printf_post_padding
    printfa.o(i._printf_core) refers to printfa.o(i._fp_digits) for _fp_digits
    printfa.o(i._printf_core) refers to uidiv.o(.text) for __aeabi_uidivmod
    printfa.o(i._printf_post_padding) refers (Special) to iusefp.o(.text) for __I$use$fp
    printfa.o(i._printf_pre_padding) refers (Special) to iusefp.o(.text) for __I$use$fp
    printfa.o(i._snputc) refers (Special) to iusefp.o(.text) for __I$use$fp
    printfa.o(i._sputc) refers (Special) to iusefp.o(.text) for __I$use$fp
    atoi.o(.text) refers to errno.o(i.__aeabi_errno_addr) for __aeabi_errno_addr
    atoi.o(.text) refers to strtol.o(.text) for strtol
    dadd.o(.text) refers (Special) to iusefp.o(.text) for __I$use$fp
    dadd.o(.text) refers to llshl.o(.text) for __aeabi_llsl
    dadd.o(.text) refers to llsshr.o(.text) for __aeabi_lasr
    dadd.o(.text) refers to depilogue.o(.text) for _double_epilogue
    dmul.o(.text) refers (Special) to iusefp.o(.text) for __I$use$fp
    dmul.o(.text) refers to depilogue.o(.text) for _double_epilogue
    ffltul.o(.text) refers (Special) to iusefp.o(.text) for __I$use$fp
    ffltul.o(.text) refers to fepilogue.o(.text) for _float_epilogue
    dfltui.o(.text) refers (Special) to iusefp.o(.text) for __I$use$fp
    dfltui.o(.text) refers to depilogue.o(.text) for _double_epilogue
    dfltul.o(.text) refers (Special) to iusefp.o(.text) for __I$use$fp
    dfltul.o(.text) refers to depilogue.o(.text) for _double_epilogue
    dfixui.o(.text) refers (Special) to iusefp.o(.text) for __I$use$fp
    dfixui.o(.text) refers to llushr.o(.text) for __aeabi_llsr
    f2d.o(.text) refers (Special) to iusefp.o(.text) for __I$use$fp
    cdcmple.o(.text) refers (Special) to iusefp.o(.text) for __I$use$fp
    cdrcmple.o(.text) refers (Special) to iusefp.o(.text) for __I$use$fp
    d2f.o(.text) refers (Special) to iusefp.o(.text) for __I$use$fp
    d2f.o(.text) refers to fepilogue.o(.text) for _float_round
    entry2.o(.ARM.Collect$$$$00000001) refers to entry2.o(.ARM.Collect$$$$00002712) for __lit__00000000
    entry2.o(.ARM.Collect$$$$00002712) refers to startup_stm32f407xx.o(STACK) for __initial_sp
    entry2.o(__vectab_stack_and_reset_area) refers to startup_stm32f407xx.o(STACK) for __initial_sp
    entry2.o(__vectab_stack_and_reset_area) refers to entry.o(.ARM.Collect$$$$00000000) for __main
    entry5.o(.ARM.Collect$$$$00000004) refers to init.o(.text) for __scatterload
    entry9a.o(.ARM.Collect$$$$0000000B) refers to main.o(.text) for main
    entry9b.o(.ARM.Collect$$$$0000000C) refers to main.o(.text) for main
    fputc.o(i.fputc) refers (Special) to iusesemip.o(.text) for __I$use$semihosting$fputc
    fputc.o(i.fputc) refers (Special) to semi.o(.text) for __semihosting_library_function
    errno.o(i.__aeabi_errno_addr) refers to errno.o(.data) for .data
    errno.o(i.__read_errno) refers to errno.o(.data) for .data
    errno.o(i.__set_errno) refers to errno.o(.data) for .data
    strtol.o(.text) refers to ctype_o.o(.text) for __rt_ctype_table
    strtol.o(.text) refers to _strtoul.o(.text) for _strtoul
    strtol.o(.text) refers to errno.o(i.__aeabi_errno_addr) for __aeabi_errno_addr
    depilogue.o(.text) refers to llshl.o(.text) for __aeabi_llsl
    depilogue.o(.text) refers to llushr.o(.text) for __aeabi_llsr
    ddiv.o(.text) refers to depilogue.o(.text) for _double_round
    dsqrt.o(.text) refers to llushr.o(.text) for __aeabi_llsr
    dsqrt.o(.text) refers to depilogue.o(.text) for _double_round
    dfixul.o(.text) refers to llushr.o(.text) for __aeabi_llsr
    dfixul.o(.text) refers to llshl.o(.text) for __aeabi_llsl
    init.o(.text) refers to entry5.o(.ARM.Collect$$$$00000004) for __main_after_scatterload
    ctype_o.o(.text) refers to ctype_o.o(.constdata) for .constdata
    ctype_o.o(.constdata) refers to ctype_o.o(.constdata) for __ctype_table
    isalnum_o.o(.text) refers to ctype_o.o(.text) for __rt_ctype_table
    isalpha_o.o(.text) refers to ctype_o.o(.text) for __rt_ctype_table
    isblank_o.o(.text) refers to ctype_o.o(.constdata) for __ctype_table
    iscntrl_o.o(.text) refers to ctype_o.o(.text) for __rt_ctype_table
    isdigit_o.o(.text) refers to ctype_o.o(.text) for __rt_ctype_table
    isgraph_o.o(.text) refers to ctype_o.o(.text) for __rt_ctype_table
    islower_o.o(.text) refers to ctype_o.o(.text) for __rt_ctype_table
    isprint_o.o(.text) refers to ctype_o.o(.text) for __rt_ctype_table
    ispunct_o.o(.text) refers to ctype_o.o(.text) for __rt_ctype_table
    isspace_o.o(.text) refers to ctype_o.o(.text) for __rt_ctype_table
    isupper_o.o(.text) refers to ctype_o.o(.text) for __rt_ctype_table
    isxdigit_o.o(.text) refers to ctype_o.o(.text) for __rt_ctype_table
    _strtoul.o(.text) refers to _chval.o(.text) for _chval
    _strtoul.o(.text) refers to errno.o(i.__aeabi_errno_addr) for __aeabi_errno_addr


==============================================================================

Removing Unused input sections from the image.

    Removing system_stm32f4xx.o(.rev16_text), (4 bytes).
    Removing system_stm32f4xx.o(.revsh_text), (4 bytes).
    Removing system_stm32f4xx.o(.rrx_text), (6 bytes).
    Removing memp.o(.conststring), (110 bytes).
    Removing memp.o(.data), (40 bytes).
    Removing err.o(.text), (16 bytes).
    Removing err.o(.conststring), (295 bytes).
    Removing err.o(.data), (64 bytes).
    Removing stm32f4xx_hal_flash_ex.o(.rev16_text), (4 bytes).
    Removing stm32f4xx_hal_flash_ex.o(.revsh_text), (4 bytes).
    Removing stm32f4xx_hal_flash_ex.o(.rrx_text), (6 bytes).
    Removing stm32f4xx_hal_flash_ex.o(.text), (1000 bytes).
    Removing stm32f4xx_hal_rcc.o(.rev16_text), (4 bytes).
    Removing stm32f4xx_hal_rcc.o(.revsh_text), (4 bytes).
    Removing stm32f4xx_hal_rcc.o(.rrx_text), (6 bytes).
    Removing stm32f4xx_hal_adc.o(.rev16_text), (4 bytes).
    Removing stm32f4xx_hal_adc.o(.revsh_text), (4 bytes).
    Removing stm32f4xx_hal_adc.o(.rrx_text), (6 bytes).
    Removing stm32f4xx_hal_flash.o(.rev16_text), (4 bytes).
    Removing stm32f4xx_hal_flash.o(.revsh_text), (4 bytes).
    Removing stm32f4xx_hal_flash.o(.rrx_text), (6 bytes).
    Removing stm32f4xx_hal_flash.o(.text), (1156 bytes).
    Removing stm32f4xx_hal_flash.o(.bss), (32 bytes).
    Removing stm32f4xx_hal.o(.rev16_text), (4 bytes).
    Removing stm32f4xx_hal.o(.revsh_text), (4 bytes).
    Removing stm32f4xx_hal.o(.rrx_text), (6 bytes).
    Removing stm32f4xx_hal_gpio.o(.rev16_text), (4 bytes).
    Removing stm32f4xx_hal_gpio.o(.revsh_text), (4 bytes).
    Removing stm32f4xx_hal_gpio.o(.rrx_text), (6 bytes).
    Removing stm32f4xx_hal_pwr.o(.rev16_text), (4 bytes).
    Removing stm32f4xx_hal_pwr.o(.revsh_text), (4 bytes).
    Removing stm32f4xx_hal_pwr.o(.rrx_text), (6 bytes).
    Removing stm32f4xx_hal_cortex.o(.rev16_text), (4 bytes).
    Removing stm32f4xx_hal_cortex.o(.revsh_text), (4 bytes).
    Removing stm32f4xx_hal_cortex.o(.rrx_text), (6 bytes).
    Removing stm32f4xx_hal_i2c.o(.rev16_text), (4 bytes).
    Removing stm32f4xx_hal_i2c.o(.revsh_text), (4 bytes).
    Removing stm32f4xx_hal_i2c.o(.rrx_text), (6 bytes).
    Removing stm32f4xx_hal_adc_ex.o(.rev16_text), (4 bytes).
    Removing stm32f4xx_hal_adc_ex.o(.revsh_text), (4 bytes).
    Removing stm32f4xx_hal_adc_ex.o(.rrx_text), (6 bytes).
    Removing stm32f4xx_hal_eth.o(.rev16_text), (4 bytes).
    Removing stm32f4xx_hal_eth.o(.revsh_text), (4 bytes).
    Removing stm32f4xx_hal_eth.o(.rrx_text), (6 bytes).
    Removing stm32f4xx_hal_dma.o(.rev16_text), (4 bytes).
    Removing stm32f4xx_hal_dma.o(.revsh_text), (4 bytes).
    Removing stm32f4xx_hal_dma.o(.rrx_text), (6 bytes).
    Removing stm32f4xx_hal_iwdg.o(.rev16_text), (4 bytes).
    Removing stm32f4xx_hal_iwdg.o(.revsh_text), (4 bytes).
    Removing stm32f4xx_hal_iwdg.o(.rrx_text), (6 bytes).
    Removing stm32f4xx_hal_rtc.o(.rev16_text), (4 bytes).
    Removing stm32f4xx_hal_rtc.o(.revsh_text), (4 bytes).
    Removing stm32f4xx_hal_rtc.o(.rrx_text), (6 bytes).
    Removing stm32f4xx_hal_rtc_ex.o(.rev16_text), (4 bytes).
    Removing stm32f4xx_hal_rtc_ex.o(.revsh_text), (4 bytes).
    Removing stm32f4xx_hal_rtc_ex.o(.rrx_text), (6 bytes).
    Removing stm32f4xx_hal_tim.o(.rev16_text), (4 bytes).
    Removing stm32f4xx_hal_tim.o(.revsh_text), (4 bytes).
    Removing stm32f4xx_hal_tim.o(.rrx_text), (6 bytes).
    Removing stm32f4xx_hal_tim_ex.o(.rev16_text), (4 bytes).
    Removing stm32f4xx_hal_tim_ex.o(.revsh_text), (4 bytes).
    Removing stm32f4xx_hal_tim_ex.o(.rrx_text), (6 bytes).
    Removing stm32f4xx_hal_spi.o(.rev16_text), (4 bytes).
    Removing stm32f4xx_hal_spi.o(.revsh_text), (4 bytes).
    Removing stm32f4xx_hal_spi.o(.rrx_text), (6 bytes).
    Removing startup_stm32f407xx.o(HEAP), (512 bytes).
    Removing stm32f4xx_hal_msp.o(.rev16_text), (4 bytes).
    Removing stm32f4xx_hal_msp.o(.revsh_text), (4 bytes).
    Removing stm32f4xx_hal_msp.o(.rrx_text), (6 bytes).
    Removing ethernetif.o(.rev16_text), (4 bytes).
    Removing ethernetif.o(.revsh_text), (4 bytes).
    Removing ethernetif.o(.rrx_text), (6 bytes).
    Removing main.o(.rev16_text), (4 bytes).
    Removing main.o(.revsh_text), (4 bytes).
    Removing main.o(.rrx_text), (6 bytes).
    Removing main.o(.data), (26 bytes).
    Removing stm32f4xx_it.o(.rev16_text), (4 bytes).
    Removing stm32f4xx_it.o(.revsh_text), (4 bytes).
    Removing stm32f4xx_it.o(.rrx_text), (6 bytes).
    Removing app_ethernet.o(.rev16_text), (4 bytes).
    Removing app_ethernet.o(.revsh_text), (4 bytes).
    Removing app_ethernet.o(.rrx_text), (6 bytes).
    Removing httpd_cgi_ssi.o(.rev16_text), (4 bytes).
    Removing httpd_cgi_ssi.o(.revsh_text), (4 bytes).
    Removing httpd_cgi_ssi.o(.rrx_text), (6 bytes).
    Removing httpd.o(.rev16_text), (4 bytes).
    Removing httpd.o(.revsh_text), (4 bytes).
    Removing httpd.o(.rrx_text), (6 bytes).
    Removing stm324xg_eval.o(.rev16_text), (4 bytes).
    Removing stm324xg_eval.o(.revsh_text), (4 bytes).
    Removing stm324xg_eval.o(.rrx_text), (6 bytes).
    Removing stm324xg_eval_eeprom.o(.rev16_text), (4 bytes).
    Removing stm324xg_eval_eeprom.o(.revsh_text), (4 bytes).
    Removing stm324xg_eval_eeprom.o(.rrx_text), (6 bytes).
    Removing init_l.o(.rev16_text), (4 bytes).
    Removing init_l.o(.revsh_text), (4 bytes).
    Removing init_l.o(.rrx_text), (6 bytes).
    Removing lab.o(.rev16_text), (4 bytes).
    Removing lab.o(.revsh_text), (4 bytes).
    Removing lab.o(.rrx_text), (6 bytes).
    Removing onewire.o(.rev16_text), (4 bytes).
    Removing onewire.o(.revsh_text), (4 bytes).
    Removing onewire.o(.rrx_text), (6 bytes).
    Removing process2.o(.rev16_text), (4 bytes).
    Removing process2.o(.revsh_text), (4 bytes).
    Removing process2.o(.rrx_text), (6 bytes).
    Removing rc5_ir_emul_receiver.o(.rev16_text), (4 bytes).
    Removing rc5_ir_emul_receiver.o(.revsh_text), (4 bytes).
    Removing rc5_ir_emul_receiver.o(.rrx_text), (6 bytes).
    Removing telnet.o(.rev16_text), (4 bytes).
    Removing telnet.o(.revsh_text), (4 bytes).
    Removing telnet.o(.rrx_text), (6 bytes).
    Removing lcd_g.o(.rev16_text), (4 bytes).
    Removing lcd_g.o(.revsh_text), (4 bytes).
    Removing lcd_g.o(.rrx_text), (6 bytes).
    Removing tm_stm32f4_fonts.o(.rev16_text), (4 bytes).
    Removing tm_stm32f4_fonts.o(.revsh_text), (4 bytes).
    Removing tm_stm32f4_fonts.o(.rrx_text), (6 bytes).
    Removing tm_stm32f4_fonts.o(.text), (28 bytes).
    Removing img.o(.rev16_text), (4 bytes).
    Removing img.o(.revsh_text), (4 bytes).
    Removing img.o(.rrx_text), (6 bytes).

122 unused section(s) (total 3797 bytes) removed from the image.

==============================================================================

Image Symbol Table

    Local Symbols

    Symbol Name                              Value     Ov Type        Size  Object(Section)

    ../clib/../cmprslib/zerorunl2.c          0x00000000   Number         0  __dczerorl2.o ABSOLUTE
    ../clib/microlib/ctype/ctype.c           0x00000000   Number         0  isgraph_o.o ABSOLUTE
    ../clib/microlib/ctype/ctype.c           0x00000000   Number         0  ctype_o.o ABSOLUTE
    ../clib/microlib/ctype/ctype.c           0x00000000   Number         0  isdigit_o.o ABSOLUTE
    ../clib/microlib/ctype/ctype.c           0x00000000   Number         0  isblank_o.o ABSOLUTE
    ../clib/microlib/ctype/ctype.c           0x00000000   Number         0  isalpha_o.o ABSOLUTE
    ../clib/microlib/ctype/ctype.c           0x00000000   Number         0  isalnum_o.o ABSOLUTE
    ../clib/microlib/ctype/ctype.c           0x00000000   Number         0  isspace_o.o ABSOLUTE
    ../clib/microlib/ctype/ctype.c           0x00000000   Number         0  isprint_o.o ABSOLUTE
    ../clib/microlib/ctype/ctype.c           0x00000000   Number         0  iscntrl_o.o ABSOLUTE
    ../clib/microlib/ctype/ctype.c           0x00000000   Number         0  islower_o.o ABSOLUTE
    ../clib/microlib/ctype/ctype.c           0x00000000   Number         0  isxdigit_o.o ABSOLUTE
    ../clib/microlib/ctype/ctype.c           0x00000000   Number         0  isupper_o.o ABSOLUTE
    ../clib/microlib/ctype/ctype.c           0x00000000   Number         0  ispunct_o.o ABSOLUTE
    ../clib/microlib/division.c              0x00000000   Number         0  uldiv.o ABSOLUTE
    ../clib/microlib/division.c              0x00000000   Number         0  ldiv.o ABSOLUTE
    ../clib/microlib/division.c              0x00000000   Number         0  uidiv.o ABSOLUTE
    ../clib/microlib/errno.c                 0x00000000   Number         0  errno.o ABSOLUTE
    ../clib/microlib/init/entry.s            0x00000000   Number         0  entry11b.o ABSOLUTE
    ../clib/microlib/init/entry.s            0x00000000   Number         0  entry5.o ABSOLUTE
    ../clib/microlib/init/entry.s            0x00000000   Number         0  entry2.o ABSOLUTE
    ../clib/microlib/init/entry.s            0x00000000   Number         0  entry.o ABSOLUTE
    ../clib/microlib/init/entry.s            0x00000000   Number         0  entry7a.o ABSOLUTE
    ../clib/microlib/init/entry.s            0x00000000   Number         0  entry9b.o ABSOLUTE
    ../clib/microlib/init/entry.s            0x00000000   Number         0  entry10a.o ABSOLUTE
    ../clib/microlib/init/entry.s            0x00000000   Number         0  entry10b.o ABSOLUTE
    ../clib/microlib/init/entry.s            0x00000000   Number         0  entry7b.o ABSOLUTE
    ../clib/microlib/init/entry.s            0x00000000   Number         0  entry11a.o ABSOLUTE
    ../clib/microlib/init/entry.s            0x00000000   Number         0  entry9a.o ABSOLUTE
    ../clib/microlib/init/entry.s            0x00000000   Number         0  entry8b.o ABSOLUTE
    ../clib/microlib/init/entry.s            0x00000000   Number         0  entry8a.o ABSOLUTE
    ../clib/microlib/longlong.c              0x00000000   Number         0  llsshr.o ABSOLUTE
    ../clib/microlib/longlong.c              0x00000000   Number         0  llushr.o ABSOLUTE
    ../clib/microlib/longlong.c              0x00000000   Number         0  llshl.o ABSOLUTE
    ../clib/microlib/printf/printf.c         0x00000000   Number         0  printfa.o ABSOLUTE
    ../clib/microlib/printf/printf.c         0x00000000   Number         0  printf2.o ABSOLUTE
    ../clib/microlib/printf/printf.c         0x00000000   Number         0  printf5.o ABSOLUTE
    ../clib/microlib/printf/printf.c         0x00000000   Number         0  printf6.o ABSOLUTE
    ../clib/microlib/printf/printf.c         0x00000000   Number         0  printf3.o ABSOLUTE
    ../clib/microlib/printf/printf.c         0x00000000   Number         0  printf7.o ABSOLUTE
    ../clib/microlib/printf/printf.c         0x00000000   Number         0  printf8.o ABSOLUTE
    ../clib/microlib/printf/printf.c         0x00000000   Number         0  printfb.o ABSOLUTE
    ../clib/microlib/printf/printf.c         0x00000000   Number         0  printf0.o ABSOLUTE
    ../clib/microlib/printf/printf.c         0x00000000   Number         0  printf1.o ABSOLUTE
    ../clib/microlib/printf/printf.c         0x00000000   Number         0  printf4.o ABSOLUTE
    ../clib/microlib/printf/stubs.s          0x00000000   Number         0  stubs.o ABSOLUTE
    ../clib/microlib/stdio/fputc.c           0x00000000   Number         0  fputc.o ABSOLUTE
    ../clib/microlib/stdio/semi.s            0x00000000   Number         0  semi.o ABSOLUTE
    ../clib/microlib/stdio/streams.c         0x00000000   Number         0  stdout.o ABSOLUTE
    ../clib/microlib/string/memcmp.c         0x00000000   Number         0  memcmp.o ABSOLUTE
    ../clib/microlib/string/memcpy.c         0x00000000   Number         0  memcpya.o ABSOLUTE
    ../clib/microlib/string/memcpy.c         0x00000000   Number         0  memcpyb.o ABSOLUTE
    ../clib/microlib/string/memset.c         0x00000000   Number         0  memseta.o ABSOLUTE
    ../clib/microlib/string/strchr.c         0x00000000   Number         0  strchr.o ABSOLUTE
    ../clib/microlib/string/strcmp.c         0x00000000   Number         0  strcmp.o ABSOLUTE
    ../clib/microlib/string/strcpy.c         0x00000000   Number         0  strcpy.o ABSOLUTE
    ../clib/microlib/string/strcspn.c        0x00000000   Number         0  strcspn.o ABSOLUTE
    ../clib/microlib/string/strlen.c         0x00000000   Number         0  strlen.o ABSOLUTE
    ../clib/microlib/string/strncmp.c        0x00000000   Number         0  strncmp.o ABSOLUTE
    ../clib/microlib/string/strstr.c         0x00000000   Number         0  strstr.o ABSOLUTE
    ../clib/microlib/stubs.s                 0x00000000   Number         0  iusefp.o ABSOLUTE
    ../clib/microlib/stubs.s                 0x00000000   Number         0  iusesemip.o ABSOLUTE
    ../clib/scanf.c                          0x00000000   Number         0  strtol.o ABSOLUTE
    ../clib/scanf.c                          0x00000000   Number         0  atoi.o ABSOLUTE
    ../clib/scanf.c                          0x00000000   Number         0  _strtoul.o ABSOLUTE
    ../clib/scanf.c                          0x00000000   Number         0  _chval.o ABSOLUTE
    ../fplib/microlib/d2f.c                  0x00000000   Number         0  d2f.o ABSOLUTE
    ../fplib/microlib/f2d.c                  0x00000000   Number         0  f2d.o ABSOLUTE
    ../fplib/microlib/fpadd.c                0x00000000   Number         0  dadd.o ABSOLUTE
    ../fplib/microlib/fpdiv.c                0x00000000   Number         0  ddiv.o ABSOLUTE
    ../fplib/microlib/fpepilogue.c           0x00000000   Number         0  depilogue.o ABSOLUTE
    ../fplib/microlib/fpepilogue.c           0x00000000   Number         0  fepilogue.o ABSOLUTE
    ../fplib/microlib/fpfix.c                0x00000000   Number         0  dfixul.o ABSOLUTE
    ../fplib/microlib/fpfix.c                0x00000000   Number         0  dfixui.o ABSOLUTE
    ../fplib/microlib/fpflt.c                0x00000000   Number         0  dfltul.o ABSOLUTE
    ../fplib/microlib/fpflt.c                0x00000000   Number         0  dfltui.o ABSOLUTE
    ../fplib/microlib/fpflt.c                0x00000000   Number         0  ffltul.o ABSOLUTE
    ../fplib/microlib/fpmul.c                0x00000000   Number         0  dmul.o ABSOLUTE
    ../fplib/microlib/fpsqrt.c               0x00000000   Number         0  dsqrt.o ABSOLUTE
    ../mathlib/sqrt.c                        0x00000000   Number         0  sqrt_x.o ABSOLUTE
    ../mathlib/sqrt.c                        0x00000000   Number         0  sqrt.o ABSOLUTE
    ..\..\..\..\..\..\Drivers\BSP\STM324xG_EVAL\stm324xg_eval.c 0x00000000   Number         0  stm324xg_eval.o ABSOLUTE
    ..\..\..\..\..\..\Drivers\BSP\STM324xG_EVAL\stm324xg_eval_eeprom.c 0x00000000   Number         0  stm324xg_eval_eeprom.o ABSOLUTE
    ..\..\..\..\..\..\Drivers\STM32F4xx_HAL_Driver\Src\stm32f4xx_hal.c 0x00000000   Number         0  stm32f4xx_hal.o ABSOLUTE
    ..\..\..\..\..\..\Drivers\STM32F4xx_HAL_Driver\Src\stm32f4xx_hal_adc.c 0x00000000   Number         0  stm32f4xx_hal_adc.o ABSOLUTE
    ..\..\..\..\..\..\Drivers\STM32F4xx_HAL_Driver\Src\stm32f4xx_hal_adc_ex.c 0x00000000   Number         0  stm32f4xx_hal_adc_ex.o ABSOLUTE
    ..\..\..\..\..\..\Drivers\STM32F4xx_HAL_Driver\Src\stm32f4xx_hal_cortex.c 0x00000000   Number         0  stm32f4xx_hal_cortex.o ABSOLUTE
    ..\..\..\..\..\..\Drivers\STM32F4xx_HAL_Driver\Src\stm32f4xx_hal_dma.c 0x00000000   Number         0  stm32f4xx_hal_dma.o ABSOLUTE
    ..\..\..\..\..\..\Drivers\STM32F4xx_HAL_Driver\Src\stm32f4xx_hal_eth.c 0x00000000   Number         0  stm32f4xx_hal_eth.o ABSOLUTE
    ..\..\..\..\..\..\Drivers\STM32F4xx_HAL_Driver\Src\stm32f4xx_hal_flash.c 0x00000000   Number         0  stm32f4xx_hal_flash.o ABSOLUTE
    ..\..\..\..\..\..\Drivers\STM32F4xx_HAL_Driver\Src\stm32f4xx_hal_flash_ex.c 0x00000000   Number         0  stm32f4xx_hal_flash_ex.o ABSOLUTE
    ..\..\..\..\..\..\Drivers\STM32F4xx_HAL_Driver\Src\stm32f4xx_hal_gpio.c 0x00000000   Number         0  stm32f4xx_hal_gpio.o ABSOLUTE
    ..\..\..\..\..\..\Drivers\STM32F4xx_HAL_Driver\Src\stm32f4xx_hal_i2c.c 0x00000000   Number         0  stm32f4xx_hal_i2c.o ABSOLUTE
    ..\..\..\..\..\..\Drivers\STM32F4xx_HAL_Driver\Src\stm32f4xx_hal_iwdg.c 0x00000000   Number         0  stm32f4xx_hal_iwdg.o ABSOLUTE
    ..\..\..\..\..\..\Drivers\STM32F4xx_HAL_Driver\Src\stm32f4xx_hal_pwr.c 0x00000000   Number         0  stm32f4xx_hal_pwr.o ABSOLUTE
    ..\..\..\..\..\..\Drivers\STM32F4xx_HAL_Driver\Src\stm32f4xx_hal_rcc.c 0x00000000   Number         0  stm32f4xx_hal_rcc.o ABSOLUTE
    ..\..\..\..\..\..\Drivers\STM32F4xx_HAL_Driver\Src\stm32f4xx_hal_rtc.c 0x00000000   Number         0  stm32f4xx_hal_rtc.o ABSOLUTE
    ..\..\..\..\..\..\Drivers\STM32F4xx_HAL_Driver\Src\stm32f4xx_hal_rtc_ex.c 0x00000000   Number         0  stm32f4xx_hal_rtc_ex.o ABSOLUTE
    ..\..\..\..\..\..\Drivers\STM32F4xx_HAL_Driver\Src\stm32f4xx_hal_spi.c 0x00000000   Number         0  stm32f4xx_hal_spi.o ABSOLUTE
    ..\..\..\..\..\..\Drivers\STM32F4xx_HAL_Driver\Src\stm32f4xx_hal_tim.c 0x00000000   Number         0  stm32f4xx_hal_tim.o ABSOLUTE
    ..\..\..\..\..\..\Drivers\STM32F4xx_HAL_Driver\Src\stm32f4xx_hal_tim_ex.c 0x00000000   Number         0  stm32f4xx_hal_tim_ex.o ABSOLUTE
    ..\..\..\..\..\..\Middlewares\Third_Party\LwIP\src\api\api_lib.c 0x00000000   Number         0  api_lib.o ABSOLUTE
    ..\..\..\..\..\..\Middlewares\Third_Party\LwIP\src\api\api_msg.c 0x00000000   Number         0  api_msg.o ABSOLUTE
    ..\..\..\..\..\..\Middlewares\Third_Party\LwIP\src\api\err.c 0x00000000   Number         0  err.o ABSOLUTE
    ..\..\..\..\..\..\Middlewares\Third_Party\LwIP\src\api\netbuf.c 0x00000000   Number         0  netbuf.o ABSOLUTE
    ..\..\..\..\..\..\Middlewares\Third_Party\LwIP\src\api\netdb.c 0x00000000   Number         0  netdb.o ABSOLUTE
    ..\..\..\..\..\..\Middlewares\Third_Party\LwIP\src\api\netifapi.c 0x00000000   Number         0  netifapi.o ABSOLUTE
    ..\..\..\..\..\..\Middlewares\Third_Party\LwIP\src\api\sockets.c 0x00000000   Number         0  sockets.o ABSOLUTE
    ..\..\..\..\..\..\Middlewares\Third_Party\LwIP\src\api\tcpip.c 0x00000000   Number         0  tcpip.o ABSOLUTE
    ..\..\..\..\..\..\Middlewares\Third_Party\LwIP\src\core\def.c 0x00000000   Number         0  def.o ABSOLUTE
    ..\..\..\..\..\..\Middlewares\Third_Party\LwIP\src\core\dhcp.c 0x00000000   Number         0  dhcp.o ABSOLUTE
    ..\..\..\..\..\..\Middlewares\Third_Party\LwIP\src\core\dns.c 0x00000000   Number         0  dns.o ABSOLUTE
    ..\..\..\..\..\..\Middlewares\Third_Party\LwIP\src\core\init.c 0x00000000   Number         0  init.o ABSOLUTE
    ..\..\..\..\..\..\Middlewares\Third_Party\LwIP\src\core\ipv4\autoip.c 0x00000000   Number         0  autoip.o ABSOLUTE
    ..\..\..\..\..\..\Middlewares\Third_Party\LwIP\src\core\ipv4\icmp.c 0x00000000   Number         0  icmp.o ABSOLUTE
    ..\..\..\..\..\..\Middlewares\Third_Party\LwIP\src\core\ipv4\igmp.c 0x00000000   Number         0  igmp.o ABSOLUTE
    ..\..\..\..\..\..\Middlewares\Third_Party\LwIP\src\core\ipv4\inet.c 0x00000000   Number         0  inet.o ABSOLUTE
    ..\..\..\..\..\..\Middlewares\Third_Party\LwIP\src\core\ipv4\inet_chksum.c 0x00000000   Number         0  inet_chksum.o ABSOLUTE
    ..\..\..\..\..\..\Middlewares\Third_Party\LwIP\src\core\ipv4\ip.c 0x00000000   Number         0  ip.o ABSOLUTE
    ..\..\..\..\..\..\Middlewares\Third_Party\LwIP\src\core\ipv4\ip_addr.c 0x00000000   Number         0  ip_addr.o ABSOLUTE
    ..\..\..\..\..\..\Middlewares\Third_Party\LwIP\src\core\ipv4\ip_frag.c 0x00000000   Number         0  ip_frag.o ABSOLUTE
    ..\..\..\..\..\..\Middlewares\Third_Party\LwIP\src\core\lwip_timers.c 0x00000000   Number         0  lwip_timers.o ABSOLUTE
    ..\..\..\..\..\..\Middlewares\Third_Party\LwIP\src\core\mem.c 0x00000000   Number         0  mem.o ABSOLUTE
    ..\..\..\..\..\..\Middlewares\Third_Party\LwIP\src\core\memp.c 0x00000000   Number         0  memp.o ABSOLUTE
    ..\..\..\..\..\..\Middlewares\Third_Party\LwIP\src\core\netif.c 0x00000000   Number         0  netif.o ABSOLUTE
    ..\..\..\..\..\..\Middlewares\Third_Party\LwIP\src\core\pbuf.c 0x00000000   Number         0  pbuf.o ABSOLUTE
    ..\..\..\..\..\..\Middlewares\Third_Party\LwIP\src\core\raw.c 0x00000000   Number         0  raw.o ABSOLUTE
    ..\..\..\..\..\..\Middlewares\Third_Party\LwIP\src\core\stats.c 0x00000000   Number         0  stats.o ABSOLUTE
    ..\..\..\..\..\..\Middlewares\Third_Party\LwIP\src\core\sys.c 0x00000000   Number         0  sys.o ABSOLUTE
    ..\..\..\..\..\..\Middlewares\Third_Party\LwIP\src\core\tcp.c 0x00000000   Number         0  tcp.o ABSOLUTE
    ..\..\..\..\..\..\Middlewares\Third_Party\LwIP\src\core\tcp_in.c 0x00000000   Number         0  tcp_in.o ABSOLUTE
    ..\..\..\..\..\..\Middlewares\Third_Party\LwIP\src\core\tcp_out.c 0x00000000   Number         0  tcp_out.o ABSOLUTE
    ..\..\..\..\..\..\Middlewares\Third_Party\LwIP\src\core\udp.c 0x00000000   Number         0  udp.o ABSOLUTE
    ..\..\..\..\..\..\Middlewares\Third_Party\LwIP\src\netif\etharp.c 0x00000000   Number         0  etharp.o ABSOLUTE
    ..\Src\app_ethernet.c                    0x00000000   Number         0  app_ethernet.o ABSOLUTE
    ..\Src\ethernetif.c                      0x00000000   Number         0  ethernetif.o ABSOLUTE
    ..\Src\fs.c                              0x00000000   Number         0  fs.o ABSOLUTE
    ..\Src\httpd.c                           0x00000000   Number         0  httpd.o ABSOLUTE
    ..\Src\httpd_cgi_ssi.c                   0x00000000   Number         0  httpd_cgi_ssi.o ABSOLUTE
    ..\Src\main.c                            0x00000000   Number         0  main.o ABSOLUTE
    ..\Src\stm32f4xx_hal_msp.c               0x00000000   Number         0  stm32f4xx_hal_msp.o ABSOLUTE
    ..\Src\stm32f4xx_it.c                    0x00000000   Number         0  stm32f4xx_it.o ABSOLUTE
    ..\Src\system_stm32f4xx.c                0x00000000   Number         0  system_stm32f4xx.o ABSOLUTE
    ..\\..\\..\\..\\..\\..\\Drivers\\BSP\\STM324xG_EVAL\\stm324xg_eval.c 0x00000000   Number         0  stm324xg_eval.o ABSOLUTE
    ..\\..\\..\\..\\..\\..\\Drivers\\BSP\\STM324xG_EVAL\\stm324xg_eval_eeprom.c 0x00000000   Number         0  stm324xg_eval_eeprom.o ABSOLUTE
    ..\\..\\..\\..\\..\\..\\Drivers\\STM32F4xx_HAL_Driver\\Src\\stm32f4xx_hal.c 0x00000000   Number         0  stm32f4xx_hal.o ABSOLUTE
    ..\\..\\..\\..\\..\\..\\Drivers\\STM32F4xx_HAL_Driver\\Src\\stm32f4xx_hal_adc.c 0x00000000   Number         0  stm32f4xx_hal_adc.o ABSOLUTE
    ..\\..\\..\\..\\..\\..\\Drivers\\STM32F4xx_HAL_Driver\\Src\\stm32f4xx_hal_adc_ex.c 0x00000000   Number         0  stm32f4xx_hal_adc_ex.o ABSOLUTE
    ..\\..\\..\\..\\..\\..\\Drivers\\STM32F4xx_HAL_Driver\\Src\\stm32f4xx_hal_cortex.c 0x00000000   Number         0  stm32f4xx_hal_cortex.o ABSOLUTE
    ..\\..\\..\\..\\..\\..\\Drivers\\STM32F4xx_HAL_Driver\\Src\\stm32f4xx_hal_dma.c 0x00000000   Number         0  stm32f4xx_hal_dma.o ABSOLUTE
    ..\\..\\..\\..\\..\\..\\Drivers\\STM32F4xx_HAL_Driver\\Src\\stm32f4xx_hal_eth.c 0x00000000   Number         0  stm32f4xx_hal_eth.o ABSOLUTE
    ..\\..\\..\\..\\..\\..\\Drivers\\STM32F4xx_HAL_Driver\\Src\\stm32f4xx_hal_flash.c 0x00000000   Number         0  stm32f4xx_hal_flash.o ABSOLUTE
    ..\\..\\..\\..\\..\\..\\Drivers\\STM32F4xx_HAL_Driver\\Src\\stm32f4xx_hal_flash_ex.c 0x00000000   Number         0  stm32f4xx_hal_flash_ex.o ABSOLUTE
    ..\\..\\..\\..\\..\\..\\Drivers\\STM32F4xx_HAL_Driver\\Src\\stm32f4xx_hal_gpio.c 0x00000000   Number         0  stm32f4xx_hal_gpio.o ABSOLUTE
    ..\\..\\..\\..\\..\\..\\Drivers\\STM32F4xx_HAL_Driver\\Src\\stm32f4xx_hal_i2c.c 0x00000000   Number         0  stm32f4xx_hal_i2c.o ABSOLUTE
    ..\\..\\..\\..\\..\\..\\Drivers\\STM32F4xx_HAL_Driver\\Src\\stm32f4xx_hal_iwdg.c 0x00000000   Number         0  stm32f4xx_hal_iwdg.o ABSOLUTE
    ..\\..\\..\\..\\..\\..\\Drivers\\STM32F4xx_HAL_Driver\\Src\\stm32f4xx_hal_pwr.c 0x00000000   Number         0  stm32f4xx_hal_pwr.o ABSOLUTE
    ..\\..\\..\\..\\..\\..\\Drivers\\STM32F4xx_HAL_Driver\\Src\\stm32f4xx_hal_rcc.c 0x00000000   Number         0  stm32f4xx_hal_rcc.o ABSOLUTE
    ..\\..\\..\\..\\..\\..\\Drivers\\STM32F4xx_HAL_Driver\\Src\\stm32f4xx_hal_rtc.c 0x00000000   Number         0  stm32f4xx_hal_rtc.o ABSOLUTE
    ..\\..\\..\\..\\..\\..\\Drivers\\STM32F4xx_HAL_Driver\\Src\\stm32f4xx_hal_rtc_ex.c 0x00000000   Number         0  stm32f4xx_hal_rtc_ex.o ABSOLUTE
    ..\\..\\..\\..\\..\\..\\Drivers\\STM32F4xx_HAL_Driver\\Src\\stm32f4xx_hal_spi.c 0x00000000   Number         0  stm32f4xx_hal_spi.o ABSOLUTE
    ..\\..\\..\\..\\..\\..\\Drivers\\STM32F4xx_HAL_Driver\\Src\\stm32f4xx_hal_tim.c 0x00000000   Number         0  stm32f4xx_hal_tim.o ABSOLUTE
    ..\\..\\..\\..\\..\\..\\Drivers\\STM32F4xx_HAL_Driver\\Src\\stm32f4xx_hal_tim_ex.c 0x00000000   Number         0  stm32f4xx_hal_tim_ex.o ABSOLUTE
    ..\\Src\\app_ethernet.c                  0x00000000   Number         0  app_ethernet.o ABSOLUTE
    ..\\Src\\ethernetif.c                    0x00000000   Number         0  ethernetif.o ABSOLUTE
    ..\\Src\\httpd.c                         0x00000000   Number         0  httpd.o ABSOLUTE
    ..\\Src\\httpd_cgi_ssi.c                 0x00000000   Number         0  httpd_cgi_ssi.o ABSOLUTE
    ..\\Src\\main.c                          0x00000000   Number         0  main.o ABSOLUTE
    ..\\Src\\stm32f4xx_hal_msp.c             0x00000000   Number         0  stm32f4xx_hal_msp.o ABSOLUTE
    ..\\Src\\stm32f4xx_it.c                  0x00000000   Number         0  stm32f4xx_it.o ABSOLUTE
    ..\\Src\\system_stm32f4xx.c              0x00000000   Number         0  system_stm32f4xx.o ABSOLUTE
    LabSpirt_files\Src\RC5_IR_Emul_Receiver.c 0x00000000   Number         0  rc5_ir_emul_receiver.o ABSOLUTE
    LabSpirt_files\Src\img.c                 0x00000000   Number         0  img.o ABSOLUTE
    LabSpirt_files\Src\init_l.c              0x00000000   Number         0  init_l.o ABSOLUTE
    LabSpirt_files\Src\lab.c                 0x00000000   Number         0  lab.o ABSOLUTE
    LabSpirt_files\Src\lcd_g.c               0x00000000   Number         0  lcd_g.o ABSOLUTE
    LabSpirt_files\Src\onewire.c             0x00000000   Number         0  onewire.o ABSOLUTE
    LabSpirt_files\Src\process2.c            0x00000000   Number         0  process2.o ABSOLUTE
    LabSpirt_files\Src\telnet.c              0x00000000   Number         0  telnet.o ABSOLUTE
    LabSpirt_files\Src\tm_stm32f4_fonts.c    0x00000000   Number         0  tm_stm32f4_fonts.o ABSOLUTE
    LabSpirt_files\\Src\\RC5_IR_Emul_Receiver.c 0x00000000   Number         0  rc5_ir_emul_receiver.o ABSOLUTE
    LabSpirt_files\\Src\\img.c               0x00000000   Number         0  img.o ABSOLUTE
    LabSpirt_files\\Src\\init_l.c            0x00000000   Number         0  init_l.o ABSOLUTE
    LabSpirt_files\\Src\\lab.c               0x00000000   Number         0  lab.o ABSOLUTE
    LabSpirt_files\\Src\\lcd_g.c             0x00000000   Number         0  lcd_g.o ABSOLUTE
    LabSpirt_files\\Src\\onewire.c           0x00000000   Number         0  onewire.o ABSOLUTE
    LabSpirt_files\\Src\\process2.c          0x00000000   Number         0  process2.o ABSOLUTE
    LabSpirt_files\\Src\\telnet.c            0x00000000   Number         0  telnet.o ABSOLUTE
    LabSpirt_files\\Src\\tm_stm32f4_fonts.c  0x00000000   Number         0  tm_stm32f4_fonts.o ABSOLUTE
    cdcmple.s                                0x00000000   Number         0  cdcmple.o ABSOLUTE
    cdrcmple.s                               0x00000000   Number         0  cdrcmple.o ABSOLUTE
    dc.s                                     0x00000000   Number         0  dc.o ABSOLUTE
    handlers.s                               0x00000000   Number         0  handlers.o ABSOLUTE
    init.s                                   0x00000000   Number         0  init.o ABSOLUTE
    startup_stm32f407xx.s                    0x00000000   Number         0  startup_stm32f407xx.o ABSOLUTE
    RESET                                    0x08000000   Section      392  startup_stm32f407xx.o(RESET)
    .ARM.Collect$$$$00000000                 0x08000188   Section        0  entry.o(.ARM.Collect$$$$00000000)
    .ARM.Collect$$$$00000001                 0x08000188   Section        4  entry2.o(.ARM.Collect$$$$00000001)
    .ARM.Collect$$$$00000004                 0x0800018c   Section        4  entry5.o(.ARM.Collect$$$$00000004)
    .ARM.Collect$$$$00000008                 0x08000190   Section        0  entry7b.o(.ARM.Collect$$$$00000008)
    .ARM.Collect$$$$0000000A                 0x08000190   Section        0  entry8b.o(.ARM.Collect$$$$0000000A)
    .ARM.Collect$$$$0000000B                 0x08000190   Section        8  entry9a.o(.ARM.Collect$$$$0000000B)
    .ARM.Collect$$$$0000000D                 0x08000198   Section        0  entry10a.o(.ARM.Collect$$$$0000000D)
    .ARM.Collect$$$$0000000F                 0x08000198   Section        0  entry11a.o(.ARM.Collect$$$$0000000F)
    .ARM.Collect$$$$00002712                 0x08000198   Section        4  entry2.o(.ARM.Collect$$$$00002712)
    __lit__00000000                          0x08000198   Data           4  entry2.o(.ARM.Collect$$$$00002712)
    .text                                    0x0800019c   Section        0  system_stm32f4xx.o(.text)
    .text                                    0x080002bc   Section        0  tcp_in.o(.text)
    tcp_receive                              0x080002bd   Thumb Code  1634  tcp_in.o(.text)
    tcp_parseopt                             0x0800091f   Thumb Code   202  tcp_in.o(.text)
    tcp_process                              0x080009e9   Thumb Code  1464  tcp_in.o(.text)
    tcp_listen_input                         0x08000fa1   Thumb Code   280  tcp_in.o(.text)
    tcp_timewait_input                       0x080010b9   Thumb Code   140  tcp_in.o(.text)
    .text                                    0x080015fc   Section        0  def.o(.text)
    .text                                    0x0800163c   Section        0  lwip_timers.o(.text)
    tcpip_tcp_timer                          0x080016d5   Thumb Code    40  lwip_timers.o(.text)
    ip_reass_timer                           0x08001723   Thumb Code    26  lwip_timers.o(.text)
    arp_timer                                0x0800173d   Thumb Code    26  lwip_timers.o(.text)
    dhcp_timer_coarse                        0x08001757   Thumb Code    26  lwip_timers.o(.text)
    dhcp_timer_fine                          0x08001771   Thumb Code    26  lwip_timers.o(.text)
    .text                                    0x080018b0   Section        0  memp.o(.text)
    .text                                    0x0800195c   Section        0  dhcp.o(.text)
    dhcp_delete_msg                          0x0800195d   Thumb Code    40  dhcp.o(.text)
    dhcp_option_trailer                      0x08001985   Thumb Code    70  dhcp.o(.text)
    dhcp_option_byte                         0x080019cb   Thumb Code    18  dhcp.o(.text)
    dhcp_option                              0x080019dd   Thumb Code    32  dhcp.o(.text)
    dhcp_option_short                        0x080019fd   Thumb Code    34  dhcp.o(.text)
    dhcp_create_msg                          0x08001a1f   Thumb Code   326  dhcp.o(.text)
    dhcp_set_state                           0x08001b65   Thumb Code    16  dhcp.o(.text)
    dhcp_discover                            0x08001b75   Thumb Code   222  dhcp.o(.text)
    dhcp_handle_nak                          0x08001c53   Thumb Code    56  dhcp.o(.text)
    dhcp_check                               0x08001c8b   Thumb Code    70  dhcp.o(.text)
    dhcp_option_long                         0x08001cd1   Thumb Code    66  dhcp.o(.text)
    dhcp_select                              0x08001d13   Thumb Code   256  dhcp.o(.text)
    dhcp_handle_offer                        0x08001e13   Thumb Code    78  dhcp.o(.text)
    dhcp_t1_timeout                          0x08001ef7   Thumb Code    40  dhcp.o(.text)
    dhcp_rebind                              0x08001f1f   Thumb Code   148  dhcp.o(.text)
    dhcp_t2_timeout                          0x08001fb3   Thumb Code    40  dhcp.o(.text)
    dhcp_reboot                              0x08002025   Thumb Code   180  dhcp.o(.text)
    dhcp_bind                                0x0800218b   Thumb Code   260  dhcp.o(.text)
    dhcp_timeout                             0x0800228f   Thumb Code   210  dhcp.o(.text)
    dhcp_handle_ack                          0x080023a5   Thumb Code   112  dhcp.o(.text)
    dhcp_parse_reply                         0x08002489   Thumb Code   808  dhcp.o(.text)
    dhcp_recv                                0x080027b1   Thumb Code   298  dhcp.o(.text)
    dhcp_decline                             0x08002ad5   Thumb Code   142  dhcp.o(.text)
    .text                                    0x08002bb0   Section        0  udp.o(.text)
    udp_new_port                             0x08002bb3   Thumb Code    80  udp.o(.text)
    .text                                    0x08003088   Section        0  mem.o(.text)
    plug_holes                               0x08003089   Thumb Code   124  mem.o(.text)
    .text                                    0x080033d4   Section        0  netif.o(.text)
    .text                                    0x080036c4   Section        0  tcp.o(.text)
    tcp_close_shutdown                       0x08003b1d   Thumb Code   470  tcp.o(.text)
    tcp_new_port                             0x08004017   Thumb Code    96  tcp.o(.text)
    tcp_accept_null                          0x08004109   Thumb Code     8  tcp.o(.text)
    tcp_kill_prio                            0x08004365   Thumb Code   122  tcp.o(.text)
    tcp_kill_timewait                        0x080043df   Thumb Code    54  tcp.o(.text)
    .text                                    0x08004524   Section        0  tcp_out.o(.text)
    tcp_output_alloc_header                  0x08004525   Thumb Code   120  tcp_out.o(.text)
    tcp_create_segment                       0x0800459d   Thumb Code   184  tcp_out.o(.text)
    tcp_pbuf_prealloc                        0x080047c5   Thumb Code   120  tcp_out.o(.text)
    tcp_write_checks                         0x0800483d   Thumb Code   128  tcp_out.o(.text)
    tcp_output_segment                       0x08004ce1   Thumb Code   210  tcp_out.o(.text)
    .text                                    0x08005208   Section        0  raw.o(.text)
    .text                                    0x080053c8   Section        0  init.o(.text)
    .text                                    0x080053e4   Section        0  pbuf.o(.text)
    .text                                    0x08005b64   Section        0  ip_addr.o(.text)
    .text                                    0x08005e1c   Section        0  inet_chksum.o(.text)
    lwip_standard_chksum                     0x08005e1d   Thumb Code    94  inet_chksum.o(.text)
    .text                                    0x08006050   Section        0  ip_frag.o(.text)
    ip_reass_dequeue_datagram                0x08006051   Thumb Code    40  ip_frag.o(.text)
    ip_reass_free_complete_datagram          0x08006079   Thumb Code   156  ip_frag.o(.text)
    ip_reass_remove_oldest_datagram          0x0800614d   Thumb Code   118  ip_frag.o(.text)
    ip_reass_enqueue_new_datagram            0x080061c3   Thumb Code    84  ip_frag.o(.text)
    ip_reass_chain_frag_into_datagram_and_validate 0x08006217   Thumb Code   352  ip_frag.o(.text)
    ip_frag_alloc_pbuf_custom_ref            0x0800651d   Thumb Code    10  ip_frag.o(.text)
    ip_frag_free_pbuf_custom_ref             0x08006527   Thumb Code    18  ip_frag.o(.text)
    ipfrag_free_pbuf_custom                  0x08006539   Thumb Code    32  ip_frag.o(.text)
    .text                                    0x08006708   Section        0  ip.o(.text)
    .text                                    0x08006a60   Section        0  icmp.o(.text)
    icmp_send_response                       0x08006bdd   Thumb Code   136  icmp.o(.text)
    .text                                    0x08006c90   Section        0  etharp.o(.text)
    etharp_free_entry                        0x08006c91   Thumb Code   112  etharp.o(.text)
    etharp_find_entry                        0x08006d91   Thumb Code   374  etharp.o(.text)
    etharp_send_ip                           0x08006f07   Thumb Code    60  etharp.o(.text)
    etharp_update_arp_entry                  0x08006f43   Thumb Code   190  etharp.o(.text)
    etharp_arp_input                         0x0800708f   Thumb Code   306  etharp.o(.text)
    etharp_raw                               0x080071c1   Thumb Code   186  etharp.o(.text)
    etharp_output_to_arp_index               0x080072a3   Thumb Code   104  etharp.o(.text)
    .text                                    0x08007678   Section        0  stm32f4xx_hal_rcc.o(.text)
    .text                                    0x08007f5c   Section        0  stm32f4xx_hal_adc.o(.text)
    ADC_Init                                 0x08007f5d   Thumb Code   362  stm32f4xx_hal_adc.o(.text)
    ADC_DMAError                             0x080086b5   Thumb Code    26  stm32f4xx_hal_adc.o(.text)
    ADC_DMAHalfConvCplt                      0x080086d1   Thumb Code    14  stm32f4xx_hal_adc.o(.text)
    ADC_DMAConvCplt                          0x080086df   Thumb Code   110  stm32f4xx_hal_adc.o(.text)
    .text                                    0x08008b34   Section        0  stm32f4xx_hal.o(.text)
    .text                                    0x08008cc8   Section        0  stm32f4xx_hal_gpio.o(.text)
    .text                                    0x0800908c   Section        0  stm32f4xx_hal_pwr.o(.text)
    .text                                    0x08009298   Section        0  stm32f4xx_hal_cortex.o(.text)
    NVIC_SetPriority                         0x08009299   Thumb Code    32  stm32f4xx_hal_cortex.o(.text)
    NVIC_GetPriorityGrouping                 0x08009595   Thumb Code    12  stm32f4xx_hal_cortex.o(.text)
    .text                                    0x080095b4   Section        0  stm32f4xx_hal_i2c.o(.text)
    I2C_IsAcknowledgeFailed                  0x08009713   Thumb Code    52  stm32f4xx_hal_i2c.o(.text)
    I2C_WaitOnBTFFlagUntilTimeout            0x08009747   Thumb Code    90  stm32f4xx_hal_i2c.o(.text)
    I2C_WaitOnTXEFlagUntilTimeout            0x080097a1   Thumb Code    90  stm32f4xx_hal_i2c.o(.text)
    I2C_WaitOnMasterAddressFlagUntilTimeout  0x080097fb   Thumb Code   178  stm32f4xx_hal_i2c.o(.text)
    I2C_WaitOnFlagUntilTimeout               0x080098ad   Thumb Code   230  stm32f4xx_hal_i2c.o(.text)
    I2C_MasterRequestWrite                   0x08009993   Thumb Code   186  stm32f4xx_hal_i2c.o(.text)
    I2C_WaitOnRXNEFlagUntilTimeout           0x08009b8d   Thumb Code   116  stm32f4xx_hal_i2c.o(.text)
    I2C_MasterRequestRead                    0x08009c01   Thumb Code   298  stm32f4xx_hal_i2c.o(.text)
    I2C_WaitOnSTOPFlagUntilTimeout           0x0800a0ff   Thumb Code    88  stm32f4xx_hal_i2c.o(.text)
    I2C_DMAError                             0x0800aabd   Thumb Code    50  stm32f4xx_hal_i2c.o(.text)
    I2C_DMAMasterTransmitCplt                0x0800aaf1   Thumb Code    88  stm32f4xx_hal_i2c.o(.text)
    I2C_DMAMasterReceiveCplt                 0x0800acad   Thumb Code    90  stm32f4xx_hal_i2c.o(.text)
    I2C_DMASlaveTransmitCplt                 0x0800aed9   Thumb Code    98  stm32f4xx_hal_i2c.o(.text)
    I2C_DMASlaveReceiveCplt                  0x0800b07b   Thumb Code   128  stm32f4xx_hal_i2c.o(.text)
    I2C_RequestMemoryWrite                   0x0800b1d1   Thumb Code   208  stm32f4xx_hal_i2c.o(.text)
    I2C_RequestMemoryRead                    0x0800b3d1   Thumb Code   344  stm32f4xx_hal_i2c.o(.text)
    I2C_DMAMemTransmitCplt                   0x0800ba13   Thumb Code    88  stm32f4xx_hal_i2c.o(.text)
    I2C_DMAMemReceiveCplt                    0x0800bba7   Thumb Code    90  stm32f4xx_hal_i2c.o(.text)
    I2C_SlaveReceive_BTF                     0x0800bf19   Thumb Code    30  stm32f4xx_hal_i2c.o(.text)
    I2C_SlaveReceive_RXNE                    0x0800bf37   Thumb Code    84  stm32f4xx_hal_i2c.o(.text)
    I2C_SlaveTransmit_BTF                    0x0800bf8b   Thumb Code    28  stm32f4xx_hal_i2c.o(.text)
    I2C_SlaveTransmit_TXE                    0x0800bfa7   Thumb Code    82  stm32f4xx_hal_i2c.o(.text)
    I2C_Slave_STOPF                          0x0800bffb   Thumb Code   136  stm32f4xx_hal_i2c.o(.text)
    I2C_Slave_ADDR                           0x0800c085   Thumb Code    54  stm32f4xx_hal_i2c.o(.text)
    I2C_MasterReceive_BTF                    0x0800c0bb   Thumb Code   300  stm32f4xx_hal_i2c.o(.text)
    I2C_MasterReceive_RXNE                   0x0800c1e7   Thumb Code   248  stm32f4xx_hal_i2c.o(.text)
    I2C_MasterTransmit_BTF                   0x0800c2df   Thumb Code   178  stm32f4xx_hal_i2c.o(.text)
    I2C_MasterTransmit_TXE                   0x0800c391   Thumb Code    42  stm32f4xx_hal_i2c.o(.text)
    I2C_Slave_AF                             0x0800c531   Thumb Code   176  stm32f4xx_hal_i2c.o(.text)
    .text                                    0x0800c748   Section        0  stm32f4xx_hal_adc_ex.o(.text)
    ADC_MultiModeDMAError                    0x0800cb0f   Thumb Code    26  stm32f4xx_hal_adc_ex.o(.text)
    ADC_MultiModeDMAHalfConvCplt             0x0800cb29   Thumb Code    14  stm32f4xx_hal_adc_ex.o(.text)
    ADC_MultiModeDMAConvCplt                 0x0800cb37   Thumb Code   130  stm32f4xx_hal_adc_ex.o(.text)
    .text                                    0x0800d00c   Section        0  stm32f4xx_hal_eth.o(.text)
    ETH_MACAddressConfig                     0x0800d00d   Thumb Code    48  stm32f4xx_hal_eth.o(.text)
    ETH_MACDMAConfig                         0x0800d03d   Thumb Code   566  stm32f4xx_hal_eth.o(.text)
    ETH_DMAReceptionEnable                   0x0800dad1   Thumb Code    22  stm32f4xx_hal_eth.o(.text)
    ETH_DMATransmissionEnable                0x0800dae7   Thumb Code    22  stm32f4xx_hal_eth.o(.text)
    ETH_FlushTransmitFIFO                    0x0800dafd   Thumb Code    56  stm32f4xx_hal_eth.o(.text)
    ETH_MACReceptionEnable                   0x0800db35   Thumb Code    40  stm32f4xx_hal_eth.o(.text)
    ETH_MACTransmissionEnable                0x0800db5d   Thumb Code    40  stm32f4xx_hal_eth.o(.text)
    ETH_MACTransmissionDisable               0x0800dbd7   Thumb Code    40  stm32f4xx_hal_eth.o(.text)
    ETH_MACReceptionDisable                  0x0800dbff   Thumb Code    40  stm32f4xx_hal_eth.o(.text)
    ETH_DMAReceptionDisable                  0x0800dc27   Thumb Code    22  stm32f4xx_hal_eth.o(.text)
    ETH_DMATransmissionDisable               0x0800dc3d   Thumb Code    22  stm32f4xx_hal_eth.o(.text)
    .text                                    0x0800deb4   Section        0  stm32f4xx_hal_dma.o(.text)
    DMA_CalcBaseAndBitshift                  0x0800deb5   Thumb Code    46  stm32f4xx_hal_dma.o(.text)
    DMA_SetConfig                            0x0800dfc7   Thumb Code    44  stm32f4xx_hal_dma.o(.text)
    .text                                    0x0800e4cc   Section        0  stm32f4xx_hal_iwdg.o(.text)
    .text                                    0x0800e5bc   Section        0  stm32f4xx_hal_rtc.o(.text)
    .text                                    0x0800f164   Section        0  stm32f4xx_hal_rtc_ex.o(.text)
    .text                                    0x0800ff04   Section        0  stm32f4xx_hal_tim.o(.text)
    TIM_DMAPeriodElapsedCplt                 0x080100ff   Thumb Code    20  stm32f4xx_hal_tim.o(.text)
    TIM_OC4_SetConfig                        0x080117c7   Thumb Code    88  stm32f4xx_hal_tim.o(.text)
    TIM_OC3_SetConfig                        0x0801181f   Thumb Code   122  stm32f4xx_hal_tim.o(.text)
    TIM_OC1_SetConfig                        0x08011909   Thumb Code   102  stm32f4xx_hal_tim.o(.text)
    TIM_TI4_SetConfig                        0x080119e3   Thumb Code    64  stm32f4xx_hal_tim.o(.text)
    TIM_TI3_SetConfig                        0x08011a23   Thumb Code    60  stm32f4xx_hal_tim.o(.text)
    TIM_TI2_SetConfig                        0x08011a5f   Thumb Code    62  stm32f4xx_hal_tim.o(.text)
    TIM_DMATriggerCplt                       0x08011e3b   Thumb Code    20  stm32f4xx_hal_tim.o(.text)
    TIM_ETR_SetConfig                        0x08012261   Thumb Code    24  stm32f4xx_hal_tim.o(.text)
    TIM_ITRx_SetConfig                       0x08012375   Thumb Code    20  stm32f4xx_hal_tim.o(.text)
    TIM_TI1_ConfigInputStage                 0x08012389   Thumb Code    42  stm32f4xx_hal_tim.o(.text)
    TIM_TI2_ConfigInputStage                 0x080123b3   Thumb Code    44  stm32f4xx_hal_tim.o(.text)
    TIM_SlaveTimer_SetConfig                 0x08012529   Thumb Code   164  stm32f4xx_hal_tim.o(.text)
    .text                                    0x080126fc   Section        0  stm32f4xx_hal_tim_ex.o(.text)
    TIM_CCxNChannelCmd                       0x0801297b   Thumb Code    28  stm32f4xx_hal_tim_ex.o(.text)
    .text                                    0x0801347c   Section        0  stm32f4xx_hal_spi.o(.text)
    SPI_WaitFlagStateUntilTimeout            0x08013543   Thumb Code   160  stm32f4xx_hal_spi.o(.text)
    SPI_CheckFlag_BSY                        0x080135e3   Thumb Code    40  stm32f4xx_hal_spi.o(.text)
    SPI_CheckForDisablingSPI                 0x08013767   Thumb Code    42  stm32f4xx_hal_spi.o(.text)
    SPI_CloseTx_ISR                          0x08013a99   Thumb Code    96  stm32f4xx_hal_spi.o(.text)
    SPI_TxISR_8BIT                           0x08013af9   Thumb Code    34  stm32f4xx_hal_spi.o(.text)
    SPI_TxISR_16BIT                          0x08013b1b   Thumb Code    36  stm32f4xx_hal_spi.o(.text)
    SPI_CloseRx_ISR                          0x08013bf1   Thumb Code    58  stm32f4xx_hal_spi.o(.text)
    SPI_RxISR_8BIT                           0x08013c2b   Thumb Code    34  stm32f4xx_hal_spi.o(.text)
    SPI_RxISR_16BIT                          0x08013c4d   Thumb Code    36  stm32f4xx_hal_spi.o(.text)
    SPI_CloseRxTx_ISR                        0x08013c73   Thumb Code    98  stm32f4xx_hal_spi.o(.text)
    SPI_2linesTxISR_8BIT                     0x08013cd5   Thumb Code    50  stm32f4xx_hal_spi.o(.text)
    SPI_2linesRxISR_8BIT                     0x08013d07   Thumb Code    50  stm32f4xx_hal_spi.o(.text)
    SPI_2linesTxISR_16BIT                    0x08013d39   Thumb Code    52  stm32f4xx_hal_spi.o(.text)
    SPI_2linesRxISR_16BIT                    0x08013d6d   Thumb Code    52  stm32f4xx_hal_spi.o(.text)
    SPI_DMAError                             0x08013f11   Thumb Code    40  stm32f4xx_hal_spi.o(.text)
    SPI_DMATransmitCplt                      0x08013f39   Thumb Code   150  stm32f4xx_hal_spi.o(.text)
    SPI_DMAHalfTransmitCplt                  0x08013fd1   Thumb Code    14  stm32f4xx_hal_spi.o(.text)
    SPI_DMAReceiveCplt                       0x0801409d   Thumb Code    76  stm32f4xx_hal_spi.o(.text)
    SPI_DMAHalfReceiveCplt                   0x080140eb   Thumb Code    14  stm32f4xx_hal_spi.o(.text)
    SPI_DMATransmitReceiveCplt               0x080140f9   Thumb Code    90  stm32f4xx_hal_spi.o(.text)
    SPI_DMAHalfTransmitReceiveCplt           0x08014155   Thumb Code    14  stm32f4xx_hal_spi.o(.text)
    .text                                    0x080144f0   Section       36  startup_stm32f407xx.o(.text)
    $v0                                      0x080144f0   Number         0  startup_stm32f407xx.o(.text)
    .text                                    0x08014514   Section        0  stm32f4xx_hal_msp.o(.text)
    .text                                    0x08014580   Section        0  ethernetif.o(.text)
    low_level_init                           0x08014583   Thumb Code   184  ethernetif.o(.text)
    low_level_output                         0x0801463b   Thumb Code   226  ethernetif.o(.text)
    low_level_input                          0x0801471d   Thumb Code   242  ethernetif.o(.text)
    .text                                    0x080149a8   Section        0  main.o(.text)
    Netif_Config                             0x080149a9   Thumb Code    86  main.o(.text)
    SystemClock_Config                       0x08014a27   Thumb Code   170  main.o(.text)
    .text                                    0x08014b0c   Section        0  stm32f4xx_it.o(.text)
    .text                                    0x08014f08   Section        0  app_ethernet.o(.text)
    .text                                    0x08014f4c   Section        0  httpd_cgi_ssi.o(.text)
    .text                                    0x08014f80   Section        0  httpd.o(.text)
    strnstr                                  0x08014f81   Thumb Code    74  httpd.o(.text)
    http_state_alloc                         0x08014fcb   Thumb Code    34  httpd.o(.text)
    http_state_free                          0x08014fed   Thumb Code    42  httpd.o(.text)
    http_write                               0x08015017   Thumb Code    86  httpd.o(.text)
    get_tag_insert                           0x0801506d   Thumb Code   178  httpd.o(.text)
    http_send_data                           0x0801511f   Thumb Code  1734  httpd.o(.text)
    http_poll                                0x080157e5   Thumb Code    92  httpd.o(.text)
    http_close_conn                          0x08015865   Thumb Code   130  httpd.o(.text)
    extract_uri_parameters                   0x080158e7   Thumb Code   126  httpd.o(.text)
    get_http_headers                         0x08015965   Thumb Code   272  httpd.o(.text)
    http_get_404_file                        0x08015a75   Thumb Code    54  httpd.o(.text)
    http_init_file                           0x08015aab   Thumb Code   138  httpd.o(.text)
    http_find_file                           0x08015b35   Thumb Code   384  httpd.o(.text)
    http_handle_post_finished                0x08015cb5   Thumb Code   144  httpd.o(.text)
    http_post_rxpbuf                         0x08015d63   Thumb Code    66  httpd.o(.text)
    http_post_request                        0x08015dc3   Thumb Code   324  httpd.o(.text)
    http_parse_request                       0x08015f07   Thumb Code   440  httpd.o(.text)
    http_err                                 0x080160bf   Thumb Code    22  httpd.o(.text)
    http_sent                                0x080160d5   Thumb Code    40  httpd.o(.text)
    http_recv                                0x08016271   Thumb Code   292  httpd.o(.text)
    http_accept                              0x08016395   Thumb Code    94  httpd.o(.text)
    httpd_init_addr                          0x080163f3   Thumb Code    72  httpd.o(.text)
    .text                                    0x080164dc   Section        0  fs.o(.text)
    fs_malloc                                0x080164dd   Thumb Code    54  fs.o(.text)
    fs_free                                  0x08016513   Thumb Code    48  fs.o(.text)
    .text                                    0x080165e4   Section        0  stm324xg_eval.o(.text)
    I2Cx_Init                                0x080165e5   Thumb Code     2  stm324xg_eval.o(.text)
    I2Cx_Error                               0x080165e7   Thumb Code    16  stm324xg_eval.o(.text)
    I2Cx_Read                                0x080165f7   Thumb Code    54  stm324xg_eval.o(.text)
    I2Cx_Write                               0x0801662d   Thumb Code    48  stm324xg_eval.o(.text)
    I2Cx_ReadMultiple                        0x0801665d   Thumb Code    60  stm324xg_eval.o(.text)
    I2Cx_WriteMultiple                       0x08016699   Thumb Code    60  stm324xg_eval.o(.text)
    I2Cx_IsDeviceReady                       0x080166d5   Thumb Code    20  stm324xg_eval.o(.text)
    .text                                    0x0801673c   Section        0  stm324xg_eval_eeprom.o(.text)
    EEPROM_WaitEepromStandbyState            0x0801677b   Thumb Code    26  stm324xg_eval_eeprom.o(.text)
    EEPROM_WritePage                         0x08016795   Thumb Code    64  stm324xg_eval_eeprom.o(.text)
    .text                                    0x0801697c   Section        0  init_l.o(.text)
    RTC_Init                                 0x0801697d   Thumb Code    76  init_l.o(.text)
    NVIC_Config                              0x080169c9   Thumb Code   126  init_l.o(.text)
    ADC_Config                               0x08016a47   Thumb Code   334  init_l.o(.text)
    TIM_Config_l                             0x08016bd5   Thumb Code   602  init_l.o(.text)
    MX_GPIO_Init_l                           0x08016e2f   Thumb Code   638  init_l.o(.text)
    RCC_Config_l                             0x080170ad   Thumb Code   806  init_l.o(.text)
    .text                                    0x08017480   Section        0  lab.o(.text)
    .text                                    0x08017960   Section        0  onewire.o(.text)
    OW_InternCommand                         0x08017d21   Thumb Code    80  onewire.o(.text)
    .text                                    0x08017efc   Section        0  process2.o(.text)
    Timer_Update                             0x08017efd   Thumb Code     2  process2.o(.text)
    SET_OCR_MOTOR                            0x08017eff   Thumb Code    18  process2.o(.text)
    SET_OCR_CEL                              0x08017f11   Thumb Code    22  process2.o(.text)
    SET_OCR_PWM                              0x08017f27   Thumb Code    22  process2.o(.text)
    Hot_STOP                                 0x08017f3d   Thumb Code   110  process2.o(.text)
    Attention                                0x08017fab   Thumb Code   634  process2.o(.text)
    PID_NBK                                  0x08018225   Thumb Code   176  process2.o(.text)
    NBK_process                              0x080182d5   Thumb Code  1150  process2.o(.text)
    PID_Power                                0x0801880b   Thumb Code   326  process2.o(.text)
    rectification_process                    0x08018951   Thumb Code   802  process2.o(.text)
    Change_OCR_PWM                           0x08018c73   Thumb Code    62  process2.o(.text)
    distillation_process                     0x08018cb1   Thumb Code   462  process2.o(.text)
    general_process                          0x08018e7f   Thumb Code    82  process2.o(.text)
    Get_Alcohol_Par                          0x08018ed1   Thumb Code   178  process2.o(.text)
    Get_Alcohol                              0x08018f83   Thumb Code   224  process2.o(.text)
    ReadTemperature                          0x08019063   Thumb Code   296  process2.o(.text)
    TIMER_change                             0x080198fd   Thumb Code   304  process2.o(.text)
    change_mode                              0x08019b45   Thumb Code   172  process2.o(.text)
    Update_OCR                               0x08019bf1   Thumb Code   134  process2.o(.text)
    RC5_val                                  0x08019c77   Thumb Code  1214  process2.o(.text)
    Save                                     0x0801a25f   Thumb Code   232  process2.o(.text)
    Key                                      0x0801a347   Thumb Code   422  process2.o(.text)
    RC5                                      0x0801a4ed   Thumb Code   130  process2.o(.text)
    Load                                     0x0801a56f   Thumb Code   164  process2.o(.text)
    WaterControl                             0x0801a683   Thumb Code   156  process2.o(.text)
    Change_OCR_CEL                           0x0801a71f   Thumb Code    62  process2.o(.text)
    .text                                    0x0801aa38   Section        0  rc5_ir_emul_receiver.o(.text)
    RC5_WaitForNextFallingEdge               0x0801aa39   Thumb Code    52  rc5_ir_emul_receiver.o(.text)
    RC5_TIM_GetCounterCLKValue               0x0801aa6d   Thumb Code    42  rc5_ir_emul_receiver.o(.text)
    .text                                    0x0801af18   Section        0  telnet.o(.text)
    Telnet_recv                              0x0801af19   Thumb Code   178  telnet.o(.text)
    Telnet_conn_err                          0x0801afcb   Thumb Code    16  telnet.o(.text)
    Telnet_accept                            0x0801afdb   Thumb Code    78  telnet.o(.text)
    .text                                    0x0801b068   Section        0  lcd_g.o(.text)
    .text                                    0x0801bcf4   Section        0  uldiv.o(.text)
    .text                                    0x0801bd56   Section        0  ldiv.o(.text)
    .text                                    0x0801bdb8   Section        0  memcpya.o(.text)
    .text                                    0x0801bddc   Section        0  memseta.o(.text)
    .text                                    0x0801be00   Section        0  strstr.o(.text)
    .text                                    0x0801be24   Section        0  strchr.o(.text)
    .text                                    0x0801be38   Section        0  strlen.o(.text)
    .text                                    0x0801be46   Section        0  strcmp.o(.text)
    .text                                    0x0801be62   Section        0  memcmp.o(.text)
    .text                                    0x0801be7c   Section        0  strcpy.o(.text)
    .text                                    0x0801be8e   Section        0  strncmp.o(.text)
    .text                                    0x0801beac   Section        0  strcspn.o(.text)
    .text                                    0x0801bece   Section        0  atoi.o(.text)
    .text                                    0x0801bee8   Section        0  dadd.o(.text)
    .text                                    0x0801c036   Section        0  dmul.o(.text)
    .text                                    0x0801c11a   Section        0  ffltul.o(.text)
    .text                                    0x0801c136   Section        0  dfltui.o(.text)
    .text                                    0x0801c150   Section        0  dfltul.o(.text)
    .text                                    0x0801c168   Section        0  dfixui.o(.text)
    .text                                    0x0801c19a   Section        0  f2d.o(.text)
    .text                                    0x0801c1c0   Section       48  cdcmple.o(.text)
    .text                                    0x0801c1f0   Section       48  cdrcmple.o(.text)
    .text                                    0x0801c220   Section        0  d2f.o(.text)
    .text                                    0x0801c258   Section        0  uidiv.o(.text)
    .text                                    0x0801c284   Section        0  llshl.o(.text)
    .text                                    0x0801c2a2   Section        0  llushr.o(.text)
    .text                                    0x0801c2c2   Section        0  llsshr.o(.text)
    .text                                    0x0801c2e6   Section        0  strtol.o(.text)
    .text                                    0x0801c356   Section        0  fepilogue.o(.text)
    .text                                    0x0801c356   Section        0  iusefp.o(.text)
    .text                                    0x0801c3c4   Section        0  depilogue.o(.text)
    .text                                    0x0801c47e   Section        0  ddiv.o(.text)
    .text                                    0x0801c55c   Section        0  dsqrt.o(.text)
    .text                                    0x0801c5fe   Section        0  dfixul.o(.text)
    .text                                    0x0801c630   Section       36  init.o(.text)
    .text                                    0x0801c654   Section        0  ctype_o.o(.text)
    .text                                    0x0801c65c   Section        0  _strtoul.o(.text)
    .text                                    0x0801c6fa   Section        0  _chval.o(.text)
    .text                                    0x0801c716   Section        0  __dczerorl2.o(.text)
    i.__0sprintf                             0x0801c76c   Section        0  printfa.o(i.__0sprintf)
    i.__aeabi_errno_addr                     0x0801c794   Section        0  errno.o(i.__aeabi_errno_addr)
    i.__hardfp_sqrt                          0x0801c79c   Section        0  sqrt.o(i.__hardfp_sqrt)
    i.__scatterload_copy                     0x0801c816   Section       14  handlers.o(i.__scatterload_copy)
    i.__scatterload_null                     0x0801c824   Section        2  handlers.o(i.__scatterload_null)
    i.__scatterload_zeroinit                 0x0801c826   Section       14  handlers.o(i.__scatterload_zeroinit)
    i.__set_errno                            0x0801c834   Section        0  errno.o(i.__set_errno)
    i._fp_digits                             0x0801c840   Section        0  printfa.o(i._fp_digits)
    _fp_digits                               0x0801c841   Thumb Code   366  printfa.o(i._fp_digits)
    i._printf_core                           0x0801c9c4   Section        0  printfa.o(i._printf_core)
    _printf_core                             0x0801c9c5   Thumb Code  1744  printfa.o(i._printf_core)
    i._printf_post_padding                   0x0801d0a0   Section        0  printfa.o(i._printf_post_padding)
    _printf_post_padding                     0x0801d0a1   Thumb Code    36  printfa.o(i._printf_post_padding)
    i._printf_pre_padding                    0x0801d0c4   Section        0  printfa.o(i._printf_pre_padding)
    _printf_pre_padding                      0x0801d0c5   Thumb Code    46  printfa.o(i._printf_pre_padding)
    i._sputc                                 0x0801d0f2   Section        0  printfa.o(i._sputc)
    _sputc                                   0x0801d0f3   Thumb Code    10  printfa.o(i._sputc)
    .constdata                               0x0801d0fc   Section       40  memp.o(.constdata)
    memp_sizes                               0x0801d0fc   Data          20  memp.o(.constdata)
    memp_num                                 0x0801d110   Data          20  memp.o(.constdata)
    .constdata                               0x0801d124   Section       80  tcp.o(.constdata)
    .constdata                               0x0801d174   Section        8  ip_addr.o(.constdata)
    .constdata                               0x0801d17c   Section       12  etharp.o(.constdata)
    .constdata                               0x0801d188   Section       16  stm32f4xx_hal_rcc.o(.constdata)
    .constdata                               0x0801d198   Section        8  stm32f4xx_hal_dma.o(.constdata)
    flagBitshiftOffset                       0x0801d198   Data           8  stm32f4xx_hal_dma.o(.constdata)
    .constdata                               0x0801d1a0   Section        8  httpd_cgi_ssi.o(.constdata)
    .constdata                               0x0801d1a8   Section       48  httpd.o(.constdata)
    .constdata                               0x0801d1d8   Section    176000  fs.o(.constdata)
    data__index_html                         0x0801d1d8   Data        7538  fs.o(.constdata)
    data__jquery_min_js                      0x0801ef4a   Data       96519  fs.o(.constdata)
    data__jquery_svg_css                     0x08036851   Data         335  fs.o(.constdata)
    data__jquery_svg_js                      0x080369a0   Data       58141  fs.o(.constdata)
    data__Press_png                          0x08044cbd   Data        9393  fs.o(.constdata)
    data__Pump_png                           0x0804716e   Data        2311  fs.o(.constdata)
    data__style_css                          0x08047a75   Data        1622  fs.o(.constdata)
    .constdata                               0x08048158   Section     5700  process2.o(.constdata)
    .constdata                               0x0804979c   Section    22804  tm_stm32f4_fonts.o(.constdata)
    .constdata                               0x0804f0b0   Section      129  ctype_o.o(.constdata)
    .constdata                               0x0804f134   Section        4  ctype_o.o(.constdata)
    table                                    0x0804f134   Data           4  ctype_o.o(.constdata)
    .conststring                             0x0804f138   Section      117  tcp.o(.conststring)
    .conststring                             0x0804f1b0   Section       14  httpd_cgi_ssi.o(.conststring)
    .conststring                             0x0804f1c0   Section     1088  httpd.o(.conststring)
    .conststring                             0x0804f600   Section      409  process2.o(.conststring)
    .conststring                             0x0804f79c   Section     1835  rc5_ir_emul_receiver.o(.conststring)
    .conststring                             0x0804fec8   Section     3073  img.o(.conststring)
    .data                                    0x20000000   Section       20  system_stm32f4xx.o(.data)
    .data                                    0x20000014   Section       32  tcp_in.o(.data)
    tcphdr                                   0x20000014   Data           4  tcp_in.o(.data)
    iphdr                                    0x20000018   Data           4  tcp_in.o(.data)
    seqno                                    0x2000001c   Data           4  tcp_in.o(.data)
    ackno                                    0x20000020   Data           4  tcp_in.o(.data)
    flags                                    0x20000024   Data           1  tcp_in.o(.data)
    tcplen                                   0x20000026   Data           2  tcp_in.o(.data)
    recv_flags                               0x20000028   Data           1  tcp_in.o(.data)
    recv_data                                0x2000002c   Data           4  tcp_in.o(.data)
    .data                                    0x20000034   Section       12  lwip_timers.o(.data)
    next_timeout                             0x20000034   Data           4  lwip_timers.o(.data)
    timeouts_last_time                       0x20000038   Data           4  lwip_timers.o(.data)
    tcpip_tcp_timer_active                   0x2000003c   Data           4  lwip_timers.o(.data)
    .data                                    0x20000040   Section        4  dhcp.o(.data)
    xid                                      0x20000040   Data           4  dhcp.o(.data)
    .data                                    0x20000044   Section        8  udp.o(.data)
    udp_port                                 0x20000044   Data           2  udp.o(.data)
    .data                                    0x2000004c   Section       12  mem.o(.data)
    ram                                      0x2000004c   Data           4  mem.o(.data)
    ram_end                                  0x20000050   Data           4  mem.o(.data)
    lfree                                    0x20000054   Data           4  mem.o(.data)
    .data                                    0x20000058   Section        9  netif.o(.data)
    netif_num                                0x20000060   Data           1  netif.o(.data)
    .data                                    0x20000064   Section       36  tcp.o(.data)
    tcp_port                                 0x20000064   Data           2  tcp.o(.data)
    tcp_timer                                0x20000081   Data           1  tcp.o(.data)
    tcp_timer_ctr                            0x20000082   Data           1  tcp.o(.data)
    iss                                      0x20000084   Data           4  tcp.o(.data)
    .data                                    0x20000088   Section        4  raw.o(.data)
    raw_pcbs                                 0x20000088   Data           4  raw.o(.data)
    .data                                    0x2000008c   Section        6  ip_frag.o(.data)
    reassdatagrams                           0x2000008c   Data           4  ip_frag.o(.data)
    ip_reass_pbufcount                       0x20000090   Data           2  ip_frag.o(.data)
    .data                                    0x20000094   Section       18  ip.o(.data)
    ip_id                                    0x200000a4   Data           2  ip.o(.data)
    .data                                    0x200000a6   Section        1  etharp.o(.data)
    etharp_cached_entry                      0x200000a6   Data           1  etharp.o(.data)
    .data                                    0x200000a8   Section        4  stm32f4xx_hal.o(.data)
    .data                                    0x200000ac   Section        4  ethernetif.o(.data)
    .data                                    0x200000b0   Section       44  stm32f4xx_it.o(.data)
    ADC_5_acc                                0x200000b0   Data           4  stm32f4xx_it.o(.data)
    ADC_Press_acc                            0x200000b4   Data           4  stm32f4xx_it.o(.data)
    Press_Atm                                0x200000b8   Data           4  stm32f4xx_it.o(.data)
    ADC_Conc_spirt_acc                       0x200000bc   Data           4  stm32f4xx_it.o(.data)
    integ                                    0x200000c0   Data           4  stm32f4xx_it.o(.data)
    sec_tmp                                  0x200000c4   Data           1  stm32f4xx_it.o(.data)
    period_tmp                               0x200000c8   Data           4  stm32f4xx_it.o(.data)
    tmp_loc3                                 0x200000d0   Data           8  stm32f4xx_it.o(.data)
    i_sum                                    0x200000d8   Data           2  stm32f4xx_it.o(.data)
    Counter_Triac2                           0x200000da   Data           2  stm32f4xx_it.o(.data)
    .data                                    0x200000dc   Section       16  httpd_cgi_ssi.o(.data)
    .data                                    0x200000ec   Section      288  httpd.o(.data)
    g_psHTTPHeaderStrings                    0x200000ec   Data         104  httpd.o(.data)
    g_psHTTPHeaders                          0x20000154   Data         136  httpd.o(.data)
    .data                                    0x2000020c   Section        7  stm324xg_eval_eeprom.o(.data)
    .data                                    0x20000213   Section        3  init_l.o(.data)
    .data                                    0x20000218   Section       36  lab.o(.data)
    .data                                    0x2000023c   Section      552  process2.o(.data)
    LCD_EditMenu_hist                        0x2000043e   Data           1  process2.o(.data)
    RC5_sticky_hist                          0x20000440   Data           4  process2.o(.data)
    sec1                                     0x20000444   Data           1  process2.o(.data)
    sec_tmp                                  0x20000445   Data           1  process2.o(.data)
    i_sum                                    0x20000448   Data           4  process2.o(.data)
    T_Par_Modee                              0x2000044c   Data           4  process2.o(.data)
    T_Par_END                                0x20000450   Data           4  process2.o(.data)
    NO_Stable_Mode                           0x20000454   Data           1  process2.o(.data)
    OCR_PWM_Hist                             0x20000455   Data           1  process2.o(.data)
    Tdef_set_rect_par                        0x20000458   Data           4  process2.o(.data)
    sec4                                     0x2000045c   Data           1  process2.o(.data)
    NumberAttention                          0x2000045d   Data           1  process2.o(.data)
    NumberAttentionSensor                    0x2000045e   Data           1  process2.o(.data)
    PWM                                      0x20000460   Data           4  process2.o(.data)
    .data                                    0x20000464   Section      680  rc5_ir_emul_receiver.o(.data)
    rc5_web                                  0x20000708   Data           1  rc5_ir_emul_receiver.o(.data)
    RC5_frame_struct                         0x20000709   Data           3  rc5_ir_emul_receiver.o(.data)
    .data                                    0x2000070c   Section       11  lcd_g.o(.data)
    .data                                    0x20000718   Section       48  tm_stm32f4_fonts.o(.data)
    .data                                    0x20000748   Section       24  img.o(.data)
    .data                                    0x20000760   Section        4  errno.o(.data)
    _errno                                   0x20000760   Data           4  errno.o(.data)
    .bss                                     0x20000764   Section       20  tcp_in.o(.bss)
    inseg                                    0x20000764   Data          20  tcp_in.o(.bss)
    .bss                                     0x20000778   Section    18475  memp.o(.bss)
    memp_tab                                 0x20000778   Data          40  memp.o(.bss)
    memp_memory                              0x200007a0   Data       18435  memp.o(.bss)
    .bss                                     0x20004fa4   Section       50  dhcp.o(.bss)
    .bss                                     0x20004fd6   Section    10260  mem.o(.bss)
    .bss                                     0x200077ea   Section       16  ip_addr.o(.bss)
    str                                      0x200077ea   Data          16  ip_addr.o(.bss)
    .bss                                     0x200077fc   Section      200  etharp.o(.bss)
    arp_table                                0x200077fc   Data         200  etharp.o(.bss)
    .bss                                     0x200078c4   Section    12520  ethernetif.o(.bss)
    .bss                                     0x2000a9ac   Section       56  main.o(.bss)
    .bss                                     0x2000a9e4   Section     2112  httpd.o(.bss)
    httpd_req_buf                            0x2000ade4   Data        1024  httpd.o(.bss)
    http_post_response_filename              0x2000b1e4   Data          64  httpd.o(.bss)
    .bss                                     0x2000b224   Section      240  fs.o(.bss)
    .bss                                     0x2000b314   Section      104  init_l.o(.bss)
    ADC_sConfig                              0x2000b314   Data          16  init_l.o(.bss)
    hdma_adc                                 0x2000b324   Data          88  init_l.o(.bss)
    .bss                                     0x2000b37c   Section     3492  lab.o(.bss)
    .bss                                     0x2000c120   Section       72  onewire.o(.bss)
    .bss                                     0x2000c168   Section    63332  process2.o(.bss)
    .bss                                     0x2001b8cc   Section       88  rc5_ir_emul_receiver.o(.bss)
    STACK                                    0x2001b928   Section     1024  startup_stm32f407xx.o(STACK)

    Global Symbols

    Symbol Name                              Value     Ov Type        Size  Object(Section)

    BuildAttributes$$THM_ISAv4$E$P$D$K$B$S$7EM$VFPi3$EXTD16$VFPS$VFMA$PE$A:L22UL41UL21$X:L11$S22US41US21$IEEE1$IW$USESV6$~STKCKD$USESV7$~SHL$OTIME$ROPI$IEEEJ$EBA8$MICROLIB$REQ8$PRES8$EABIv2 0x00000000   Number         0  anon$$obj.o ABSOLUTE
    __ARM_use_no_argv                        0x00000000   Number         0  main.o ABSOLUTE
    _printf_a                                0x00000000   Number         0  stubs.o ABSOLUTE
    _printf_c                                0x00000000   Number         0  stubs.o ABSOLUTE
    _printf_charcount                        0x00000000   Number         0  stubs.o ABSOLUTE
    _printf_d                                0x00000000   Number         0  stubs.o ABSOLUTE
    _printf_e                                0x00000000   Number         0  stubs.o ABSOLUTE
    _printf_f                                0x00000000   Number         0  stubs.o ABSOLUTE
    _printf_flags                            0x00000000   Number         0  stubs.o ABSOLUTE
    _printf_fp_dec                           0x00000000   Number         0  stubs.o ABSOLUTE
    _printf_fp_hex                           0x00000000   Number         0  stubs.o ABSOLUTE
    _printf_g                                0x00000000   Number         0  stubs.o ABSOLUTE
    _printf_i                                0x00000000   Number         0  stubs.o ABSOLUTE
    _printf_int_dec                          0x00000000   Number         0  stubs.o ABSOLUTE
    _printf_l                                0x00000000   Number         0  stubs.o ABSOLUTE
    _printf_lc                               0x00000000   Number         0  stubs.o ABSOLUTE
    _printf_ll                               0x00000000   Number         0  stubs.o ABSOLUTE
    _printf_lld                              0x00000000   Number         0  stubs.o ABSOLUTE
    _printf_lli                              0x00000000   Number         0  stubs.o ABSOLUTE
    _printf_llo                              0x00000000   Number         0  stubs.o ABSOLUTE
    _printf_llu                              0x00000000   Number         0  stubs.o ABSOLUTE
    _printf_llx                              0x00000000   Number         0  stubs.o ABSOLUTE
    _printf_longlong_dec                     0x00000000   Number         0  stubs.o ABSOLUTE
    _printf_longlong_hex                     0x00000000   Number         0  stubs.o ABSOLUTE
    _printf_longlong_oct                     0x00000000   Number         0  stubs.o ABSOLUTE
    _printf_ls                               0x00000000   Number         0  stubs.o ABSOLUTE
    _printf_mbtowc                           0x00000000   Number         0  stubs.o ABSOLUTE
    _printf_n                                0x00000000   Number         0  stubs.o ABSOLUTE
    _printf_o                                0x00000000   Number         0  stubs.o ABSOLUTE
    _printf_p                                0x00000000   Number         0  stubs.o ABSOLUTE
    _printf_percent                          0x00000000   Number         0  stubs.o ABSOLUTE
    _printf_pre_padding                      0x00000000   Number         0  stubs.o ABSOLUTE
    _printf_return_value                     0x00000000   Number         0  stubs.o ABSOLUTE
    _printf_s                                0x00000000   Number         0  stubs.o ABSOLUTE
    _printf_sizespec                         0x00000000   Number         0  stubs.o ABSOLUTE
    _printf_str                              0x00000000   Number         0  stubs.o ABSOLUTE
    _printf_truncate_signed                  0x00000000   Number         0  stubs.o ABSOLUTE
    _printf_truncate_unsigned                0x00000000   Number         0  stubs.o ABSOLUTE
    _printf_u                                0x00000000   Number         0  stubs.o ABSOLUTE
    _printf_wc                               0x00000000   Number         0  stubs.o ABSOLUTE
    _printf_wctomb                           0x00000000   Number         0  stubs.o ABSOLUTE
    _printf_widthprec                        0x00000000   Number         0  stubs.o ABSOLUTE
    _printf_x                                0x00000000   Number         0  stubs.o ABSOLUTE
    __cpp_initialize__aeabi_                  - Undefined Weak Reference
    __cxa_finalize                            - Undefined Weak Reference
    _clock_init                               - Undefined Weak Reference
    _microlib_exit                            - Undefined Weak Reference
    __Vectors_Size                           0x00000188   Number         0  startup_stm32f407xx.o ABSOLUTE
    __Vectors                                0x08000000   Data           4  startup_stm32f407xx.o(RESET)
    __Vectors_End                            0x08000188   Data           0  startup_stm32f407xx.o(RESET)
    __main                                   0x08000189   Thumb Code     0  entry.o(.ARM.Collect$$$$00000000)
    _main_stk                                0x08000189   Thumb Code     0  entry2.o(.ARM.Collect$$$$00000001)
    _main_scatterload                        0x0800018d   Thumb Code     0  entry5.o(.ARM.Collect$$$$00000004)
    __main_after_scatterload                 0x08000191   Thumb Code     0  entry5.o(.ARM.Collect$$$$00000004)
    _main_clock                              0x08000191   Thumb Code     0  entry7b.o(.ARM.Collect$$$$00000008)
    _main_cpp_init                           0x08000191   Thumb Code     0  entry8b.o(.ARM.Collect$$$$0000000A)
    _main_init                               0x08000191   Thumb Code     0  entry9a.o(.ARM.Collect$$$$0000000B)
    __rt_final_cpp                           0x08000199   Thumb Code     0  entry10a.o(.ARM.Collect$$$$0000000D)
    __rt_final_exit                          0x08000199   Thumb Code     0  entry11a.o(.ARM.Collect$$$$0000000F)
    SystemInit                               0x0800019d   Thumb Code    82  system_stm32f4xx.o(.text)
    SystemCoreClockUpdate                    0x080001ef   Thumb Code   174  system_stm32f4xx.o(.text)
    tcp_input                                0x08001145   Thumb Code  1154  tcp_in.o(.text)
    lwip_htons                               0x080015fd   Thumb Code    12  def.o(.text)
    lwip_ntohs                               0x08001609   Thumb Code    12  def.o(.text)
    lwip_htonl                               0x08001615   Thumb Code    26  def.o(.text)
    lwip_ntohl                               0x0800162f   Thumb Code    12  def.o(.text)
    sys_timeout                              0x0800163d   Thumb Code   152  lwip_timers.o(.text)
    tcp_timer_needed                         0x080016fd   Thumb Code    38  lwip_timers.o(.text)
    sys_timeouts_init                        0x0800178b   Thumb Code    60  lwip_timers.o(.text)
    sys_untimeout                            0x080017c7   Thumb Code    90  lwip_timers.o(.text)
    sys_check_timeouts                       0x08001821   Thumb Code    92  lwip_timers.o(.text)
    sys_restart_timeouts                     0x0800187d   Thumb Code    12  lwip_timers.o(.text)
    memp_init                                0x080018b1   Thumb Code    82  memp.o(.text)
    memp_malloc                              0x08001903   Thumb Code    44  memp.o(.text)
    memp_free                                0x0800192f   Thumb Code    28  memp.o(.text)
    dhcp_renew                               0x08001e61   Thumb Code   150  dhcp.o(.text)
    dhcp_coarse_tmr                          0x08001fdb   Thumb Code    74  dhcp.o(.text)
    dhcp_release                             0x080020d9   Thumb Code   178  dhcp.o(.text)
    dhcp_fine_tmr                            0x08002361   Thumb Code    68  dhcp.o(.text)
    dhcp_set_struct                          0x08002415   Thumb Code    30  dhcp.o(.text)
    dhcp_cleanup                             0x08002433   Thumb Code    24  dhcp.o(.text)
    dhcp_stop                                0x0800244b   Thumb Code    62  dhcp.o(.text)
    dhcp_start                               0x080028db   Thumb Code   238  dhcp.o(.text)
    dhcp_inform                              0x080029c9   Thumb Code   188  dhcp.o(.text)
    dhcp_network_changed                     0x08002a85   Thumb Code    80  dhcp.o(.text)
    dhcp_arp_reply                           0x08002b63   Thumb Code    58  dhcp.o(.text)
    udp_init                                 0x08002bb1   Thumb Code     2  udp.o(.text)
    udp_input                                0x08002c03   Thumb Code   470  udp.o(.text)
    udp_bind                                 0x08002dd9   Thumb Code   146  udp.o(.text)
    udp_sendto_if                            0x08002e6b   Thumb Code   240  udp.o(.text)
    udp_sendto                               0x08002f5b   Thumb Code    54  udp.o(.text)
    udp_send                                 0x08002f91   Thumb Code    36  udp.o(.text)
    udp_connect                              0x08002fb5   Thumb Code    98  udp.o(.text)
    udp_disconnect                           0x08003017   Thumb Code    16  udp.o(.text)
    udp_recv                                 0x08003027   Thumb Code     6  udp.o(.text)
    udp_remove                               0x0800302d   Thumb Code    60  udp.o(.text)
    udp_new                                  0x08003069   Thumb Code    28  udp.o(.text)
    mem_init                                 0x08003105   Thumb Code    74  mem.o(.text)
    mem_free                                 0x0800314f   Thumb Code    76  mem.o(.text)
    mem_trim                                 0x0800319b   Thumb Code   292  mem.o(.text)
    mem_malloc                               0x080032bf   Thumb Code   226  mem.o(.text)
    mem_calloc                               0x080033a1   Thumb Code    34  mem.o(.text)
    netif_init                               0x080033d5   Thumb Code     2  netif.o(.text)
    netif_set_gw                             0x080033d7   Thumb Code    16  netif.o(.text)
    netif_set_netmask                        0x080033e7   Thumb Code    16  netif.o(.text)
    netif_set_ipaddr                         0x080033f7   Thumb Code   124  netif.o(.text)
    netif_set_addr                           0x08003473   Thumb Code    40  netif.o(.text)
    netif_add                                0x0800349b   Thumb Code   132  netif.o(.text)
    netif_set_default                        0x0800351f   Thumb Code    10  netif.o(.text)
    netif_set_down                           0x08003529   Thumb Code    42  netif.o(.text)
    netif_remove                             0x08003553   Thumb Code    94  netif.o(.text)
    netif_find                               0x080035b1   Thumb Code    72  netif.o(.text)
    netif_set_up                             0x080035f9   Thumb Code    54  netif.o(.text)
    netif_set_link_up                        0x0800362f   Thumb Code    80  netif.o(.text)
    netif_set_link_down                      0x0800367f   Thumb Code    42  netif.o(.text)
    netif_set_link_callback                  0x080036a9   Thumb Code     6  netif.o(.text)
    tcp_init                                 0x080036c5   Thumb Code     2  tcp.o(.text)
    tcp_seg_free                             0x080036c7   Thumb Code    26  tcp.o(.text)
    tcp_segs_free                            0x080036e1   Thumb Code    24  tcp.o(.text)
    tcp_pcb_purge                            0x080036f9   Thumb Code    88  tcp.o(.text)
    tcp_slowtmr                              0x08003751   Thumb Code   832  tcp.o(.text)
    tcp_pcb_remove                           0x08003a91   Thumb Code   140  tcp.o(.text)
    tcp_close                                0x08003cf3   Thumb Code    28  tcp.o(.text)
    tcp_update_rcv_ann_wnd                   0x08003d0f   Thumb Code    78  tcp.o(.text)
    tcp_recved                               0x08003d5d   Thumb Code    74  tcp.o(.text)
    tcp_recv_null                            0x08003da7   Thumb Code    46  tcp.o(.text)
    tcp_process_refused_data                 0x08003dd5   Thumb Code   148  tcp.o(.text)
    tcp_fasttmr                              0x08003e69   Thumb Code   114  tcp.o(.text)
    tcp_tmr                                  0x08003edb   Thumb Code    30  tcp.o(.text)
    tcp_shutdown                             0x08003ef9   Thumb Code    98  tcp.o(.text)
    tcp_abandon                              0x08003f5b   Thumb Code   174  tcp.o(.text)
    tcp_abort                                0x08004009   Thumb Code    14  tcp.o(.text)
    tcp_bind                                 0x08004077   Thumb Code   146  tcp.o(.text)
    tcp_listen_with_backlog                  0x08004111   Thumb Code   198  tcp.o(.text)
    tcp_eff_send_mss                         0x080041d7   Thumb Code    46  tcp.o(.text)
    tcp_next_iss                             0x08004205   Thumb Code    20  tcp.o(.text)
    tcp_connect                              0x08004219   Thumb Code   328  tcp.o(.text)
    tcp_setprio                              0x08004361   Thumb Code     4  tcp.o(.text)
    tcp_alloc                                0x08004415   Thumb Code   182  tcp.o(.text)
    tcp_new                                  0x080044cb   Thumb Code    10  tcp.o(.text)
    tcp_arg                                  0x080044d5   Thumb Code     4  tcp.o(.text)
    tcp_recv                                 0x080044d9   Thumb Code     8  tcp.o(.text)
    tcp_sent                                 0x080044e1   Thumb Code     8  tcp.o(.text)
    tcp_err                                  0x080044e9   Thumb Code    10  tcp.o(.text)
    tcp_accept                               0x080044f3   Thumb Code     4  tcp.o(.text)
    tcp_poll                                 0x080044f7   Thumb Code    14  tcp.o(.text)
    tcp_debug_state_str                      0x08004505   Thumb Code    10  tcp.o(.text)
    tcp_enqueue_flags                        0x08004655   Thumb Code   294  tcp_out.o(.text)
    tcp_send_fin                             0x0800477b   Thumb Code    74  tcp_out.o(.text)
    tcp_write                                0x080048bd   Thumb Code   976  tcp_out.o(.text)
    tcp_send_empty_ack                       0x08004c8d   Thumb Code    84  tcp_out.o(.text)
    tcp_output                               0x08004db3   Thumb Code   444  tcp_out.o(.text)
    tcp_rst                                  0x08004f6f   Thumb Code   132  tcp_out.o(.text)
    tcp_rexmit_rto                           0x08004ff3   Thumb Code    58  tcp_out.o(.text)
    tcp_rexmit                               0x0800502d   Thumb Code    90  tcp_out.o(.text)
    tcp_rexmit_fast                          0x08005087   Thumb Code   120  tcp_out.o(.text)
    tcp_keepalive                            0x080050ff   Thumb Code    86  tcp_out.o(.text)
    tcp_zero_window_probe                    0x08005155   Thumb Code   180  tcp_out.o(.text)
    raw_input                                0x08005209   Thumb Code   102  raw.o(.text)
    raw_bind                                 0x0800526f   Thumb Code    16  raw.o(.text)
    raw_connect                              0x0800527f   Thumb Code    16  raw.o(.text)
    raw_recv                                 0x0800528f   Thumb Code     6  raw.o(.text)
    raw_sendto                               0x08005295   Thumb Code   172  raw.o(.text)
    raw_send                                 0x08005341   Thumb Code    18  raw.o(.text)
    raw_remove                               0x08005353   Thumb Code    60  raw.o(.text)
    raw_new                                  0x0800538f   Thumb Code    46  raw.o(.text)
    lwip_init                                0x080053c9   Thumb Code    28  init.o(.text)
    pbuf_free                                0x080053e5   Thumb Code   150  pbuf.o(.text)
    pbuf_alloc                               0x0800547b   Thumb Code   424  pbuf.o(.text)
    pbuf_alloced_custom                      0x08005623   Thumb Code   116  pbuf.o(.text)
    pbuf_realloc                             0x08005697   Thumb Code   120  pbuf.o(.text)
    pbuf_header                              0x0800570f   Thumb Code   134  pbuf.o(.text)
    pbuf_clen                                0x08005795   Thumb Code    18  pbuf.o(.text)
    pbuf_ref                                 0x080057a7   Thumb Code    10  pbuf.o(.text)
    pbuf_cat                                 0x080057b1   Thumb Code    56  pbuf.o(.text)
    pbuf_chain                               0x080057e9   Thumb Code    26  pbuf.o(.text)
    pbuf_dechain                             0x08005803   Thumb Code    66  pbuf.o(.text)
    pbuf_copy                                0x08005845   Thumb Code   200  pbuf.o(.text)
    pbuf_copy_partial                        0x0800590d   Thumb Code   146  pbuf.o(.text)
    pbuf_take                                0x0800599f   Thumb Code   116  pbuf.o(.text)
    pbuf_coalesce                            0x08005a13   Thumb Code    60  pbuf.o(.text)
    pbuf_get_at                              0x08005a4f   Thumb Code    46  pbuf.o(.text)
    pbuf_memcmp                              0x08005a7d   Thumb Code    96  pbuf.o(.text)
    pbuf_memfind                             0x08005add   Thumb Code    76  pbuf.o(.text)
    pbuf_strstr                              0x08005b29   Thumb Code    60  pbuf.o(.text)
    ip4_addr_isbroadcast                     0x08005b65   Thumb Code    78  ip_addr.o(.text)
    ip4_addr_netmask_valid                   0x08005bb3   Thumb Code    56  ip_addr.o(.text)
    ipaddr_aton                              0x08005beb   Thumb Code   348  ip_addr.o(.text)
    ipaddr_addr                              0x08005d47   Thumb Code    24  ip_addr.o(.text)
    ipaddr_ntoa_r                            0x08005d5f   Thumb Code   168  ip_addr.o(.text)
    ipaddr_ntoa                              0x08005e07   Thumb Code    16  ip_addr.o(.text)
    inet_chksum_pseudo                       0x08005e7b   Thumb Code   170  inet_chksum.o(.text)
    inet_chksum_pseudo_partial               0x08005f25   Thumb Code   192  inet_chksum.o(.text)
    inet_chksum                              0x08005fe5   Thumb Code    20  inet_chksum.o(.text)
    inet_chksum_pbuf                         0x08005ff9   Thumb Code    86  inet_chksum.o(.text)
    ip_reass_tmr                             0x08006115   Thumb Code    56  ip_frag.o(.text)
    ip_reass                                 0x08006377   Thumb Code   422  ip_frag.o(.text)
    ip_frag                                  0x08006559   Thumb Code   424  ip_frag.o(.text)
    ip_route                                 0x08006709   Thumb Code    80  ip.o(.text)
    ip_input                                 0x08006759   Thumb Code   484  ip.o(.text)
    ip_output_if                             0x0800693d   Thumb Code   204  ip.o(.text)
    ip_output                                0x08006a09   Thumb Code    60  ip.o(.text)
    icmp_input                               0x08006a61   Thumb Code   380  icmp.o(.text)
    icmp_dest_unreach                        0x08006c65   Thumb Code    18  icmp.o(.text)
    icmp_time_exceeded                       0x08006c77   Thumb Code    18  icmp.o(.text)
    etharp_tmr                               0x08006d01   Thumb Code   144  etharp.o(.text)
    etharp_cleanup_netif                     0x08007001   Thumb Code    52  etharp.o(.text)
    etharp_find_addr                         0x08007035   Thumb Code    90  etharp.o(.text)
    etharp_request                           0x0800727b   Thumb Code    40  etharp.o(.text)
    etharp_query                             0x0800730b   Thumb Code   362  etharp.o(.text)
    etharp_output                            0x08007475   Thumb Code   318  etharp.o(.text)
    ethernet_input                           0x080075b3   Thumb Code   198  etharp.o(.text)
    HAL_RCC_DeInit                           0x08007679   Thumb Code     2  stm32f4xx_hal_rcc.o(.text)
    HAL_RCC_OscConfig                        0x0800767b   Thumb Code   906  stm32f4xx_hal_rcc.o(.text)
    HAL_RCC_ClockConfig                      0x08007a05   Thumb Code   450  stm32f4xx_hal_rcc.o(.text)
    HAL_RCC_MCOConfig                        0x08007bc7   Thumb Code   186  stm32f4xx_hal_rcc.o(.text)
    HAL_RCC_EnableCSS                        0x08007c81   Thumb Code     8  stm32f4xx_hal_rcc.o(.text)
    HAL_RCC_DisableCSS                       0x08007c89   Thumb Code     8  stm32f4xx_hal_rcc.o(.text)
    HAL_RCC_GetSysClockFreq                  0x08007c91   Thumb Code   170  stm32f4xx_hal_rcc.o(.text)
    HAL_RCC_GetHCLKFreq                      0x08007d3b   Thumb Code    44  stm32f4xx_hal_rcc.o(.text)
    HAL_RCC_GetPCLK1Freq                     0x08007d67   Thumb Code    38  stm32f4xx_hal_rcc.o(.text)
    HAL_RCC_GetPCLK2Freq                     0x08007d8d   Thumb Code    38  stm32f4xx_hal_rcc.o(.text)
    HAL_RCC_GetOscConfig                     0x08007db3   Thumb Code   320  stm32f4xx_hal_rcc.o(.text)
    HAL_RCC_GetClockConfig                   0x08007ef3   Thumb Code    66  stm32f4xx_hal_rcc.o(.text)
    HAL_RCC_CSSCallback                      0x08007f35   Thumb Code     2  stm32f4xx_hal_rcc.o(.text)
    HAL_RCC_NMI_IRQHandler                   0x08007f37   Thumb Code    30  stm32f4xx_hal_rcc.o(.text)
    HAL_ADC_Init                             0x080080c9   Thumb Code   100  stm32f4xx_hal_adc.o(.text)
    HAL_ADC_MspDeInit                        0x0800812d   Thumb Code     2  stm32f4xx_hal_adc.o(.text)
    HAL_ADC_DeInit                           0x0800812f   Thumb Code    68  stm32f4xx_hal_adc.o(.text)
    HAL_ADC_Start                            0x08008173   Thumb Code   236  stm32f4xx_hal_adc.o(.text)
    HAL_ADC_Stop                             0x0800825f   Thumb Code    72  stm32f4xx_hal_adc.o(.text)
    HAL_ADC_PollForConversion                0x080082a7   Thumb Code   208  stm32f4xx_hal_adc.o(.text)
    HAL_ADC_PollForEvent                     0x08008377   Thumb Code   118  stm32f4xx_hal_adc.o(.text)
    HAL_ADC_Start_IT                         0x080083ed   Thumb Code   248  stm32f4xx_hal_adc.o(.text)
    HAL_ADC_Stop_IT                          0x080084e5   Thumb Code    86  stm32f4xx_hal_adc.o(.text)
    HAL_ADC_ErrorCallback                    0x0800853b   Thumb Code     2  stm32f4xx_hal_adc.o(.text)
    HAL_ADC_LevelOutOfWindowCallback         0x0800853d   Thumb Code     2  stm32f4xx_hal_adc.o(.text)
    HAL_ADC_ConvCpltCallback                 0x0800853f   Thumb Code     2  stm32f4xx_hal_adc.o(.text)
    HAL_ADC_IRQHandler                       0x08008541   Thumb Code   372  stm32f4xx_hal_adc.o(.text)
    HAL_ADC_ConvHalfCpltCallback             0x080086cf   Thumb Code     2  stm32f4xx_hal_adc.o(.text)
    HAL_ADC_Start_DMA                        0x0800874d   Thumb Code   334  stm32f4xx_hal_adc.o(.text)
    HAL_ADC_Stop_DMA                         0x0800889b   Thumb Code   108  stm32f4xx_hal_adc.o(.text)
    HAL_ADC_GetValue                         0x08008907   Thumb Code     8  stm32f4xx_hal_adc.o(.text)
    HAL_ADC_ConfigChannel                    0x0800890f   Thumb Code   386  stm32f4xx_hal_adc.o(.text)
    HAL_ADC_AnalogWDGConfig                  0x08008a91   Thumb Code   132  stm32f4xx_hal_adc.o(.text)
    HAL_ADC_GetState                         0x08008b15   Thumb Code     6  stm32f4xx_hal_adc.o(.text)
    HAL_ADC_GetError                         0x08008b1b   Thumb Code     6  stm32f4xx_hal_adc.o(.text)
    HAL_MspInit                              0x08008b35   Thumb Code     2  stm32f4xx_hal.o(.text)
    HAL_InitTick                             0x08008b37   Thumb Code    36  stm32f4xx_hal.o(.text)
    HAL_Init                                 0x08008b5b   Thumb Code    44  stm32f4xx_hal.o(.text)
    HAL_MspDeInit                            0x08008b87   Thumb Code     2  stm32f4xx_hal.o(.text)
    HAL_DeInit                               0x08008b89   Thumb Code    64  stm32f4xx_hal.o(.text)
    HAL_IncTick                              0x08008bc9   Thumb Code    12  stm32f4xx_hal.o(.text)
    HAL_GetTick                              0x08008bd5   Thumb Code     6  stm32f4xx_hal.o(.text)
    HAL_Delay                                0x08008bdb   Thumb Code    26  stm32f4xx_hal.o(.text)
    HAL_SuspendTick                          0x08008bf5   Thumb Code    18  stm32f4xx_hal.o(.text)
    HAL_ResumeTick                           0x08008c07   Thumb Code    18  stm32f4xx_hal.o(.text)
    HAL_GetHalVersion                        0x08008c19   Thumb Code     4  stm32f4xx_hal.o(.text)
    HAL_GetREVID                             0x08008c1d   Thumb Code     8  stm32f4xx_hal.o(.text)
    HAL_GetDEVID                             0x08008c25   Thumb Code    10  stm32f4xx_hal.o(.text)
    HAL_DBGMCU_EnableDBGSleepMode            0x08008c2f   Thumb Code    14  stm32f4xx_hal.o(.text)
    HAL_DBGMCU_DisableDBGSleepMode           0x08008c3d   Thumb Code    14  stm32f4xx_hal.o(.text)
    HAL_DBGMCU_EnableDBGStopMode             0x08008c4b   Thumb Code    14  stm32f4xx_hal.o(.text)
    HAL_DBGMCU_DisableDBGStopMode            0x08008c59   Thumb Code    14  stm32f4xx_hal.o(.text)
    HAL_DBGMCU_EnableDBGStandbyMode          0x08008c67   Thumb Code    14  stm32f4xx_hal.o(.text)
    HAL_DBGMCU_DisableDBGStandbyMode         0x08008c75   Thumb Code    14  stm32f4xx_hal.o(.text)
    HAL_EnableCompensationCell               0x08008c83   Thumb Code    22  stm32f4xx_hal.o(.text)
    HAL_DisableCompensationCell              0x08008c99   Thumb Code    24  stm32f4xx_hal.o(.text)
    HAL_GPIO_Init                            0x08008cc9   Thumb Code   476  stm32f4xx_hal_gpio.o(.text)
    HAL_GPIO_DeInit                          0x08008ea5   Thumb Code   326  stm32f4xx_hal_gpio.o(.text)
    HAL_GPIO_ReadPin                         0x08008feb   Thumb Code    16  stm32f4xx_hal_gpio.o(.text)
    HAL_GPIO_WritePin                        0x08008ffb   Thumb Code    12  stm32f4xx_hal_gpio.o(.text)
    HAL_GPIO_TogglePin                       0x08009007   Thumb Code     8  stm32f4xx_hal_gpio.o(.text)
    HAL_GPIO_LockPin                         0x0800900f   Thumb Code    46  stm32f4xx_hal_gpio.o(.text)
    HAL_GPIO_EXTI_Callback                   0x0800903d   Thumb Code     2  stm32f4xx_hal_gpio.o(.text)
    HAL_GPIO_EXTI_IRQHandler                 0x0800903f   Thumb Code    28  stm32f4xx_hal_gpio.o(.text)
    HAL_PWR_DeInit                           0x0800908d   Thumb Code    24  stm32f4xx_hal_pwr.o(.text)
    HAL_PWR_EnableBkUpAccess                 0x080090a5   Thumb Code    20  stm32f4xx_hal_pwr.o(.text)
    HAL_PWR_DisableBkUpAccess                0x080090b9   Thumb Code    22  stm32f4xx_hal_pwr.o(.text)
    HAL_PWR_ConfigPVD                        0x080090cf   Thumb Code   172  stm32f4xx_hal_pwr.o(.text)
    HAL_PWR_EnablePVD                        0x0800917b   Thumb Code    20  stm32f4xx_hal_pwr.o(.text)
    HAL_PWR_DisablePVD                       0x0800918f   Thumb Code    20  stm32f4xx_hal_pwr.o(.text)
    HAL_PWR_EnableWakeUpPin                  0x080091a3   Thumb Code    12  stm32f4xx_hal_pwr.o(.text)
    HAL_PWR_DisableWakeUpPin                 0x080091af   Thumb Code    12  stm32f4xx_hal_pwr.o(.text)
    HAL_PWR_EnterSLEEPMode                   0x080091bb   Thumb Code    28  stm32f4xx_hal_pwr.o(.text)
    HAL_PWR_EnterSTOPMode                    0x080091d7   Thumb Code    54  stm32f4xx_hal_pwr.o(.text)
    HAL_PWR_EnterSTANDBYMode                 0x0800920d   Thumb Code    32  stm32f4xx_hal_pwr.o(.text)
    HAL_PWR_PVDCallback                      0x0800922d   Thumb Code     2  stm32f4xx_hal_pwr.o(.text)
    HAL_PWR_PVD_IRQHandler                   0x0800922f   Thumb Code    30  stm32f4xx_hal_pwr.o(.text)
    HAL_PWR_EnableSleepOnExit                0x0800924d   Thumb Code    14  stm32f4xx_hal_pwr.o(.text)
    HAL_PWR_DisableSleepOnExit               0x0800925b   Thumb Code    14  stm32f4xx_hal_pwr.o(.text)
    HAL_PWR_EnableSEVOnPend                  0x08009269   Thumb Code    14  stm32f4xx_hal_pwr.o(.text)
    HAL_PWR_DisableSEVOnPend                 0x08009277   Thumb Code    14  stm32f4xx_hal_pwr.o(.text)
    HAL_NVIC_SetPriorityGrouping             0x080092b9   Thumb Code    36  stm32f4xx_hal_cortex.o(.text)
    HAL_NVIC_SetPriority                     0x080092dd   Thumb Code   124  stm32f4xx_hal_cortex.o(.text)
    HAL_NVIC_EnableIRQ                       0x08009359   Thumb Code    26  stm32f4xx_hal_cortex.o(.text)
    HAL_NVIC_DisableIRQ                      0x08009373   Thumb Code    22  stm32f4xx_hal_cortex.o(.text)
    HAL_NVIC_SystemReset                     0x08009389   Thumb Code    64  stm32f4xx_hal_cortex.o(.text)
    HAL_SYSTICK_Config                       0x080093c9   Thumb Code    52  stm32f4xx_hal_cortex.o(.text)
    HAL_MPU_ConfigRegion                     0x080093fd   Thumb Code    90  stm32f4xx_hal_cortex.o(.text)
    HAL_NVIC_GetPriorityGrouping             0x08009457   Thumb Code     8  stm32f4xx_hal_cortex.o(.text)
    HAL_NVIC_GetPriority                     0x0800945f   Thumb Code   138  stm32f4xx_hal_cortex.o(.text)
    HAL_NVIC_SetPendingIRQ                   0x080094e9   Thumb Code    24  stm32f4xx_hal_cortex.o(.text)
    HAL_NVIC_GetPendingIRQ                   0x08009501   Thumb Code    38  stm32f4xx_hal_cortex.o(.text)
    HAL_NVIC_ClearPendingIRQ                 0x08009527   Thumb Code    22  stm32f4xx_hal_cortex.o(.text)
    HAL_NVIC_GetActive                       0x0800953d   Thumb Code    38  stm32f4xx_hal_cortex.o(.text)
    HAL_SYSTICK_CLKSourceConfig              0x08009563   Thumb Code    40  stm32f4xx_hal_cortex.o(.text)
    HAL_SYSTICK_Callback                     0x0800958b   Thumb Code     2  stm32f4xx_hal_cortex.o(.text)
    HAL_SYSTICK_IRQHandler                   0x0800958d   Thumb Code     8  stm32f4xx_hal_cortex.o(.text)
    HAL_I2C_MspInit                          0x080095b5   Thumb Code     2  stm32f4xx_hal_i2c.o(.text)
    HAL_I2C_Init                             0x080095b7   Thumb Code   286  stm32f4xx_hal_i2c.o(.text)
    HAL_I2C_MspDeInit                        0x080096d5   Thumb Code     2  stm32f4xx_hal_i2c.o(.text)
    HAL_I2C_DeInit                           0x080096d7   Thumb Code    60  stm32f4xx_hal_i2c.o(.text)
    HAL_I2C_Master_Transmit                  0x08009a4d   Thumb Code   320  stm32f4xx_hal_i2c.o(.text)
    HAL_I2C_Master_Receive                   0x08009d2b   Thumb Code   630  stm32f4xx_hal_i2c.o(.text)
    HAL_I2C_Slave_Transmit                   0x08009fa1   Thumb Code   350  stm32f4xx_hal_i2c.o(.text)
    HAL_I2C_Slave_Receive                    0x0800a157   Thumb Code   350  stm32f4xx_hal_i2c.o(.text)
    HAL_I2C_Master_Transmit_IT               0x0800a2b5   Thumb Code   250  stm32f4xx_hal_i2c.o(.text)
    HAL_I2C_Master_Receive_IT                0x0800a3af   Thumb Code   372  stm32f4xx_hal_i2c.o(.text)
    HAL_I2C_Master_Sequential_Transmit_IT    0x0800a523   Thumb Code   272  stm32f4xx_hal_i2c.o(.text)
    HAL_I2C_Master_Sequential_Receive_IT     0x0800a633   Thumb Code   494  stm32f4xx_hal_i2c.o(.text)
    HAL_I2C_Slave_Transmit_IT                0x0800a821   Thumb Code   146  stm32f4xx_hal_i2c.o(.text)
    HAL_I2C_Slave_Receive_IT                 0x0800a8b3   Thumb Code   146  stm32f4xx_hal_i2c.o(.text)
    HAL_I2C_Slave_Sequential_Transmit_IT     0x0800a945   Thumb Code   128  stm32f4xx_hal_i2c.o(.text)
    HAL_I2C_Slave_Sequential_Receive_IT      0x0800a9c5   Thumb Code   128  stm32f4xx_hal_i2c.o(.text)
    HAL_I2C_EnableListen_IT                  0x0800aa45   Thumb Code    48  stm32f4xx_hal_i2c.o(.text)
    HAL_I2C_DisableListen_IT                 0x0800aa75   Thumb Code    70  stm32f4xx_hal_i2c.o(.text)
    HAL_I2C_ErrorCallback                    0x0800aabb   Thumb Code     2  stm32f4xx_hal_i2c.o(.text)
    HAL_I2C_MasterTxCpltCallback             0x0800aaef   Thumb Code     2  stm32f4xx_hal_i2c.o(.text)
    HAL_I2C_Master_Transmit_DMA              0x0800ab49   Thumb Code   354  stm32f4xx_hal_i2c.o(.text)
    HAL_I2C_MasterRxCpltCallback             0x0800acab   Thumb Code     2  stm32f4xx_hal_i2c.o(.text)
    HAL_I2C_Master_Receive_DMA               0x0800ad07   Thumb Code   346  stm32f4xx_hal_i2c.o(.text)
    HAL_I2C_Master_Abort_IT                  0x0800ae61   Thumb Code   118  stm32f4xx_hal_i2c.o(.text)
    HAL_I2C_SlaveTxCpltCallback              0x0800aed7   Thumb Code     2  stm32f4xx_hal_i2c.o(.text)
    HAL_I2C_Slave_Transmit_DMA               0x0800af3b   Thumb Code   318  stm32f4xx_hal_i2c.o(.text)
    HAL_I2C_SlaveRxCpltCallback              0x0800b079   Thumb Code     2  stm32f4xx_hal_i2c.o(.text)
    HAL_I2C_Slave_Receive_DMA                0x0800b0fb   Thumb Code   214  stm32f4xx_hal_i2c.o(.text)
    HAL_I2C_Mem_Write                        0x0800b2a1   Thumb Code   304  stm32f4xx_hal_i2c.o(.text)
    HAL_I2C_Mem_Read                         0x0800b529   Thumb Code   612  stm32f4xx_hal_i2c.o(.text)
    HAL_I2C_Mem_Write_IT                     0x0800b78d   Thumb Code   244  stm32f4xx_hal_i2c.o(.text)
    HAL_I2C_Mem_Read_IT                      0x0800b881   Thumb Code   400  stm32f4xx_hal_i2c.o(.text)
    HAL_I2C_MemTxCpltCallback                0x0800ba11   Thumb Code     2  stm32f4xx_hal_i2c.o(.text)
    HAL_I2C_Mem_Write_DMA                    0x0800ba6b   Thumb Code   314  stm32f4xx_hal_i2c.o(.text)
    HAL_I2C_MemRxCpltCallback                0x0800bba5   Thumb Code     2  stm32f4xx_hal_i2c.o(.text)
    HAL_I2C_Mem_Read_DMA                     0x0800bc01   Thumb Code   366  stm32f4xx_hal_i2c.o(.text)
    HAL_I2C_IsDeviceReady                    0x0800bd6f   Thumb Code   426  stm32f4xx_hal_i2c.o(.text)
    HAL_I2C_ListenCpltCallback               0x0800bff9   Thumb Code     2  stm32f4xx_hal_i2c.o(.text)
    HAL_I2C_AddrCallback                     0x0800c083   Thumb Code     2  stm32f4xx_hal_i2c.o(.text)
    HAL_I2C_EV_IRQHandler                    0x0800c3bb   Thumb Code   374  stm32f4xx_hal_i2c.o(.text)
    HAL_I2C_ER_IRQHandler                    0x0800c5e1   Thumb Code   332  stm32f4xx_hal_i2c.o(.text)
    HAL_I2C_GetState                         0x0800c72d   Thumb Code     8  stm32f4xx_hal_i2c.o(.text)
    HAL_I2C_GetMode                          0x0800c735   Thumb Code     8  stm32f4xx_hal_i2c.o(.text)
    HAL_I2C_GetError                         0x0800c73d   Thumb Code     6  stm32f4xx_hal_i2c.o(.text)
    HAL_ADCEx_InjectedStart                  0x0800c749   Thumb Code   252  stm32f4xx_hal_adc_ex.o(.text)
    HAL_ADCEx_InjectedStart_IT               0x0800c845   Thumb Code   264  stm32f4xx_hal_adc_ex.o(.text)
    HAL_ADCEx_InjectedStop                   0x0800c94d   Thumb Code   104  stm32f4xx_hal_adc_ex.o(.text)
    HAL_ADCEx_InjectedPollForConversion      0x0800c9b5   Thumb Code   160  stm32f4xx_hal_adc_ex.o(.text)
    HAL_ADCEx_InjectedStop_IT                0x0800ca55   Thumb Code   116  stm32f4xx_hal_adc_ex.o(.text)
    HAL_ADCEx_InjectedGetValue               0x0800cac9   Thumb Code    70  stm32f4xx_hal_adc_ex.o(.text)
    HAL_ADCEx_MultiModeStart_DMA             0x0800cbb9   Thumb Code   278  stm32f4xx_hal_adc_ex.o(.text)
    HAL_ADCEx_MultiModeStop_DMA              0x0800cccf   Thumb Code   108  stm32f4xx_hal_adc_ex.o(.text)
    HAL_ADCEx_MultiModeGetValue              0x0800cd3b   Thumb Code    10  stm32f4xx_hal_adc_ex.o(.text)
    HAL_ADCEx_InjectedConvCpltCallback       0x0800cd45   Thumb Code     2  stm32f4xx_hal_adc_ex.o(.text)
    HAL_ADCEx_InjectedConfigChannel          0x0800cd47   Thumb Code   548  stm32f4xx_hal_adc_ex.o(.text)
    HAL_ADCEx_MultiModeConfigChannel         0x0800cf6b   Thumb Code   162  stm32f4xx_hal_adc_ex.o(.text)
    HAL_ETH_WritePHYRegister                 0x0800d273   Thumb Code   144  stm32f4xx_hal_eth.o(.text)
    HAL_ETH_ReadPHYRegister                  0x0800d303   Thumb Code   146  stm32f4xx_hal_eth.o(.text)
    HAL_ETH_Init                             0x0800d397   Thumb Code   670  stm32f4xx_hal_eth.o(.text)
    HAL_ETH_MspDeInit                        0x0800d635   Thumb Code     2  stm32f4xx_hal_eth.o(.text)
    HAL_ETH_DeInit                           0x0800d637   Thumb Code    32  stm32f4xx_hal_eth.o(.text)
    HAL_ETH_DMATxDescListInit                0x0800d657   Thumb Code   132  stm32f4xx_hal_eth.o(.text)
    HAL_ETH_DMARxDescListInit                0x0800d6db   Thumb Code   140  stm32f4xx_hal_eth.o(.text)
    HAL_ETH_TransmitFrame                    0x0800d767   Thumb Code   340  stm32f4xx_hal_eth.o(.text)
    HAL_ETH_GetReceivedFrame                 0x0800d8bb   Thumb Code   178  stm32f4xx_hal_eth.o(.text)
    HAL_ETH_GetReceivedFrame_IT              0x0800d96d   Thumb Code   186  stm32f4xx_hal_eth.o(.text)
    HAL_ETH_ErrorCallback                    0x0800da27   Thumb Code     2  stm32f4xx_hal_eth.o(.text)
    HAL_ETH_TxCpltCallback                   0x0800da29   Thumb Code     2  stm32f4xx_hal_eth.o(.text)
    HAL_ETH_RxCpltCallback                   0x0800da2b   Thumb Code     2  stm32f4xx_hal_eth.o(.text)
    HAL_ETH_IRQHandler                       0x0800da2d   Thumb Code   164  stm32f4xx_hal_eth.o(.text)
    HAL_ETH_Start                            0x0800db85   Thumb Code    82  stm32f4xx_hal_eth.o(.text)
    HAL_ETH_Stop                             0x0800dc53   Thumb Code    82  stm32f4xx_hal_eth.o(.text)
    HAL_ETH_ConfigMAC                        0x0800dca5   Thumb Code   314  stm32f4xx_hal_eth.o(.text)
    HAL_ETH_ConfigDMA                        0x0800dddf   Thumb Code   196  stm32f4xx_hal_eth.o(.text)
    HAL_ETH_GetState                         0x0800dea3   Thumb Code     8  stm32f4xx_hal_eth.o(.text)
    HAL_DMA_Init                             0x0800dee3   Thumb Code   128  stm32f4xx_hal_dma.o(.text)
    HAL_DMA_DeInit                           0x0800df63   Thumb Code   100  stm32f4xx_hal_dma.o(.text)
    HAL_DMA_Start                            0x0800dff3   Thumb Code    82  stm32f4xx_hal_dma.o(.text)
    HAL_DMA_Start_IT                         0x0800e045   Thumb Code   106  stm32f4xx_hal_dma.o(.text)
    HAL_DMA_Abort                            0x0800e0af   Thumb Code    94  stm32f4xx_hal_dma.o(.text)
    HAL_DMA_PollForTransfer                  0x0800e10d   Thumb Code   412  stm32f4xx_hal_dma.o(.text)
    HAL_DMA_IRQHandler                       0x0800e2a9   Thumb Code   530  stm32f4xx_hal_dma.o(.text)
    HAL_DMA_GetState                         0x0800e4bb   Thumb Code     8  stm32f4xx_hal_dma.o(.text)
    HAL_DMA_GetError                         0x0800e4c3   Thumb Code     6  stm32f4xx_hal_dma.o(.text)
    HAL_IWDG_MspInit                         0x0800e4cd   Thumb Code     2  stm32f4xx_hal_iwdg.o(.text)
    HAL_IWDG_Init                            0x0800e4cf   Thumb Code    76  stm32f4xx_hal_iwdg.o(.text)
    HAL_IWDG_Start                           0x0800e51b   Thumb Code    56  stm32f4xx_hal_iwdg.o(.text)
    HAL_IWDG_Refresh                         0x0800e553   Thumb Code   100  stm32f4xx_hal_iwdg.o(.text)
    HAL_IWDG_GetState                        0x0800e5b7   Thumb Code     6  stm32f4xx_hal_iwdg.o(.text)
    RTC_EnterInitMode                        0x0800e5bd   Thumb Code    62  stm32f4xx_hal_rtc.o(.text)
    HAL_RTC_MspInit                          0x0800e5fb   Thumb Code     2  stm32f4xx_hal_rtc.o(.text)
    HAL_RTC_Init                             0x0800e5fd   Thumb Code   176  stm32f4xx_hal_rtc.o(.text)
    HAL_RTC_MspDeInit                        0x0800e6ad   Thumb Code     2  stm32f4xx_hal_rtc.o(.text)
    HAL_RTC_WaitForSynchro                   0x0800e6af   Thumb Code    58  stm32f4xx_hal_rtc.o(.text)
    HAL_RTC_DeInit                           0x0800e6e9   Thumb Code   254  stm32f4xx_hal_rtc.o(.text)
    RTC_Bcd2ToByte                           0x0800e7e7   Thumb Code    22  stm32f4xx_hal_rtc.o(.text)
    RTC_ByteToBcd2                           0x0800e7fd   Thumb Code    26  stm32f4xx_hal_rtc.o(.text)
    HAL_RTC_SetTime                          0x0800e817   Thumb Code   304  stm32f4xx_hal_rtc.o(.text)
    HAL_RTC_GetTime                          0x0800e947   Thumb Code    92  stm32f4xx_hal_rtc.o(.text)
    HAL_RTC_SetDate                          0x0800e9a3   Thumb Code   284  stm32f4xx_hal_rtc.o(.text)
    HAL_RTC_GetDate                          0x0800eabf   Thumb Code    72  stm32f4xx_hal_rtc.o(.text)
    HAL_RTC_SetAlarm                         0x0800eb07   Thumb Code   488  stm32f4xx_hal_rtc.o(.text)
    HAL_RTC_SetAlarm_IT                      0x0800ecef   Thumb Code   554  stm32f4xx_hal_rtc.o(.text)
    HAL_RTC_DeactivateAlarm                  0x0800ef19   Thumb Code   244  stm32f4xx_hal_rtc.o(.text)
    HAL_RTC_GetAlarm                         0x0800f00d   Thumb Code   154  stm32f4xx_hal_rtc.o(.text)
    HAL_RTC_AlarmAEventCallback              0x0800f0a7   Thumb Code     2  stm32f4xx_hal_rtc.o(.text)
    HAL_RTC_AlarmIRQHandler                  0x0800f0a9   Thumb Code   104  stm32f4xx_hal_rtc.o(.text)
    HAL_RTC_PollForAlarmAEvent               0x0800f111   Thumb Code    74  stm32f4xx_hal_rtc.o(.text)
    HAL_RTC_GetState                         0x0800f15b   Thumb Code     6  stm32f4xx_hal_rtc.o(.text)
    HAL_RTCEx_SetTimeStamp                   0x0800f165   Thumb Code   122  stm32f4xx_hal_rtc_ex.o(.text)
    HAL_RTCEx_SetTimeStamp_IT                0x0800f1df   Thumb Code   162  stm32f4xx_hal_rtc_ex.o(.text)
    HAL_RTCEx_DeactivateTimeStamp            0x0800f281   Thumb Code    96  stm32f4xx_hal_rtc_ex.o(.text)
    HAL_RTCEx_GetTimeStamp                   0x0800f2e1   Thumb Code   166  stm32f4xx_hal_rtc_ex.o(.text)
    HAL_RTCEx_SetTamper                      0x0800f387   Thumb Code   124  stm32f4xx_hal_rtc_ex.o(.text)
    HAL_RTCEx_SetTamper_IT                   0x0800f403   Thumb Code   160  stm32f4xx_hal_rtc_ex.o(.text)
    HAL_RTCEx_DeactivateTamper               0x0800f4a3   Thumb Code    50  stm32f4xx_hal_rtc_ex.o(.text)
    HAL_RTCEx_Tamper2EventCallback           0x0800f4d5   Thumb Code     2  stm32f4xx_hal_rtc_ex.o(.text)
    HAL_RTCEx_Tamper1EventCallback           0x0800f4d7   Thumb Code     2  stm32f4xx_hal_rtc_ex.o(.text)
    HAL_RTCEx_TimeStampEventCallback         0x0800f4d9   Thumb Code     2  stm32f4xx_hal_rtc_ex.o(.text)
    HAL_RTCEx_TamperTimeStampIRQHandler      0x0800f4db   Thumb Code   146  stm32f4xx_hal_rtc_ex.o(.text)
    HAL_RTCEx_PollForTimeStampEvent          0x0800f56d   Thumb Code    92  stm32f4xx_hal_rtc_ex.o(.text)
    HAL_RTCEx_PollForTamper1Event            0x0800f5c9   Thumb Code    74  stm32f4xx_hal_rtc_ex.o(.text)
    HAL_RTCEx_PollForTamper2Event            0x0800f613   Thumb Code    86  stm32f4xx_hal_rtc_ex.o(.text)
    HAL_RTCEx_SetWakeUpTimer                 0x0800f669   Thumb Code   254  stm32f4xx_hal_rtc_ex.o(.text)
    HAL_RTCEx_SetWakeUpTimer_IT              0x0800f767   Thumb Code   294  stm32f4xx_hal_rtc_ex.o(.text)
    HAL_RTCEx_DeactivateWakeUpTimer          0x0800f88d   Thumb Code   152  stm32f4xx_hal_rtc_ex.o(.text)
    HAL_RTCEx_GetWakeUpTimer                 0x0800f925   Thumb Code    10  stm32f4xx_hal_rtc_ex.o(.text)
    HAL_RTCEx_WakeUpTimerEventCallback       0x0800f92f   Thumb Code     2  stm32f4xx_hal_rtc_ex.o(.text)
    HAL_RTCEx_WakeUpTimerIRQHandler          0x0800f931   Thumb Code    62  stm32f4xx_hal_rtc_ex.o(.text)
    HAL_RTCEx_PollForWakeUpTimerEvent        0x0800f96f   Thumb Code    74  stm32f4xx_hal_rtc_ex.o(.text)
    HAL_RTCEx_BKUPWrite                      0x0800f9b9   Thumb Code    18  stm32f4xx_hal_rtc_ex.o(.text)
    HAL_RTCEx_BKUPRead                       0x0800f9cb   Thumb Code    18  stm32f4xx_hal_rtc_ex.o(.text)
    HAL_RTCEx_SetCoarseCalib                 0x0800f9dd   Thumb Code   138  stm32f4xx_hal_rtc_ex.o(.text)
    HAL_RTCEx_DeactivateCoarseCalib          0x0800fa67   Thumb Code   126  stm32f4xx_hal_rtc_ex.o(.text)
    HAL_RTCEx_SetSmoothCalib                 0x0800fae5   Thumb Code   162  stm32f4xx_hal_rtc_ex.o(.text)
    HAL_RTCEx_SetSynchroShift                0x0800fb87   Thumb Code   230  stm32f4xx_hal_rtc_ex.o(.text)
    HAL_RTCEx_SetCalibrationOutPut           0x0800fc6d   Thumb Code   100  stm32f4xx_hal_rtc_ex.o(.text)
    HAL_RTCEx_DeactivateCalibrationOutPut    0x0800fcd1   Thumb Code    78  stm32f4xx_hal_rtc_ex.o(.text)
    HAL_RTCEx_SetRefClock                    0x0800fd1f   Thumb Code   126  stm32f4xx_hal_rtc_ex.o(.text)
    HAL_RTCEx_DeactivateRefClock             0x0800fd9d   Thumb Code   126  stm32f4xx_hal_rtc_ex.o(.text)
    HAL_RTCEx_EnableBypassShadow             0x0800fe1b   Thumb Code    78  stm32f4xx_hal_rtc_ex.o(.text)
    HAL_RTCEx_DisableBypassShadow            0x0800fe69   Thumb Code    78  stm32f4xx_hal_rtc_ex.o(.text)
    HAL_RTCEx_AlarmBEventCallback            0x0800feb7   Thumb Code     2  stm32f4xx_hal_rtc_ex.o(.text)
    HAL_RTCEx_PollForAlarmBEvent             0x0800feb9   Thumb Code    74  stm32f4xx_hal_rtc_ex.o(.text)
    TIM_Base_SetConfig                       0x0800ff05   Thumb Code   184  stm32f4xx_hal_tim.o(.text)
    HAL_TIM_Base_MspInit                     0x0800ffbd   Thumb Code     2  stm32f4xx_hal_tim.o(.text)
    HAL_TIM_Base_Init                        0x0800ffbf   Thumb Code    52  stm32f4xx_hal_tim.o(.text)
    HAL_TIM_Base_MspDeInit                   0x0800fff3   Thumb Code     2  stm32f4xx_hal_tim.o(.text)
    HAL_TIM_Base_DeInit                      0x0800fff5   Thumb Code    70  stm32f4xx_hal_tim.o(.text)
    HAL_TIM_Base_Start                       0x0801003b   Thumb Code    30  stm32f4xx_hal_tim.o(.text)
    HAL_TIM_Base_Stop                        0x08010059   Thumb Code    56  stm32f4xx_hal_tim.o(.text)
    HAL_TIM_Base_Start_IT                    0x08010091   Thumb Code    30  stm32f4xx_hal_tim.o(.text)
    HAL_TIM_Base_Stop_IT                     0x080100af   Thumb Code    56  stm32f4xx_hal_tim.o(.text)
    HAL_TIM_ErrorCallback                    0x080100e7   Thumb Code     2  stm32f4xx_hal_tim.o(.text)
    TIM_DMAError                             0x080100e9   Thumb Code    20  stm32f4xx_hal_tim.o(.text)
    HAL_TIM_PeriodElapsedCallback            0x080100fd   Thumb Code     2  stm32f4xx_hal_tim.o(.text)
    HAL_TIM_Base_Start_DMA                   0x08010113   Thumb Code    96  stm32f4xx_hal_tim.o(.text)
    HAL_TIM_Base_Stop_DMA                    0x08010173   Thumb Code    62  stm32f4xx_hal_tim.o(.text)
    HAL_TIM_OC_MspInit                       0x080101b1   Thumb Code     2  stm32f4xx_hal_tim.o(.text)
    HAL_TIM_OC_Init                          0x080101b3   Thumb Code    52  stm32f4xx_hal_tim.o(.text)
    HAL_TIM_OC_MspDeInit                     0x080101e7   Thumb Code     2  stm32f4xx_hal_tim.o(.text)
    HAL_TIM_OC_DeInit                        0x080101e9   Thumb Code    70  stm32f4xx_hal_tim.o(.text)
    TIM_CCxChannelCmd                        0x0801022f   Thumb Code    28  stm32f4xx_hal_tim.o(.text)
    HAL_TIM_OC_Start                         0x0801024b   Thumb Code    68  stm32f4xx_hal_tim.o(.text)
    HAL_TIM_OC_Stop                          0x0801028f   Thumb Code   170  stm32f4xx_hal_tim.o(.text)
    HAL_TIM_OC_Start_IT                      0x08010339   Thumb Code   144  stm32f4xx_hal_tim.o(.text)
    HAL_TIM_OC_Stop_IT                       0x080103c9   Thumb Code   196  stm32f4xx_hal_tim.o(.text)
    HAL_TIM_PWM_PulseFinishedCallback        0x0801048d   Thumb Code     2  stm32f4xx_hal_tim.o(.text)
    TIM_DMADelayPulseCplt                    0x0801048f   Thumb Code    70  stm32f4xx_hal_tim.o(.text)
    HAL_TIM_OC_Start_DMA                     0x080104d5   Thumb Code   310  stm32f4xx_hal_tim.o(.text)
    HAL_TIM_OC_Stop_DMA                      0x0801060b   Thumb Code   202  stm32f4xx_hal_tim.o(.text)
    HAL_TIM_PWM_MspInit                      0x080106d5   Thumb Code     2  stm32f4xx_hal_tim.o(.text)
    HAL_TIM_PWM_Init                         0x080106d7   Thumb Code    52  stm32f4xx_hal_tim.o(.text)
    HAL_TIM_PWM_MspDeInit                    0x0801070b   Thumb Code     2  stm32f4xx_hal_tim.o(.text)
    HAL_TIM_PWM_DeInit                       0x0801070d   Thumb Code    70  stm32f4xx_hal_tim.o(.text)
    HAL_TIM_PWM_Start                        0x08010753   Thumb Code    78  stm32f4xx_hal_tim.o(.text)
    HAL_TIM_PWM_Stop                         0x080107a1   Thumb Code   126  stm32f4xx_hal_tim.o(.text)
    HAL_TIM_PWM_Start_IT                     0x0801081f   Thumb Code   144  stm32f4xx_hal_tim.o(.text)
    HAL_TIM_PWM_Stop_IT                      0x080108af   Thumb Code   196  stm32f4xx_hal_tim.o(.text)
    HAL_TIM_PWM_Start_DMA                    0x08010973   Thumb Code   310  stm32f4xx_hal_tim.o(.text)
    HAL_TIM_PWM_Stop_DMA                     0x08010aa9   Thumb Code   202  stm32f4xx_hal_tim.o(.text)
    HAL_TIM_IC_MspInit                       0x08010b73   Thumb Code     2  stm32f4xx_hal_tim.o(.text)
    HAL_TIM_IC_Init                          0x08010b75   Thumb Code    60  stm32f4xx_hal_tim.o(.text)
    HAL_TIM_IC_MspDeInit                     0x08010bb1   Thumb Code     2  stm32f4xx_hal_tim.o(.text)
    HAL_TIM_IC_DeInit                        0x08010bb3   Thumb Code    70  stm32f4xx_hal_tim.o(.text)
    HAL_TIM_IC_Start                         0x08010bf9   Thumb Code    32  stm32f4xx_hal_tim.o(.text)
    HAL_TIM_IC_Stop                          0x08010c19   Thumb Code    58  stm32f4xx_hal_tim.o(.text)
    HAL_TIM_IC_Start_IT                      0x08010c53   Thumb Code   108  stm32f4xx_hal_tim.o(.text)
    HAL_TIM_IC_Stop_IT                       0x08010cbf   Thumb Code   134  stm32f4xx_hal_tim.o(.text)
    HAL_TIM_IC_CaptureCallback               0x08010d45   Thumb Code     2  stm32f4xx_hal_tim.o(.text)
    TIM_DMACaptureCplt                       0x08010d47   Thumb Code    70  stm32f4xx_hal_tim.o(.text)
    HAL_TIM_IC_Start_DMA                     0x08010d8d   Thumb Code   274  stm32f4xx_hal_tim.o(.text)
    HAL_TIM_IC_Stop_DMA                      0x08010e9f   Thumb Code   140  stm32f4xx_hal_tim.o(.text)
    HAL_TIM_OnePulse_MspInit                 0x08010f2b   Thumb Code     2  stm32f4xx_hal_tim.o(.text)
    HAL_TIM_OnePulse_Init                    0x08010f2d   Thumb Code    76  stm32f4xx_hal_tim.o(.text)
    HAL_TIM_OnePulse_MspDeInit               0x08010f79   Thumb Code     2  stm32f4xx_hal_tim.o(.text)
    HAL_TIM_OnePulse_DeInit                  0x08010f7b   Thumb Code    70  stm32f4xx_hal_tim.o(.text)
    HAL_TIM_OnePulse_Start                   0x08010fc1   Thumb Code    66  stm32f4xx_hal_tim.o(.text)
    HAL_TIM_OnePulse_Stop                    0x08011003   Thumb Code   130  stm32f4xx_hal_tim.o(.text)
    HAL_TIM_OnePulse_Start_IT                0x08011085   Thumb Code    90  stm32f4xx_hal_tim.o(.text)
    HAL_TIM_OnePulse_Stop_IT                 0x080110df   Thumb Code   154  stm32f4xx_hal_tim.o(.text)
    HAL_TIM_Encoder_MspInit                  0x08011179   Thumb Code     2  stm32f4xx_hal_tim.o(.text)
    HAL_TIM_Encoder_Init                     0x0801117b   Thumb Code   180  stm32f4xx_hal_tim.o(.text)
    HAL_TIM_Encoder_MspDeInit                0x0801122f   Thumb Code     2  stm32f4xx_hal_tim.o(.text)
    HAL_TIM_Encoder_DeInit                   0x08011231   Thumb Code    70  stm32f4xx_hal_tim.o(.text)
    HAL_TIM_Encoder_Start                    0x08011277   Thumb Code    78  stm32f4xx_hal_tim.o(.text)
    HAL_TIM_Encoder_Stop                     0x080112c5   Thumb Code   104  stm32f4xx_hal_tim.o(.text)
    HAL_TIM_Encoder_Start_IT                 0x0801132d   Thumb Code   126  stm32f4xx_hal_tim.o(.text)
    HAL_TIM_Encoder_Stop_IT                  0x080113ab   Thumb Code   162  stm32f4xx_hal_tim.o(.text)
    HAL_TIM_Encoder_Start_DMA                0x0801144d   Thumb Code   328  stm32f4xx_hal_tim.o(.text)
    HAL_TIM_Encoder_Stop_DMA                 0x08011595   Thumb Code   152  stm32f4xx_hal_tim.o(.text)
    HAL_TIM_TriggerCallback                  0x0801162d   Thumb Code     2  stm32f4xx_hal_tim.o(.text)
    HAL_TIM_OC_DelayElapsedCallback          0x0801162f   Thumb Code     2  stm32f4xx_hal_tim.o(.text)
    HAL_TIM_IRQHandler                       0x08011631   Thumb Code   406  stm32f4xx_hal_tim.o(.text)
    TIM_OC2_SetConfig                        0x08011899   Thumb Code   112  stm32f4xx_hal_tim.o(.text)
    HAL_TIM_OC_ConfigChannel                 0x0801196f   Thumb Code   116  stm32f4xx_hal_tim.o(.text)
    TIM_TI1_SetConfig                        0x08011a9d   Thumb Code   122  stm32f4xx_hal_tim.o(.text)
    HAL_TIM_IC_ConfigChannel                 0x08011b17   Thumb Code   224  stm32f4xx_hal_tim.o(.text)
    HAL_TIM_PWM_ConfigChannel                0x08011bf7   Thumb Code   294  stm32f4xx_hal_tim.o(.text)
    HAL_TIM_OnePulse_ConfigChannel           0x08011d1d   Thumb Code   286  stm32f4xx_hal_tim.o(.text)
    HAL_TIM_DMABurst_WriteStart              0x08011e4f   Thumb Code   366  stm32f4xx_hal_tim.o(.text)
    HAL_TIM_DMABurst_WriteStop               0x08011fbd   Thumb Code   128  stm32f4xx_hal_tim.o(.text)
    HAL_TIM_DMABurst_ReadStart               0x0801203d   Thumb Code   366  stm32f4xx_hal_tim.o(.text)
    HAL_TIM_DMABurst_ReadStop                0x080121ab   Thumb Code   128  stm32f4xx_hal_tim.o(.text)
    HAL_TIM_GenerateEvent                    0x0801222b   Thumb Code    54  stm32f4xx_hal_tim.o(.text)
    HAL_TIM_ConfigOCrefClear                 0x08012279   Thumb Code   252  stm32f4xx_hal_tim.o(.text)
    HAL_TIM_ConfigClockSource                0x080123df   Thumb Code   306  stm32f4xx_hal_tim.o(.text)
    HAL_TIM_ConfigTI1Input                   0x08012511   Thumb Code    24  stm32f4xx_hal_tim.o(.text)
    HAL_TIM_SlaveConfigSynchronization       0x080125cd   Thumb Code    86  stm32f4xx_hal_tim.o(.text)
    HAL_TIM_SlaveConfigSynchronization_IT    0x08012623   Thumb Code    86  stm32f4xx_hal_tim.o(.text)
    HAL_TIM_ReadCapturedValue                0x08012679   Thumb Code    84  stm32f4xx_hal_tim.o(.text)
    HAL_TIM_Base_GetState                    0x080126cd   Thumb Code     8  stm32f4xx_hal_tim.o(.text)
    HAL_TIM_OC_GetState                      0x080126d5   Thumb Code     8  stm32f4xx_hal_tim.o(.text)
    HAL_TIM_PWM_GetState                     0x080126dd   Thumb Code     8  stm32f4xx_hal_tim.o(.text)
    HAL_TIM_IC_GetState                      0x080126e5   Thumb Code     8  stm32f4xx_hal_tim.o(.text)
    HAL_TIM_OnePulse_GetState                0x080126ed   Thumb Code     8  stm32f4xx_hal_tim.o(.text)
    HAL_TIM_Encoder_GetState                 0x080126f5   Thumb Code     8  stm32f4xx_hal_tim.o(.text)
    HAL_TIMEx_HallSensor_MspInit             0x080126fd   Thumb Code     2  stm32f4xx_hal_tim_ex.o(.text)
    HAL_TIMEx_HallSensor_Init                0x080126ff   Thumb Code   196  stm32f4xx_hal_tim_ex.o(.text)
    HAL_TIMEx_HallSensor_MspDeInit           0x080127c3   Thumb Code     2  stm32f4xx_hal_tim_ex.o(.text)
    HAL_TIMEx_HallSensor_DeInit              0x080127c5   Thumb Code    70  stm32f4xx_hal_tim_ex.o(.text)
    HAL_TIMEx_HallSensor_Start               0x0801280b   Thumb Code    30  stm32f4xx_hal_tim_ex.o(.text)
    HAL_TIMEx_HallSensor_Stop                0x08012829   Thumb Code    56  stm32f4xx_hal_tim_ex.o(.text)
    HAL_TIMEx_HallSensor_Start_IT            0x08012861   Thumb Code    42  stm32f4xx_hal_tim_ex.o(.text)
    HAL_TIMEx_HallSensor_Stop_IT             0x0801288b   Thumb Code    68  stm32f4xx_hal_tim_ex.o(.text)
    HAL_TIMEx_HallSensor_Start_DMA           0x080128cf   Thumb Code   104  stm32f4xx_hal_tim_ex.o(.text)
    HAL_TIMEx_HallSensor_Stop_DMA            0x08012937   Thumb Code    68  stm32f4xx_hal_tim_ex.o(.text)
    HAL_TIMEx_OCN_Start                      0x08012997   Thumb Code    44  stm32f4xx_hal_tim_ex.o(.text)
    HAL_TIMEx_OCN_Stop                       0x080129c3   Thumb Code    96  stm32f4xx_hal_tim_ex.o(.text)
    HAL_TIMEx_OCN_Start_IT                   0x08012a23   Thumb Code   132  stm32f4xx_hal_tim_ex.o(.text)
    HAL_TIMEx_OCN_Stop_IT                    0x08012aa7   Thumb Code   196  stm32f4xx_hal_tim_ex.o(.text)
    HAL_TIMEx_OCN_Start_DMA                  0x08012b6b   Thumb Code   270  stm32f4xx_hal_tim_ex.o(.text)
    HAL_TIMEx_OCN_Stop_DMA                   0x08012c79   Thumb Code   192  stm32f4xx_hal_tim_ex.o(.text)
    HAL_TIMEx_PWMN_Start                     0x08012d39   Thumb Code    44  stm32f4xx_hal_tim_ex.o(.text)
    HAL_TIMEx_PWMN_Stop                      0x08012d65   Thumb Code    96  stm32f4xx_hal_tim_ex.o(.text)
    HAL_TIMEx_PWMN_Start_IT                  0x08012dc5   Thumb Code   132  stm32f4xx_hal_tim_ex.o(.text)
    HAL_TIMEx_PWMN_Stop_IT                   0x08012e49   Thumb Code   196  stm32f4xx_hal_tim_ex.o(.text)
    HAL_TIMEx_PWMN_Start_DMA                 0x08012f0d   Thumb Code   270  stm32f4xx_hal_tim_ex.o(.text)
    HAL_TIMEx_PWMN_Stop_DMA                  0x0801301b   Thumb Code   178  stm32f4xx_hal_tim_ex.o(.text)
    HAL_TIMEx_OnePulseN_Start                0x080130cd   Thumb Code    32  stm32f4xx_hal_tim_ex.o(.text)
    HAL_TIMEx_OnePulseN_Stop                 0x080130ed   Thumb Code    96  stm32f4xx_hal_tim_ex.o(.text)
    HAL_TIMEx_OnePulseN_Start_IT             0x0801314d   Thumb Code    56  stm32f4xx_hal_tim_ex.o(.text)
    HAL_TIMEx_OnePulseN_Stop_IT              0x08013185   Thumb Code   120  stm32f4xx_hal_tim_ex.o(.text)
    HAL_TIMEx_ConfigCommutationEvent         0x080131fd   Thumb Code   110  stm32f4xx_hal_tim_ex.o(.text)
    HAL_TIMEx_ConfigCommutationEvent_IT      0x0801326b   Thumb Code   122  stm32f4xx_hal_tim_ex.o(.text)
    HAL_TIMEx_CommutationCallback            0x080132e5   Thumb Code     2  stm32f4xx_hal_tim_ex.o(.text)
    TIMEx_DMACommutationCplt                 0x080132e7   Thumb Code    20  stm32f4xx_hal_tim_ex.o(.text)
    HAL_TIMEx_ConfigCommutationEvent_DMA     0x080132fb   Thumb Code   146  stm32f4xx_hal_tim_ex.o(.text)
    HAL_TIMEx_MasterConfigSynchronization    0x0801338d   Thumb Code    98  stm32f4xx_hal_tim_ex.o(.text)
    HAL_TIMEx_ConfigBreakDeadTime            0x080133ef   Thumb Code    80  stm32f4xx_hal_tim_ex.o(.text)
    HAL_TIMEx_RemapConfig                    0x0801343f   Thumb Code    48  stm32f4xx_hal_tim_ex.o(.text)
    HAL_TIMEx_BreakCallback                  0x0801346f   Thumb Code     2  stm32f4xx_hal_tim_ex.o(.text)
    HAL_TIMEx_HallSensor_GetState            0x08013471   Thumb Code     8  stm32f4xx_hal_tim_ex.o(.text)
    HAL_SPI_MspInit                          0x0801347d   Thumb Code     2  stm32f4xx_hal_spi.o(.text)
    HAL_SPI_Init                             0x0801347f   Thumb Code   140  stm32f4xx_hal_spi.o(.text)
    HAL_SPI_MspDeInit                        0x0801350b   Thumb Code     2  stm32f4xx_hal_spi.o(.text)
    HAL_SPI_DeInit                           0x0801350d   Thumb Code    54  stm32f4xx_hal_spi.o(.text)
    HAL_SPI_Transmit                         0x0801360b   Thumb Code   348  stm32f4xx_hal_spi.o(.text)
    HAL_SPI_TransmitReceive                  0x08013791   Thumb Code   404  stm32f4xx_hal_spi.o(.text)
    HAL_SPI_Receive                          0x08013925   Thumb Code   368  stm32f4xx_hal_spi.o(.text)
    HAL_SPI_TxCpltCallback                   0x08013a95   Thumb Code     2  stm32f4xx_hal_spi.o(.text)
    HAL_SPI_ErrorCallback                    0x08013a97   Thumb Code     2  stm32f4xx_hal_spi.o(.text)
    HAL_SPI_Transmit_IT                      0x08013b3f   Thumb Code   176  stm32f4xx_hal_spi.o(.text)
    HAL_SPI_RxCpltCallback                   0x08013bef   Thumb Code     2  stm32f4xx_hal_spi.o(.text)
    HAL_SPI_TxRxCpltCallback                 0x08013c71   Thumb Code     2  stm32f4xx_hal_spi.o(.text)
    HAL_SPI_TransmitReceive_IT               0x08013da1   Thumb Code   174  stm32f4xx_hal_spi.o(.text)
    HAL_SPI_Receive_IT                       0x08013e4f   Thumb Code   194  stm32f4xx_hal_spi.o(.text)
    HAL_SPI_TxHalfCpltCallback               0x08013fcf   Thumb Code     2  stm32f4xx_hal_spi.o(.text)
    HAL_SPI_Transmit_DMA                     0x08013fdf   Thumb Code   190  stm32f4xx_hal_spi.o(.text)
    HAL_SPI_RxHalfCpltCallback               0x080140e9   Thumb Code     2  stm32f4xx_hal_spi.o(.text)
    HAL_SPI_TxRxHalfCpltCallback             0x08014153   Thumb Code     2  stm32f4xx_hal_spi.o(.text)
    HAL_SPI_TransmitReceive_DMA              0x08014163   Thumb Code   276  stm32f4xx_hal_spi.o(.text)
    HAL_SPI_Receive_DMA                      0x08014277   Thumb Code   220  stm32f4xx_hal_spi.o(.text)
    HAL_SPI_DMAPause                         0x08014353   Thumb Code    50  stm32f4xx_hal_spi.o(.text)
    HAL_SPI_DMAResume                        0x08014385   Thumb Code    50  stm32f4xx_hal_spi.o(.text)
    HAL_SPI_DMAStop                          0x080143b7   Thumb Code    46  stm32f4xx_hal_spi.o(.text)
    HAL_SPI_IRQHandler                       0x080143e5   Thumb Code   252  stm32f4xx_hal_spi.o(.text)
    HAL_SPI_GetState                         0x080144e1   Thumb Code     8  stm32f4xx_hal_spi.o(.text)
    HAL_SPI_GetError                         0x080144e9   Thumb Code     6  stm32f4xx_hal_spi.o(.text)
    Reset_Handler                            0x080144f1   Thumb Code     8  startup_stm32f407xx.o(.text)
    SVC_Handler                              0x08014503   Thumb Code     2  startup_stm32f407xx.o(.text)
    PendSV_Handler                           0x08014507   Thumb Code     2  startup_stm32f407xx.o(.text)
    ADC_IRQHandler                           0x0801450b   Thumb Code     0  startup_stm32f407xx.o(.text)
    CAN1_RX0_IRQHandler                      0x0801450b   Thumb Code     0  startup_stm32f407xx.o(.text)
    CAN1_RX1_IRQHandler                      0x0801450b   Thumb Code     0  startup_stm32f407xx.o(.text)
    CAN1_SCE_IRQHandler                      0x0801450b   Thumb Code     0  startup_stm32f407xx.o(.text)
    CAN1_TX_IRQHandler                       0x0801450b   Thumb Code     0  startup_stm32f407xx.o(.text)
    CAN2_RX0_IRQHandler                      0x0801450b   Thumb Code     0  startup_stm32f407xx.o(.text)
    CAN2_RX1_IRQHandler                      0x0801450b   Thumb Code     0  startup_stm32f407xx.o(.text)
    CAN2_SCE_IRQHandler                      0x0801450b   Thumb Code     0  startup_stm32f407xx.o(.text)
    CAN2_TX_IRQHandler                       0x0801450b   Thumb Code     0  startup_stm32f407xx.o(.text)
    DCMI_IRQHandler                          0x0801450b   Thumb Code     0  startup_stm32f407xx.o(.text)
    DMA1_Stream0_IRQHandler                  0x0801450b   Thumb Code     0  startup_stm32f407xx.o(.text)
    DMA1_Stream1_IRQHandler                  0x0801450b   Thumb Code     0  startup_stm32f407xx.o(.text)
    DMA1_Stream2_IRQHandler                  0x0801450b   Thumb Code     0  startup_stm32f407xx.o(.text)
    DMA1_Stream3_IRQHandler                  0x0801450b   Thumb Code     0  startup_stm32f407xx.o(.text)
    DMA1_Stream4_IRQHandler                  0x0801450b   Thumb Code     0  startup_stm32f407xx.o(.text)
    DMA1_Stream5_IRQHandler                  0x0801450b   Thumb Code     0  startup_stm32f407xx.o(.text)
    DMA1_Stream6_IRQHandler                  0x0801450b   Thumb Code     0  startup_stm32f407xx.o(.text)
    DMA1_Stream7_IRQHandler                  0x0801450b   Thumb Code     0  startup_stm32f407xx.o(.text)
    DMA2_Stream0_IRQHandler                  0x0801450b   Thumb Code     0  startup_stm32f407xx.o(.text)
    DMA2_Stream1_IRQHandler                  0x0801450b   Thumb Code     0  startup_stm32f407xx.o(.text)
    DMA2_Stream2_IRQHandler                  0x0801450b   Thumb Code     0  startup_stm32f407xx.o(.text)
    DMA2_Stream3_IRQHandler                  0x0801450b   Thumb Code     0  startup_stm32f407xx.o(.text)
    DMA2_Stream4_IRQHandler                  0x0801450b   Thumb Code     0  startup_stm32f407xx.o(.text)
    DMA2_Stream5_IRQHandler                  0x0801450b   Thumb Code     0  startup_stm32f407xx.o(.text)
    DMA2_Stream6_IRQHandler                  0x0801450b   Thumb Code     0  startup_stm32f407xx.o(.text)
    DMA2_Stream7_IRQHandler                  0x0801450b   Thumb Code     0  startup_stm32f407xx.o(.text)
    ETH_IRQHandler                           0x0801450b   Thumb Code     0  startup_stm32f407xx.o(.text)
    ETH_WKUP_IRQHandler                      0x0801450b   Thumb Code     0  startup_stm32f407xx.o(.text)
    EXTI15_10_IRQHandler                     0x0801450b   Thumb Code     0  startup_stm32f407xx.o(.text)
    EXTI1_IRQHandler                         0x0801450b   Thumb Code     0  startup_stm32f407xx.o(.text)
    EXTI2_IRQHandler                         0x0801450b   Thumb Code     0  startup_stm32f407xx.o(.text)
    EXTI4_IRQHandler                         0x0801450b   Thumb Code     0  startup_stm32f407xx.o(.text)
    FLASH_IRQHandler                         0x0801450b   Thumb Code     0  startup_stm32f407xx.o(.text)
    FMC_IRQHandler                           0x0801450b   Thumb Code     0  startup_stm32f407xx.o(.text)
    FPU_IRQHandler                           0x0801450b   Thumb Code     0  startup_stm32f407xx.o(.text)
    HASH_RNG_IRQHandler                      0x0801450b   Thumb Code     0  startup_stm32f407xx.o(.text)
    I2C1_ER_IRQHandler                       0x0801450b   Thumb Code     0  startup_stm32f407xx.o(.text)
    I2C1_EV_IRQHandler                       0x0801450b   Thumb Code     0  startup_stm32f407xx.o(.text)
    I2C2_ER_IRQHandler                       0x0801450b   Thumb Code     0  startup_stm32f407xx.o(.text)
    I2C2_EV_IRQHandler                       0x0801450b   Thumb Code     0  startup_stm32f407xx.o(.text)
    I2C3_ER_IRQHandler                       0x0801450b   Thumb Code     0  startup_stm32f407xx.o(.text)
    I2C3_EV_IRQHandler                       0x0801450b   Thumb Code     0  startup_stm32f407xx.o(.text)
    OTG_FS_IRQHandler                        0x0801450b   Thumb Code     0  startup_stm32f407xx.o(.text)
    OTG_FS_WKUP_IRQHandler                   0x0801450b   Thumb Code     0  startup_stm32f407xx.o(.text)
    OTG_HS_EP1_IN_IRQHandler                 0x0801450b   Thumb Code     0  startup_stm32f407xx.o(.text)
    OTG_HS_EP1_OUT_IRQHandler                0x0801450b   Thumb Code     0  startup_stm32f407xx.o(.text)
    OTG_HS_IRQHandler                        0x0801450b   Thumb Code     0  startup_stm32f407xx.o(.text)
    OTG_HS_WKUP_IRQHandler                   0x0801450b   Thumb Code     0  startup_stm32f407xx.o(.text)
    PVD_IRQHandler                           0x0801450b   Thumb Code     0  startup_stm32f407xx.o(.text)
    RCC_IRQHandler                           0x0801450b   Thumb Code     0  startup_stm32f407xx.o(.text)
    RTC_Alarm_IRQHandler                     0x0801450b   Thumb Code     0  startup_stm32f407xx.o(.text)
    RTC_WKUP_IRQHandler                      0x0801450b   Thumb Code     0  startup_stm32f407xx.o(.text)
    SDIO_IRQHandler                          0x0801450b   Thumb Code     0  startup_stm32f407xx.o(.text)
    SPI1_IRQHandler                          0x0801450b   Thumb Code     0  startup_stm32f407xx.o(.text)
    SPI2_IRQHandler                          0x0801450b   Thumb Code     0  startup_stm32f407xx.o(.text)
    SPI3_IRQHandler                          0x0801450b   Thumb Code     0  startup_stm32f407xx.o(.text)
    TAMP_STAMP_IRQHandler                    0x0801450b   Thumb Code     0  startup_stm32f407xx.o(.text)
    TIM1_CC_IRQHandler                       0x0801450b   Thumb Code     0  startup_stm32f407xx.o(.text)
    TIM1_TRG_COM_TIM11_IRQHandler            0x0801450b   Thumb Code     0  startup_stm32f407xx.o(.text)
    TIM1_UP_TIM10_IRQHandler                 0x0801450b   Thumb Code     0  startup_stm32f407xx.o(.text)
    TIM2_IRQHandler                          0x0801450b   Thumb Code     0  startup_stm32f407xx.o(.text)
    TIM3_IRQHandler                          0x0801450b   Thumb Code     0  startup_stm32f407xx.o(.text)
    TIM4_IRQHandler                          0x0801450b   Thumb Code     0  startup_stm32f407xx.o(.text)
    TIM5_IRQHandler                          0x0801450b   Thumb Code     0  startup_stm32f407xx.o(.text)
    TIM8_CC_IRQHandler                       0x0801450b   Thumb Code     0  startup_stm32f407xx.o(.text)
    TIM8_TRG_COM_TIM14_IRQHandler            0x0801450b   Thumb Code     0  startup_stm32f407xx.o(.text)
    TIM8_UP_TIM13_IRQHandler                 0x0801450b   Thumb Code     0  startup_stm32f407xx.o(.text)
    UART4_IRQHandler                         0x0801450b   Thumb Code     0  startup_stm32f407xx.o(.text)
    UART5_IRQHandler                         0x0801450b   Thumb Code     0  startup_stm32f407xx.o(.text)
    USART1_IRQHandler                        0x0801450b   Thumb Code     0  startup_stm32f407xx.o(.text)
    USART2_IRQHandler                        0x0801450b   Thumb Code     0  startup_stm32f407xx.o(.text)
    USART3_IRQHandler                        0x0801450b   Thumb Code     0  startup_stm32f407xx.o(.text)
    USART6_IRQHandler                        0x0801450b   Thumb Code     0  startup_stm32f407xx.o(.text)
    WWDG_IRQHandler                          0x0801450b   Thumb Code     0  startup_stm32f407xx.o(.text)
    HAL_ADC_MspInit                          0x08014515   Thumb Code    98  stm32f4xx_hal_msp.o(.text)
    HAL_ETH_MspInit                          0x08014581   Thumb Code     2  ethernetif.o(.text)
    ethernetif_input                         0x0801480f   Thumb Code    44  ethernetif.o(.text)
    ethernetif_init                          0x0801483b   Thumb Code    38  ethernetif.o(.text)
    sys_now                                  0x08014861   Thumb Code     8  ethernetif.o(.text)
    ethernetif_set_link                      0x08014869   Thumb Code    60  ethernetif.o(.text)
    ethernetif_update_config                 0x080148a7   Thumb Code   252  ethernetif.o(.text)
    Init                                     0x080149ff   Thumb Code    40  main.o(.text)
    main                                     0x08014ad1   Thumb Code    22  main.o(.text)
    TIM1_BRK_TIM9_IRQHandler                 0x08014b0d   Thumb Code   166  stm32f4xx_it.o(.text)
    TIM7_IRQHandler                          0x08014bb3   Thumb Code     8  stm32f4xx_it.o(.text)
    EXTI0_IRQHandler                         0x08014bbb   Thumb Code    14  stm32f4xx_it.o(.text)
    EXTI3_IRQHandler                         0x08014bc9   Thumb Code   544  stm32f4xx_it.o(.text)
    TIM8_BRK_TIM12_IRQHandler                0x08014de9   Thumb Code    98  stm32f4xx_it.o(.text)
    EXTI9_5_IRQHandler                       0x08014e4b   Thumb Code    44  stm32f4xx_it.o(.text)
    NMI_Handler                              0x08014e77   Thumb Code     2  stm32f4xx_it.o(.text)
    HardFault_Handler                        0x08014e79   Thumb Code     4  stm32f4xx_it.o(.text)
    MemManage_Handler                        0x08014e7d   Thumb Code     4  stm32f4xx_it.o(.text)
    BusFault_Handler                         0x08014e81   Thumb Code     4  stm32f4xx_it.o(.text)
    UsageFault_Handler                       0x08014e85   Thumb Code     4  stm32f4xx_it.o(.text)
    DebugMon_Handler                         0x08014e89   Thumb Code     2  stm32f4xx_it.o(.text)
    SysTick_Handler                          0x08014e8b   Thumb Code     8  stm32f4xx_it.o(.text)
    User_notification                        0x08014f09   Thumb Code     2  app_ethernet.o(.text)
    ethernetif_notify_conn_changed           0x08014f0b   Thumb Code    56  app_ethernet.o(.text)
    RC5_CGI_Handler                          0x08014f4d   Thumb Code     8  httpd_cgi_ssi.o(.text)
    httpd_ssi_init                           0x08014f55   Thumb Code     2  httpd_cgi_ssi.o(.text)
    httpd_cgi_init                           0x08014f57   Thumb Code    20  httpd_cgi_ssi.o(.text)
    httpd_post_finished                      0x08015841   Thumb Code    36  httpd.o(.text)
    httpd_post_receive_data                  0x08015d45   Thumb Code    30  httpd.o(.text)
    httpd_post_begin                         0x08015da5   Thumb Code    30  httpd.o(.text)
    HTTP_Send_String                         0x080160fd   Thumb Code    32  httpd.o(.text)
    Send_LED                                 0x0801611d   Thumb Code   340  httpd.o(.text)
    httpd_init                               0x0801643b   Thumb Code    22  httpd.o(.text)
    http_set_ssi_handler                     0x08016451   Thumb Code    30  httpd.o(.text)
    http_set_cgi_handlers                    0x0801646f   Thumb Code    18  httpd.o(.text)
    fs_open                                  0x08016543   Thumb Code    70  fs.o(.text)
    fs_close                                 0x08016589   Thumb Code    12  fs.o(.text)
    fs_read                                  0x08016595   Thumb Code    62  fs.o(.text)
    fs_bytes_left                            0x080165d3   Thumb Code    10  fs.o(.text)
    EEPROM_IO_Init                           0x080166e9   Thumb Code     8  stm324xg_eval.o(.text)
    EEPROM_IO_WriteData                      0x080166f1   Thumb Code    28  stm324xg_eval.o(.text)
    EEPROM_IO_ReadData                       0x0801670d   Thumb Code    28  stm324xg_eval.o(.text)
    EEPROM_IO_IsDeviceReady                  0x08016729   Thumb Code    16  stm324xg_eval.o(.text)
    BSP_EEPROM_Init                          0x0801673d   Thumb Code    26  stm324xg_eval_eeprom.o(.text)
    BSP_EEPROM_TIMEOUT_UserCallback          0x08016757   Thumb Code     2  stm324xg_eval_eeprom.o(.text)
    BSP_EEPROM_ReadBuffer                    0x08016759   Thumb Code    34  stm324xg_eval_eeprom.o(.text)
    BSP_EEPROM_WriteBuffer                   0x080167d5   Thumb Code   420  stm324xg_eval_eeprom.o(.text)
    I2C_Config                               0x08016b95   Thumb Code    64  init_l.o(.text)
    Init_Config                              0x080173d3   Thumb Code    46  init_l.o(.text)
    IWDG_Init                                0x08017401   Thumb Code    32  init_l.o(.text)
    SPI_Init                                 0x08017421   Thumb Code    70  init_l.o(.text)
    Parse_Time                               0x08017481   Thumb Code    58  lab.o(.text)
    Update_Time                              0x080174bb   Thumb Code    80  lab.o(.text)
    Get_Var                                  0x0801750b   Thumb Code    60  lab.o(.text)
    Get_uint32                               0x08017547   Thumb Code    56  lab.o(.text)
    Interpolation                            0x0801757f   Thumb Code    90  lab.o(.text)
    GFX_Rect                                 0x080175d9   Thumb Code   442  lab.o(.text)
    GFX_NBK                                  0x08017793   Thumb Code   398  lab.o(.text)
    RGB565ToRGB888                           0x08017921   Thumb Code    46  lab.o(.text)
    ds2482_reset                             0x08017961   Thumb Code    72  onewire.o(.text)
    ds2482_write_config                      0x080179a9   Thumb Code    84  onewire.o(.text)
    ds2482_detect                            0x080179fd   Thumb Code    30  onewire.o(.text)
    OW_Reset                                 0x08017a1b   Thumb Code   122  onewire.o(.text)
    OW_WriteByte                             0x08017a95   Thumb Code   110  onewire.o(.text)
    OW_TouchBit                              0x08017b03   Thumb Code   138  onewire.o(.text)
    OW_ReadByte                              0x08017b8d   Thumb Code   138  onewire.o(.text)
    OW_WriteBit                              0x08017c17   Thumb Code    16  onewire.o(.text)
    OW_ReadBit                               0x08017c27   Thumb Code    14  onewire.o(.text)
    OW_SearchRom                             0x08017c35   Thumb Code   140  onewire.o(.text)
    OW_Search                                0x08017cc1   Thumb Code    96  onewire.o(.text)
    OW_Command                               0x08017d71   Thumb Code    28  onewire.o(.text)
    OW_Checksum                              0x08017d8d   Thumb Code    82  onewire.o(.text)
    Read_ds18b20                             0x08017ddf   Thumb Code   144  onewire.o(.text)
    ConvertTemperature_ds18b20               0x08017e6f   Thumb Code    30  onewire.o(.text)
    crc8                                     0x08017e8d   Thumb Code    62  onewire.o(.text)
    OW_CRC_Byte                              0x08017ecb   Thumb Code    32  onewire.o(.text)
    Def_OSR                                  0x08018753   Thumb Code   184  process2.o(.text)
    PrintToLCD                               0x0801918b   Thumb Code  1906  process2.o(.text)
    load_OW                                  0x08019a2d   Thumb Code   280  process2.o(.text)
    Edit_Menu                                0x0801a135   Thumb Code   298  process2.o(.text)
    main2                                    0x0801a613   Thumb Code    90  process2.o(.text)
    TIM6_DAC_IRQHandler                      0x0801a66d   Thumb Code    22  process2.o(.text)
    Change_OCR_MOTOR                         0x0801a75d   Thumb Code    56  process2.o(.text)
    Get_Buffer_Telnet                        0x0801a795   Thumb Code   518  process2.o(.text)
    RC5_Receiver_Init                        0x0801aa97   Thumb Code   180  rc5_ir_emul_receiver.o(.text)
    RC5_Sample_Data                          0x0801ab4b   Thumb Code   122  rc5_ir_emul_receiver.o(.text)
    RC5_MeasureFirstLowDuration              0x0801abc5   Thumb Code   292  rc5_ir_emul_receiver.o(.text)
    RC5_Decode                               0x0801ace9   Thumb Code   290  rc5_ir_emul_receiver.o(.text)
    RC5_CGI                                  0x0801ae0b   Thumb Code   256  rc5_ir_emul_receiver.o(.text)
    Telnet_init                              0x0801b029   Thumb Code    38  telnet.o(.text)
    TM_SPI_SetDataSize                       0x0801b069   Thumb Code    16  lcd_g.o(.text)
    TM_ILI9341_SendData16                    0x0801b079   Thumb Code    48  lcd_g.o(.text)
    TM_ILI9341_SendCommand                   0x0801b0a9   Thumb Code    48  lcd_g.o(.text)
    TM_ILI9341_SendData                      0x0801b0d9   Thumb Code    48  lcd_g.o(.text)
    TM_ILI9341_SetCursorPosition             0x0801b109   Thumb Code    76  lcd_g.o(.text)
    TM_ILI9341_SetSquare                     0x0801b155   Thumb Code    40  lcd_g.o(.text)
    TM_ILI9341_Putc                          0x0801b17d   Thumb Code   214  lcd_g.o(.text)
    TM_ILI9341_Puts                          0x0801b253   Thumb Code   118  lcd_g.o(.text)
    TM_ILI9341_INT_Fill                      0x0801b2c9   Thumb Code    82  lcd_g.o(.text)
    TM_ILI9341_Fill                          0x0801b31b   Thumb Code    28  lcd_g.o(.text)
    TM_ILI9341_Rotate                        0x0801b337   Thumb Code    96  lcd_g.o(.text)
    TM_ILI9341_InitLCD                       0x0801b397   Thumb Code   334  lcd_g.o(.text)
    TM_ILI9341_Init                          0x0801b4e5   Thumb Code   102  lcd_g.o(.text)
    TM_ILI9341_InitLCD__                     0x0801b54b   Thumb Code   616  lcd_g.o(.text)
    TM_ILI9341_DisplayOn                     0x0801b7b3   Thumb Code    10  lcd_g.o(.text)
    TM_ILI9341_DisplayOff                    0x0801b7bd   Thumb Code    10  lcd_g.o(.text)
    TM_ILI9341_DrawPixel                     0x0801b7c7   Thumb Code    42  lcd_g.o(.text)
    TM_ILI9341_GetStringSize                 0x0801b7f1   Thumb Code    28  lcd_g.o(.text)
    TM_ILI9341_DrawLine                      0x0801b80d   Thumb Code   316  lcd_g.o(.text)
    TM_ILI9341_DrawRectangle                 0x0801b949   Thumb Code    74  lcd_g.o(.text)
    TM_ILI9341_DrawFilledRectangle           0x0801b993   Thumb Code    68  lcd_g.o(.text)
    TM_ILI9341_DrawCircle                    0x0801b9d7   Thumb Code   260  lcd_g.o(.text)
    TM_ILI9341_DrawFilledCircle              0x0801badb   Thumb Code   334  lcd_g.o(.text)
    TM_ILI9341_GetPixel                      0x0801bc29   Thumb Code    74  lcd_g.o(.text)
    GG_ILI9341_PutImage                      0x0801bc73   Thumb Code   118  lcd_g.o(.text)
    __aeabi_uldivmod                         0x0801bcf5   Thumb Code    98  uldiv.o(.text)
    __aeabi_ldivmod                          0x0801bd57   Thumb Code    98  ldiv.o(.text)
    __aeabi_memcpy                           0x0801bdb9   Thumb Code    36  memcpya.o(.text)
    __aeabi_memcpy4                          0x0801bdb9   Thumb Code     0  memcpya.o(.text)
    __aeabi_memcpy8                          0x0801bdb9   Thumb Code     0  memcpya.o(.text)
    __aeabi_memset                           0x0801bddd   Thumb Code    14  memseta.o(.text)
    __aeabi_memset4                          0x0801bddd   Thumb Code     0  memseta.o(.text)
    __aeabi_memset8                          0x0801bddd   Thumb Code     0  memseta.o(.text)
    __aeabi_memclr                           0x0801bdeb   Thumb Code     4  memseta.o(.text)
    __aeabi_memclr4                          0x0801bdeb   Thumb Code     0  memseta.o(.text)
    __aeabi_memclr8                          0x0801bdeb   Thumb Code     0  memseta.o(.text)
    _memset$wrapper                          0x0801bdef   Thumb Code    18  memseta.o(.text)
    strstr                                   0x0801be01   Thumb Code    36  strstr.o(.text)
    strchr                                   0x0801be25   Thumb Code    20  strchr.o(.text)
    strlen                                   0x0801be39   Thumb Code    14  strlen.o(.text)
    strcmp                                   0x0801be47   Thumb Code    28  strcmp.o(.text)
    memcmp                                   0x0801be63   Thumb Code    26  memcmp.o(.text)
    strcpy                                   0x0801be7d   Thumb Code    18  strcpy.o(.text)
    strncmp                                  0x0801be8f   Thumb Code    30  strncmp.o(.text)
    strcspn                                  0x0801bead   Thumb Code    34  strcspn.o(.text)
    atoi                                     0x0801becf   Thumb Code    26  atoi.o(.text)
    __aeabi_dadd                             0x0801bee9   Thumb Code   322  dadd.o(.text)
    __aeabi_dsub                             0x0801c02b   Thumb Code     6  dadd.o(.text)
    __aeabi_drsub                            0x0801c031   Thumb Code     6  dadd.o(.text)
    __aeabi_dmul                             0x0801c037   Thumb Code   228  dmul.o(.text)
    __aeabi_ul2f                             0x0801c11b   Thumb Code    28  ffltul.o(.text)
    __aeabi_ui2d                             0x0801c137   Thumb Code    26  dfltui.o(.text)
    __aeabi_ul2d                             0x0801c151   Thumb Code    24  dfltul.o(.text)
    __aeabi_d2uiz                            0x0801c169   Thumb Code    50  dfixui.o(.text)
    __aeabi_f2d                              0x0801c19b   Thumb Code    38  f2d.o(.text)
    __aeabi_cdcmpeq                          0x0801c1c1   Thumb Code     0  cdcmple.o(.text)
    __aeabi_cdcmple                          0x0801c1c1   Thumb Code    48  cdcmple.o(.text)
    __aeabi_cdrcmple                         0x0801c1f1   Thumb Code    48  cdrcmple.o(.text)
    __aeabi_d2f                              0x0801c221   Thumb Code    56  d2f.o(.text)
    __aeabi_uidiv                            0x0801c259   Thumb Code     0  uidiv.o(.text)
    __aeabi_uidivmod                         0x0801c259   Thumb Code    44  uidiv.o(.text)
    __aeabi_llsl                             0x0801c285   Thumb Code    30  llshl.o(.text)
    _ll_shift_l                              0x0801c285   Thumb Code     0  llshl.o(.text)
    __aeabi_llsr                             0x0801c2a3   Thumb Code    32  llushr.o(.text)
    _ll_ushift_r                             0x0801c2a3   Thumb Code     0  llushr.o(.text)
    __aeabi_lasr                             0x0801c2c3   Thumb Code    36  llsshr.o(.text)
    _ll_sshift_r                             0x0801c2c3   Thumb Code     0  llsshr.o(.text)
    strtol                                   0x0801c2e7   Thumb Code   112  strtol.o(.text)
    __I$use$fp                               0x0801c357   Thumb Code     0  iusefp.o(.text)
    _float_round                             0x0801c357   Thumb Code    18  fepilogue.o(.text)
    _float_epilogue                          0x0801c369   Thumb Code    92  fepilogue.o(.text)
    _double_round                            0x0801c3c5   Thumb Code    30  depilogue.o(.text)
    _double_epilogue                         0x0801c3e3   Thumb Code   156  depilogue.o(.text)
    __aeabi_ddiv                             0x0801c47f   Thumb Code   222  ddiv.o(.text)
    _dsqrt                                   0x0801c55d   Thumb Code   162  dsqrt.o(.text)
    __aeabi_d2ulz                            0x0801c5ff   Thumb Code    48  dfixul.o(.text)
    __scatterload                            0x0801c631   Thumb Code    28  init.o(.text)
    __scatterload_rt2                        0x0801c631   Thumb Code     0  init.o(.text)
    __rt_ctype_table                         0x0801c655   Thumb Code     4  ctype_o.o(.text)
    _strtoul                                 0x0801c65d   Thumb Code   158  _strtoul.o(.text)
    _chval                                   0x0801c6fb   Thumb Code    28  _chval.o(.text)
    __decompress                             0x0801c717   Thumb Code     0  __dczerorl2.o(.text)
    __decompress1                            0x0801c717   Thumb Code    86  __dczerorl2.o(.text)
    __0sprintf                               0x0801c76d   Thumb Code    34  printfa.o(i.__0sprintf)
    __1sprintf                               0x0801c76d   Thumb Code     0  printfa.o(i.__0sprintf)
    __2sprintf                               0x0801c76d   Thumb Code     0  printfa.o(i.__0sprintf)
    __c89sprintf                             0x0801c76d   Thumb Code     0  printfa.o(i.__0sprintf)
    sprintf                                  0x0801c76d   Thumb Code     0  printfa.o(i.__0sprintf)
    __aeabi_errno_addr                       0x0801c795   Thumb Code     4  errno.o(i.__aeabi_errno_addr)
    __rt_errno_addr                          0x0801c795   Thumb Code     0  errno.o(i.__aeabi_errno_addr)
    __hardfp_sqrt                            0x0801c79d   Thumb Code   122  sqrt.o(i.__hardfp_sqrt)
    __scatterload_copy                       0x0801c817   Thumb Code    14  handlers.o(i.__scatterload_copy)
    __scatterload_null                       0x0801c825   Thumb Code     2  handlers.o(i.__scatterload_null)
    __scatterload_zeroinit                   0x0801c827   Thumb Code    14  handlers.o(i.__scatterload_zeroinit)
    __set_errno                              0x0801c835   Thumb Code     6  errno.o(i.__set_errno)
    tcp_state_str                            0x0801d124   Data          44  tcp.o(.constdata)
    tcp_backoff                              0x0801d150   Data          13  tcp.o(.constdata)
    tcp_persist_backoff                      0x0801d15d   Data           7  tcp.o(.constdata)
    tcp_pcb_lists                            0x0801d164   Data          16  tcp.o(.constdata)
    ip_addr_any                              0x0801d174   Data           4  ip_addr.o(.constdata)
    ip_addr_broadcast                        0x0801d178   Data           4  ip_addr.o(.constdata)
    ethbroadcast                             0x0801d17c   Data           6  etharp.o(.constdata)
    ethzero                                  0x0801d182   Data           6  etharp.o(.constdata)
    APBAHBPrescTable                         0x0801d188   Data          16  stm32f4xx_hal_rcc.o(.constdata)
    LEDS_CGI                                 0x0801d1a0   Data           8  httpd_cgi_ssi.o(.constdata)
    g_psDefaultFilenames                     0x0801d1a8   Data          40  httpd.o(.constdata)
    g_pcTagLeadIn                            0x0801d1d0   Data           4  httpd.o(.constdata)
    g_pcTagLeadOut                           0x0801d1d4   Data           4  httpd.o(.constdata)
    file__index_html                         0x080480cc   Data          20  fs.o(.constdata)
    file__jquery_min_js                      0x080480e0   Data          20  fs.o(.constdata)
    file__jquery_svg_css                     0x080480f4   Data          20  fs.o(.constdata)
    file__jquery_svg_js                      0x08048108   Data          20  fs.o(.constdata)
    file__Press_png                          0x0804811c   Data          20  fs.o(.constdata)
    file__Pump_png                           0x08048130   Data          20  fs.o(.constdata)
    file__style_css                          0x08048144   Data          20  fs.o(.constdata)
    arr_spirt                                0x08048158   Data        1500  process2.o(.constdata)
    MenuVarNBK                               0x08048734   Data        1080  process2.o(.constdata)
    MenuVarRect                              0x08048b6c   Data        1500  process2.o(.constdata)
    MenuSettingRect                          0x08049148   Data         600  process2.o(.constdata)
    MenuSettingNBK                           0x080493a0   Data         360  process2.o(.constdata)
    MenuVarDist                              0x08049508   Data         660  process2.o(.constdata)
    TM_Font7x10                              0x0804979c   Data        1900  tm_stm32f4_fonts.o(.constdata)
    TM_Font11x18                             0x08049f08   Data        3420  tm_stm32f4_fonts.o(.constdata)
    TM_Font16x26                             0x0804ac64   Data        4940  tm_stm32f4_fonts.o(.constdata)
    Font_16x27_Table                         0x0804bfb0   Data       12544  tm_stm32f4_fonts.o(.constdata)
    __ctype_table                            0x0804f0b0   Data         129  ctype_o.o(.constdata)
    Region$$Table$$Base                      0x08050acc   Number         0  anon$$obj.o(Region$$Table)
    Region$$Table$$Limit                     0x08050aec   Number         0  anon$$obj.o(Region$$Table)
    SystemCoreClock                          0x20000000   Data           4  system_stm32f4xx.o(.data)
    AHBPrescTable                            0x20000004   Data          16  system_stm32f4xx.o(.data)
    tcp_input_pcb                            0x20000030   Data           4  tcp_in.o(.data)
    udp_pcbs                                 0x20000048   Data           4  udp.o(.data)
    netif_list                               0x20000058   Data           4  netif.o(.data)
    netif_default                            0x2000005c   Data           4  netif.o(.data)
    tcp_ticks                                0x20000068   Data           4  tcp.o(.data)
    tcp_bound_pcbs                           0x2000006c   Data           4  tcp.o(.data)
    tcp_listen_pcbs                          0x20000070   Data           4  tcp.o(.data)
    tcp_active_pcbs                          0x20000074   Data           4  tcp.o(.data)
    tcp_tw_pcbs                              0x20000078   Data           4  tcp.o(.data)
    tcp_tmp_pcb                              0x2000007c   Data           4  tcp.o(.data)
    tcp_active_pcbs_changed                  0x20000080   Data           1  tcp.o(.data)
    current_netif                            0x20000094   Data           4  ip.o(.data)
    current_header                           0x20000098   Data           4  ip.o(.data)
    current_iphdr_src                        0x2000009c   Data           4  ip.o(.data)
    current_iphdr_dest                       0x200000a0   Data           4  ip.o(.data)
    uwTick                                   0x200000a8   Data           4  stm32f4xx_hal.o(.data)
    lnetif                                   0x200000ac   Data           4  ethernetif.o(.data)
    TAGCHAR                                  0x200000dc   Data           4  httpd_cgi_ssi.o(.data)
    TAGS                                     0x200000e0   Data           4  httpd_cgi_ssi.o(.data)
    CGI_TAB                                  0x200000e4   Data           8  httpd_cgi_ssi.o(.data)
    post_buf_write_pos                       0x200001dc   Data           4  httpd.o(.data)
    post_target_uri                          0x200001e0   Data           4  httpd.o(.data)
    g_pcSSIExtensions                        0x200001e4   Data          16  httpd.o(.data)
    lab_uri                                  0x200001f4   Data           4  httpd.o(.data)
    g_pfnSSIHandler                          0x200001f8   Data           4  httpd.o(.data)
    g_iNumTags                               0x200001fc   Data           4  httpd.o(.data)
    g_ppcTags                                0x20000200   Data           4  httpd.o(.data)
    g_pCGIs                                  0x20000204   Data           4  httpd.o(.data)
    g_iNumCGIs                               0x20000208   Data           4  httpd.o(.data)
    EEPROMTimeout                            0x2000020c   Data           4  stm324xg_eval_eeprom.o(.data)
    EEPROMDataRead                           0x20000210   Data           2  stm324xg_eval_eeprom.o(.data)
    EEPROMDataWrite                          0x20000212   Data           1  stm324xg_eval_eeprom.o(.data)
    mm                                       0x20000213   Data           1  init_l.o(.data)
    tt                                       0x20000214   Data           1  init_l.o(.data)
    er                                       0x20000215   Data           1  init_l.o(.data)
    ADC_5                                    0x20000218   Data           4  lab.o(.data)
    number_ADC                               0x2000021c   Data           4  lab.o(.data)
    sum_ADC                                  0x20000220   Data           4  lab.o(.data)
    Triac_Power_Real                         0x20000224   Data           2  lab.o(.data)
    Triac_Power_Val                          0x20000226   Data           2  lab.o(.data)
    n_RC5_TRIAC                              0x20000228   Data           4  lab.o(.data)
    hour                                     0x2000022c   Data           1  lab.o(.data)
    min                                      0x2000022d   Data           1  lab.o(.data)
    sec                                      0x2000022e   Data           1  lab.o(.data)
    time_loc                                 0x20000230   Data           8  lab.o(.data)
    Err_Power                                0x20000238   Data           4  lab.o(.data)
    LCDNoAutoUpdate                          0x2000023c   Data           1  process2.o(.data)
    RC5_sticky                               0x20000240   Data           4  process2.o(.data)
    STOP                                     0x20000244   Data           1  process2.o(.data)
    Power_Rect                               0x20000246   Data           2  process2.o(.data)
    Power                                    0x20000248   Data           2  process2.o(.data)
    Triac_Power_sum                          0x2000024c   Data           4  process2.o(.data)
    Corect_Power                             0x20000250   Data           4  process2.o(.data)
    sum_PWM_Print                            0x20000254   Data           4  process2.o(.data)
    hour_set                                 0x20000258   Data           1  process2.o(.data)
    min_set                                  0x20000259   Data           1  process2.o(.data)
    hour_golov_timer                         0x2000025a   Data           1  process2.o(.data)
    type_selection_golov                     0x2000025b   Data           1  process2.o(.data)
    hour_delta                               0x2000025c   Data           1  process2.o(.data)
    min_delta                                0x2000025d   Data           1  process2.o(.data)
    sec_delta                                0x2000025e   Data           1  process2.o(.data)
    sec_lcd                                  0x20000260   Data           4  process2.o(.data)
    sec_set                                  0x20000264   Data           1  process2.o(.data)
    sec_start                                0x20000268   Data           4  process2.o(.data)
    glob_interval                            0x2000026c   Data           4  process2.o(.data)
    glob_interval2                           0x20000270   Data           4  process2.o(.data)
    glob_interval_set                        0x20000274   Data           4  process2.o(.data)
    glob_interval_def                        0x20000278   Data           4  process2.o(.data)
    glob_interval_def_set                    0x2000027c   Data           4  process2.o(.data)
    counter                                  0x20000280   Data           4  process2.o(.data)
    LCD_Update                               0x20000284   Data           1  process2.o(.data)
    First_WEB                                0x20000285   Data           1  process2.o(.data)
    Tdef                                     0x20000288   Data           4  process2.o(.data)
    T_Att_Dim                                0x2000028c   Data           4  process2.o(.data)
    T_Att_Aqua                               0x20000290   Data           4  process2.o(.data)
    Tn                                       0x20000294   Data           4  process2.o(.data)
    T_3cm                                    0x20000298   Data           4  process2.o(.data)
    T_10cm                                   0x2000029c   Data           4  process2.o(.data)
    T_Par                                    0x200002a0   Data           4  process2.o(.data)
    T_NBK_Set                                0x200002a4   Data           4  process2.o(.data)
    T_10cm_Maxx                              0x200002a8   Data           4  process2.o(.data)
    Tkyb                                     0x200002ac   Data           4  process2.o(.data)
    KI_Motor                                 0x200002b0   Data           4  process2.o(.data)
    KP_Motor                                 0x200002b4   Data           4  process2.o(.data)
    error_I_Motor                            0x200002b8   Data           4  process2.o(.data)
    error_P_Motor                            0x200002bc   Data           4  process2.o(.data)
    KI_Power                                 0x200002c0   Data           4  process2.o(.data)
    KP_Power                                 0x200002c4   Data           4  process2.o(.data)
    error_I_Power                            0x200002c8   Data           4  process2.o(.data)
    error_P_Power                            0x200002cc   Data           4  process2.o(.data)
    KI_Dimrot                                0x200002d0   Data           4  process2.o(.data)
    KP_Dimrot                                0x200002d4   Data           4  process2.o(.data)
    error_P_Dimrot                           0x200002d8   Data           4  process2.o(.data)
    error_I_Dimrot                           0x200002dc   Data           4  process2.o(.data)
    nDTdef                                   0x200002e0   Data           1  process2.o(.data)
    nDTkyb                                   0x200002e1   Data           1  process2.o(.data)
    nDTattention                             0x200002e2   Data           1  process2.o(.data)
    T_d_Att_Dim_OW                           0x200002e4   Data          16  process2.o(.data)
    Tdef_OW                                  0x200002f4   Data          16  process2.o(.data)
    T_Att_Dim_OW                             0x20000304   Data          16  process2.o(.data)
    T_Att_Aqua_OW                            0x20000314   Data          16  process2.o(.data)
    Tn_OW                                    0x20000324   Data          16  process2.o(.data)
    T_10cm_OW                                0x20000334   Data          16  process2.o(.data)
    T_Par_OW                                 0x20000344   Data          16  process2.o(.data)
    Tkyb_OW                                  0x20000354   Data          16  process2.o(.data)
    Tattention                               0x20000364   Data           4  process2.o(.data)
    Tdef_set_dist                            0x20000368   Data           4  process2.o(.data)
    Tkyb_set_dist_END                        0x2000036c   Data           4  process2.o(.data)
    Tdef_set_rect_default                    0x20000370   Data           4  process2.o(.data)
    Tdef_set_rect_hol                        0x20000374   Data           4  process2.o(.data)
    Tdef_set_rect_podghol                    0x20000378   Data           4  process2.o(.data)
    Tdef_set_rect_hvst                       0x2000037c   Data           4  process2.o(.data)
    Theating_elements_Att                    0x20000380   Data           4  process2.o(.data)
    ADC_Conc_spirt_Att                       0x20000384   Data           4  process2.o(.data)
    Alcohol                                  0x20000388   Data           4  process2.o(.data)
    Corect_Alcohol_NBK                       0x2000038c   Data           4  process2.o(.data)
    Corect_Alcohol_Kyb                       0x20000390   Data           4  process2.o(.data)
    NO_Att                                   0x20000394   Data           2  process2.o(.data)
    TIMER_250                                0x20000396   Data           1  process2.o(.data)
    Timer_flag                               0x20000397   Data           1  process2.o(.data)
    OCR_CEL_Start                            0x20000398   Data           1  process2.o(.data)
    OCR_CEL_End                              0x20000399   Data           1  process2.o(.data)
    Tkyb_set_rect_End                        0x2000039c   Data           4  process2.o(.data)
    Tkyb_set_rect_Start                      0x200003a0   Data           4  process2.o(.data)
    OCR_PWM                                  0x200003a4   Data           1  process2.o(.data)
    OCR_PWM_hist                             0x200003a5   Data           1  process2.o(.data)
    OCR_CEL                                  0x200003a6   Data           1  process2.o(.data)
    OCR_Motor                                0x200003a7   Data           1  process2.o(.data)
    body_head                                0x200003a8   Data           1  process2.o(.data)
    stop_start                               0x200003a9   Data           1  process2.o(.data)
    auto_hand                                0x200003aa   Data           1  process2.o(.data)
    mode_proc                                0x200003ab   Data           1  process2.o(.data)
    mode_proc_hist                           0x200003ac   Data           1  process2.o(.data)
    mode                                     0x200003ad   Data           1  process2.o(.data)
    END                                      0x200003ae   Data           1  process2.o(.data)
    Lock_Menu                                0x200003af   Data           1  process2.o(.data)
    mode_setting                             0x200003b0   Data           1  process2.o(.data)
    current_mode                             0x200003b1   Data           1  process2.o(.data)
    EditMenu                                 0x200003b2   Data           1  process2.o(.data)
    EditMenu_hist                            0x200003b3   Data           1  process2.o(.data)
    Disable_LCD                              0x200003b4   Data           1  process2.o(.data)
    ADC_Press_Set                            0x200003b6   Data           2  process2.o(.data)
    ADC_Press                                0x200003b8   Data           2  process2.o(.data)
    ADC_Press_long                           0x200003bc   Data           4  process2.o(.data)
    ADC_Conc_spirt                           0x200003c0   Data           2  process2.o(.data)
    Water_start                              0x200003c2   Data           1  process2.o(.data)
    Water_Attention2                         0x200003c3   Data           1  process2.o(.data)
    size_mas                                 0x200003c4   Data           1  process2.o(.data)
    MenuTime                                 0x200003c8   Data           4  process2.o(.data)
    start_menu                               0x200003cc   Data           8  process2.o(.data)
    NBK_menu                                 0x200003d4   Data          12  process2.o(.data)
    rect_menu                                0x200003e0   Data          24  process2.o(.data)
    mode_menu                                0x200003f8   Data          12  process2.o(.data)
    auto_menu                                0x20000404   Data           8  process2.o(.data)
    type_selection_gol_menu                  0x2000040c   Data           8  process2.o(.data)
    show_def_00                              0x20000414   Data           7  process2.o(.data)
    show_def_Gol                             0x2000041b   Data           7  process2.o(.data)
    show_def_Rect                            0x20000422   Data           7  process2.o(.data)
    show_def_Hvost                           0x20000429   Data           7  process2.o(.data)
    show_Tn                                  0x20000430   Data           7  process2.o(.data)
    show_Tv                                  0x20000437   Data           7  process2.o(.data)
    EdgesNumber                              0x20000464   Data           1  rc5_ir_emul_receiver.o(.data)
    Bit4_HasBeen_Sampled                     0x20000465   Data           1  rc5_ir_emul_receiver.o(.data)
    RC5_FrameReceived                        0x20000466   Data           1  rc5_ir_emul_receiver.o(.data)
    BitTimeStatus                            0x20000467   Data           1  rc5_ir_emul_receiver.o(.data)
    FieldBit                                 0x20000468   Data           1  rc5_ir_emul_receiver.o(.data)
    RC5_Indexdata                            0x20000469   Data           1  rc5_ir_emul_receiver.o(.data)
    LowDuration                              0x2000046a   Data           2  rc5_ir_emul_receiver.o(.data)
    RC5_TIM_CLKValuekHz                      0x2000046c   Data           4  rc5_ir_emul_receiver.o(.data)
    HalfBitDurationCount_Min                 0x20000470   Data           2  rc5_ir_emul_receiver.o(.data)
    HalfBitDurationCount_Max                 0x20000472   Data           2  rc5_ir_emul_receiver.o(.data)
    NominalHalfBitDurationCount              0x20000474   Data           2  rc5_ir_emul_receiver.o(.data)
    FullBitDurationCount_Min                 0x20000476   Data           2  rc5_ir_emul_receiver.o(.data)
    FullBitDurationCount_Max                 0x20000478   Data           2  rc5_ir_emul_receiver.o(.data)
    NominalBitDurationCount                  0x2000047a   Data           2  rc5_ir_emul_receiver.o(.data)
    NominalBitDurationCount_3div4            0x2000047c   Data           2  rc5_ir_emul_receiver.o(.data)
    RC5_Frame                                0x2000047e   Data           3  rc5_ir_emul_receiver.o(.data)
    RC5_TogglePrevious                       0x20000481   Data           1  rc5_ir_emul_receiver.o(.data)
    FirstTimeIssued                          0x20000482   Data           1  rc5_ir_emul_receiver.o(.data)
    Command_hist                             0x20000483   Data           1  rc5_ir_emul_receiver.o(.data)
    Disable_Ext                              0x20000484   Data           1  rc5_ir_emul_receiver.o(.data)
    RC5_Devices                              0x20000488   Data         128  rc5_ir_emul_receiver.o(.data)
    RC5_Commands                             0x20000508   Data         512  rc5_ir_emul_receiver.o(.data)
    ILI9341_x                                0x2000070c   Data           2  lcd_g.o(.data)
    ILI9341_y                                0x2000070e   Data           2  lcd_g.o(.data)
    ILI9341_Opts                             0x20000710   Data           6  lcd_g.o(.data)
    ILI9341_INT_CalledFromPuts               0x20000716   Data           1  lcd_g.o(.data)
    TM_Font_7x10                             0x20000718   Data          12  tm_stm32f4_fonts.o(.data)
    TM_Font_11x18                            0x20000724   Data          12  tm_stm32f4_fonts.o(.data)
    TM_Font_16x26                            0x20000730   Data          12  tm_stm32f4_fonts.o(.data)
    UB_Font_Font_16x27                       0x2000073c   Data          12  tm_stm32f4_fonts.o(.data)
    press_image                              0x20000748   Data          12  img.o(.data)
    pump_image                               0x20000754   Data          12  img.o(.data)
    dhcp_rx_options_val                      0x20004fa4   Data          40  dhcp.o(.bss)
    dhcp_rx_options_given                    0x20004fcc   Data          10  dhcp.o(.bss)
    ram_heap                                 0x20004fd6   Data       10260  mem.o(.bss)
    DMARxDscrTab                             0x200078c4   Data         128  ethernetif.o(.bss)
    DMATxDscrTab                             0x20007944   Data         128  ethernetif.o(.bss)
    Rx_Buff                                  0x200079c4   Data        6096  ethernetif.o(.bss)
    Tx_Buff                                  0x20009194   Data        6096  ethernetif.o(.bss)
    EthHandle                                0x2000a964   Data          72  ethernetif.o(.bss)
    gnetif                                   0x2000a9ac   Data          56  main.o(.bss)
    post_buffer                              0x2000a9e4   Data        1024  httpd.o(.bss)
    fs_memory                                0x2000b224   Data         240  fs.o(.bss)
    hi2c1                                    0x2000b37c   Data          68  lab.o(.bss)
    SpiHandle                                0x2000b3c0   Data          88  lab.o(.bss)
    SpiTFTHandle                             0x2000b418   Data          88  lab.o(.bss)
    RtcHandle                                0x2000b470   Data          32  lab.o(.bss)
    TimHandle50ms                            0x2000b490   Data          60  lab.o(.bss)
    TimHandleTRIAC                           0x2000b4cc   Data          60  lab.o(.bss)
    TimHandleADC                             0x2000b508   Data          60  lab.o(.bss)
    TimHandle6                               0x2000b544   Data          60  lab.o(.bss)
    TimHandlePWM_Spirt                       0x2000b580   Data          60  lab.o(.bss)
    TimHandlePWM_Motor                       0x2000b5bc   Data          60  lab.o(.bss)
    TimHandlePWM_Dimrot                      0x2000b5f8   Data          60  lab.o(.bss)
    TimHandlePWM_Buzzer                      0x2000b634   Data          60  lab.o(.bss)
    TimHandlePWM_LED_ILI                     0x2000b670   Data          60  lab.o(.bss)
    sConfig_Dimrot                           0x2000b6ac   Data          28  lab.o(.bss)
    sConfig_Spirt                            0x2000b6c8   Data          28  lab.o(.bss)
    sConfig_Motor                            0x2000b6e4   Data          28  lab.o(.bss)
    sConfig_Buzzer                           0x2000b700   Data          28  lab.o(.bss)
    sConfig__LED_ILI                         0x2000b71c   Data          28  lab.o(.bss)
    AdcHandle                                0x2000b738   Data          72  lab.o(.bss)
    AdcHandle_ADC                            0x2000b780   Data          72  lab.o(.bss)
    PWM_SPIRT_TimHandle                      0x2000b7c8   Data          60  lab.o(.bss)
    stimestructure                           0x2000b804   Data          20  lab.o(.bss)
    sConfigTRIAC                             0x2000b818   Data          28  lab.o(.bss)
    Hiwdg                                    0x2000b834   Data          16  lab.o(.bss)
    ADCxConvertedValue                       0x2000b844   Data        2048  lab.o(.bss)
    Buffer_LCD                               0x2000c044   Data          20  lab.o(.bss)
    Buffer_Att                               0x2000c058   Data         200  lab.o(.bss)
    OW_SEARCH_BUFFER                         0x2000c120   Data          72  onewire.o(.bss)
    sum_PWM                                  0x2000c168   Data       60000  process2.o(.bss)
    var_cache_LCD                            0x2001abc8   Data         400  process2.o(.bss)
    var_cache_WEB                            0x2001ad58   Data         400  process2.o(.bss)
    WEB_Arr                                  0x2001aee8   Data        2500  process2.o(.bss)
    End_LCD_Print                            0x2001b8ac   Data          32  process2.o(.bss)
    RC5_data                                 0x2001b8cc   Data          26  rc5_ir_emul_receiver.o(.bss)
    TimHandle                                0x2001b8e8   Data          60  rc5_ir_emul_receiver.o(.bss)
    __initial_sp                             0x2001bd28   Data           0  startup_stm32f407xx.o(STACK)



==============================================================================

Memory Map of the image

  Image Entry point : 0x08000189

  Load Region LR_IROM1 (Base: 0x08000000, Size: 0x00051250, Max: 0x00080000, ABSOLUTE, COMPRESSED[0x00050e80])

    Execution Region ER_IROM1 (Exec base: 0x08000000, Load base: 0x08000000, Size: 0x00050aec, Max: 0x00080000, ABSOLUTE)

    Exec Addr    Load Addr    Size         Type   Attr      Idx    E Section Name        Object

    0x08000000   0x08000000   0x00000188   Data   RO         1317    RESET               startup_stm32f407xx.o
    0x08000188   0x08000188   0x00000000   Code   RO         2033  * .ARM.Collect$$$$00000000  mc_w.l(entry.o)
    0x08000188   0x08000188   0x00000004   Code   RO         2345    .ARM.Collect$$$$00000001  mc_w.l(entry2.o)
    0x0800018c   0x0800018c   0x00000004   Code   RO         2348    .ARM.Collect$$$$00000004  mc_w.l(entry5.o)
    0x08000190   0x08000190   0x00000000   Code   RO         2350    .ARM.Collect$$$$00000008  mc_w.l(entry7b.o)
    0x08000190   0x08000190   0x00000000   Code   RO         2352    .ARM.Collect$$$$0000000A  mc_w.l(entry8b.o)
    0x08000190   0x08000190   0x00000008   Code   RO         2353    .ARM.Collect$$$$0000000B  mc_w.l(entry9a.o)
    0x08000198   0x08000198   0x00000000   Code   RO         2355    .ARM.Collect$$$$0000000D  mc_w.l(entry10a.o)
    0x08000198   0x08000198   0x00000000   Code   RO         2357    .ARM.Collect$$$$0000000F  mc_w.l(entry11a.o)
    0x08000198   0x08000198   0x00000004   Code   RO         2346    .ARM.Collect$$$$00002712  mc_w.l(entry2.o)
    0x0800019c   0x0800019c   0x00000120   Code   RO            4    .text               system_stm32f4xx.o
    0x080002bc   0x080002bc   0x00001340   Code   RO          183    .text               tcp_in.o
    0x080015fc   0x080015fc   0x0000003e   Code   RO          270    .text               def.o
    0x0800163a   0x0800163a   0x00000002   PAD
    0x0800163c   0x0800163c   0x00000274   Code   RO          282    .text               lwip_timers.o
    0x080018b0   0x080018b0   0x000000ac   Code   RO          343    .text               memp.o
    0x0800195c   0x0800195c   0x00001254   Code   RO          387    .text               dhcp.o
    0x08002bb0   0x08002bb0   0x000004d8   Code   RO          403    .text               udp.o
    0x08003088   0x08003088   0x0000034c   Code   RO          432    .text               mem.o
    0x080033d4   0x080033d4   0x000002f0   Code   RO          454    .text               netif.o
    0x080036c4   0x080036c4   0x00000e60   Code   RO          476    .text               tcp.o
    0x08004524   0x08004524   0x00000ce4   Code   RO          500    .text               tcp_out.o
    0x08005208   0x08005208   0x000001c0   Code   RO          512    .text               raw.o
    0x080053c8   0x080053c8   0x0000001c   Code   RO          532    .text               init.o
    0x080053e4   0x080053e4   0x00000780   Code   RO          556    .text               pbuf.o
    0x08005b64   0x08005b64   0x000002b8   Code   RO          587    .text               ip_addr.o
    0x08005e1c   0x08005e1c   0x00000232   Code   RO          610    .text               inet_chksum.o
    0x0800604e   0x0800604e   0x00000002   PAD
    0x08006050   0x08006050   0x000006b8   Code   RO          625    .text               ip_frag.o
    0x08006708   0x08006708   0x00000358   Code   RO          645    .text               ip.o
    0x08006a60   0x08006a60   0x00000230   Code   RO          666    .text               icmp.o
    0x08006c90   0x08006c90   0x000009e8   Code   RO          741    .text               etharp.o
    0x08007678   0x08007678   0x000008e4   Code   RO          896    .text               stm32f4xx_hal_rcc.o
    0x08007f5c   0x08007f5c   0x00000bd8   Code   RO          923    .text               stm32f4xx_hal_adc.o
    0x08008b34   0x08008b34   0x00000194   Code   RO          974    .text               stm32f4xx_hal.o
    0x08008cc8   0x08008cc8   0x000003c4   Code   RO         1001    .text               stm32f4xx_hal_gpio.o
    0x0800908c   0x0800908c   0x0000020c   Code   RO         1025    .text               stm32f4xx_hal_pwr.o
    0x08009298   0x08009298   0x0000031c   Code   RO         1049    .text               stm32f4xx_hal_cortex.o
    0x080095b4   0x080095b4   0x00003194   Code   RO         1077    .text               stm32f4xx_hal_i2c.o
    0x0800c748   0x0800c748   0x000008c4   Code   RO         1101    .text               stm32f4xx_hal_adc_ex.o
    0x0800d00c   0x0800d00c   0x00000ea8   Code   RO         1125    .text               stm32f4xx_hal_eth.o
    0x0800deb4   0x0800deb4   0x00000618   Code   RO         1149    .text               stm32f4xx_hal_dma.o
    0x0800e4cc   0x0800e4cc   0x000000f0   Code   RO         1174    .text               stm32f4xx_hal_iwdg.o
    0x0800e5bc   0x0800e5bc   0x00000ba8   Code   RO         1198    .text               stm32f4xx_hal_rtc.o
    0x0800f164   0x0800f164   0x00000d9e   Code   RO         1222    .text               stm32f4xx_hal_rtc_ex.o
    0x0800ff02   0x0800ff02   0x00000002   PAD
    0x0800ff04   0x0800ff04   0x000027f8   Code   RO         1246    .text               stm32f4xx_hal_tim.o
    0x080126fc   0x080126fc   0x00000d80   Code   RO         1270    .text               stm32f4xx_hal_tim_ex.o
    0x0801347c   0x0801347c   0x00001072   Code   RO         1294    .text               stm32f4xx_hal_spi.o
    0x080144ee   0x080144ee   0x00000002   PAD
    0x080144f0   0x080144f0   0x00000024   Code   RO         1318    .text               startup_stm32f407xx.o
    0x08014514   0x08014514   0x0000006c   Code   RO         1325    .text               stm32f4xx_hal_msp.o
    0x08014580   0x08014580   0x00000428   Code   RO         1353    .text               ethernetif.o
    0x080149a8   0x080149a8   0x00000164   Code   RO         1444    .text               main.o
    0x08014b0c   0x08014b0c   0x000003fc   Code   RO         1498    .text               stm32f4xx_it.o
    0x08014f08   0x08014f08   0x00000044   Code   RO         1541    .text               app_ethernet.o
    0x08014f4c   0x08014f4c   0x00000034   Code   RO         1584    .text               httpd_cgi_ssi.o
    0x08014f80   0x08014f80   0x0000155c   Code   RO         1631    .text               httpd.o
    0x080164dc   0x080164dc   0x00000108   Code   RO         1664    .text               fs.o
    0x080165e4   0x080165e4   0x00000158   Code   RO         1692    .text               stm324xg_eval.o
    0x0801673c   0x0801673c   0x00000240   Code   RO         1716    .text               stm324xg_eval_eeprom.o
    0x0801697c   0x0801697c   0x00000b04   Code   RO         1743    .text               init_l.o
    0x08017480   0x08017480   0x000004e0   Code   RO         1771    .text               lab.o
    0x08017960   0x08017960   0x0000059c   Code   RO         1803    .text               onewire.o
    0x08017efc   0x08017efc   0x00002b3c   Code   RO         1833    .text               process2.o
    0x0801aa38   0x0801aa38   0x000004e0   Code   RO         1871    .text               rc5_ir_emul_receiver.o
    0x0801af18   0x0801af18   0x00000150   Code   RO         1907    .text               telnet.o
    0x0801b068   0x0801b068   0x00000c8c   Code   RO         1937    .text               lcd_g.o
    0x0801bcf4   0x0801bcf4   0x00000062   Code   RO         2036    .text               mc_w.l(uldiv.o)
    0x0801bd56   0x0801bd56   0x00000062   Code   RO         2038    .text               mc_w.l(ldiv.o)
    0x0801bdb8   0x0801bdb8   0x00000024   Code   RO         2040    .text               mc_w.l(memcpya.o)
    0x0801bddc   0x0801bddc   0x00000024   Code   RO         2042    .text               mc_w.l(memseta.o)
    0x0801be00   0x0801be00   0x00000024   Code   RO         2044    .text               mc_w.l(strstr.o)
    0x0801be24   0x0801be24   0x00000014   Code   RO         2046    .text               mc_w.l(strchr.o)
    0x0801be38   0x0801be38   0x0000000e   Code   RO         2048    .text               mc_w.l(strlen.o)
    0x0801be46   0x0801be46   0x0000001c   Code   RO         2050    .text               mc_w.l(strcmp.o)
    0x0801be62   0x0801be62   0x0000001a   Code   RO         2052    .text               mc_w.l(memcmp.o)
    0x0801be7c   0x0801be7c   0x00000012   Code   RO         2054    .text               mc_w.l(strcpy.o)
    0x0801be8e   0x0801be8e   0x0000001e   Code   RO         2056    .text               mc_w.l(strncmp.o)
    0x0801beac   0x0801beac   0x00000022   Code   RO         2058    .text               mc_w.l(strcspn.o)
    0x0801bece   0x0801bece   0x0000001a   Code   RO         2323    .text               mc_w.l(atoi.o)
    0x0801bee8   0x0801bee8   0x0000014e   Code   RO         2325    .text               mf_w.l(dadd.o)
    0x0801c036   0x0801c036   0x000000e4   Code   RO         2327    .text               mf_w.l(dmul.o)
    0x0801c11a   0x0801c11a   0x0000001c   Code   RO         2329    .text               mf_w.l(ffltul.o)
    0x0801c136   0x0801c136   0x0000001a   Code   RO         2331    .text               mf_w.l(dfltui.o)
    0x0801c150   0x0801c150   0x00000018   Code   RO         2333    .text               mf_w.l(dfltul.o)
    0x0801c168   0x0801c168   0x00000032   Code   RO         2335    .text               mf_w.l(dfixui.o)
    0x0801c19a   0x0801c19a   0x00000026   Code   RO         2337    .text               mf_w.l(f2d.o)
    0x0801c1c0   0x0801c1c0   0x00000030   Code   RO         2339    .text               mf_w.l(cdcmple.o)
    0x0801c1f0   0x0801c1f0   0x00000030   Code   RO         2341    .text               mf_w.l(cdrcmple.o)
    0x0801c220   0x0801c220   0x00000038   Code   RO         2343    .text               mf_w.l(d2f.o)
    0x0801c258   0x0801c258   0x0000002c   Code   RO         2362    .text               mc_w.l(uidiv.o)
    0x0801c284   0x0801c284   0x0000001e   Code   RO         2364    .text               mc_w.l(llshl.o)
    0x0801c2a2   0x0801c2a2   0x00000020   Code   RO         2366    .text               mc_w.l(llushr.o)
    0x0801c2c2   0x0801c2c2   0x00000024   Code   RO         2368    .text               mc_w.l(llsshr.o)
    0x0801c2e6   0x0801c2e6   0x00000070   Code   RO         2377    .text               mc_w.l(strtol.o)
    0x0801c356   0x0801c356   0x00000000   Code   RO         2379    .text               mc_w.l(iusefp.o)
    0x0801c356   0x0801c356   0x0000006e   Code   RO         2380    .text               mf_w.l(fepilogue.o)
    0x0801c3c4   0x0801c3c4   0x000000ba   Code   RO         2382    .text               mf_w.l(depilogue.o)
    0x0801c47e   0x0801c47e   0x000000de   Code   RO         2384    .text               mf_w.l(ddiv.o)
    0x0801c55c   0x0801c55c   0x000000a2   Code   RO         2386    .text               mf_w.l(dsqrt.o)
    0x0801c5fe   0x0801c5fe   0x00000030   Code   RO         2388    .text               mf_w.l(dfixul.o)
    0x0801c62e   0x0801c62e   0x00000002   PAD
    0x0801c630   0x0801c630   0x00000024   Code   RO         2390    .text               mc_w.l(init.o)
    0x0801c654   0x0801c654   0x00000008   Code   RO         2393    .text               mc_w.l(ctype_o.o)
    0x0801c65c   0x0801c65c   0x0000009e   Code   RO         2421    .text               mc_w.l(_strtoul.o)
    0x0801c6fa   0x0801c6fa   0x0000001c   Code   RO         2424    .text               mc_w.l(_chval.o)
    0x0801c716   0x0801c716   0x00000056   Code   RO         2434    .text               mc_w.l(__dczerorl2.o)
    0x0801c76c   0x0801c76c   0x00000028   Code   RO         2297    i.__0sprintf        mc_w.l(printfa.o)
    0x0801c794   0x0801c794   0x00000008   Code   RO         2370    i.__aeabi_errno_addr  mc_w.l(errno.o)
    0x0801c79c   0x0801c79c   0x0000007a   Code   RO         2021    i.__hardfp_sqrt     m_wm.l(sqrt.o)
    0x0801c816   0x0801c816   0x0000000e   Code   RO         2428    i.__scatterload_copy  mc_w.l(handlers.o)
    0x0801c824   0x0801c824   0x00000002   Code   RO         2429    i.__scatterload_null  mc_w.l(handlers.o)
    0x0801c826   0x0801c826   0x0000000e   Code   RO         2430    i.__scatterload_zeroinit  mc_w.l(handlers.o)
    0x0801c834   0x0801c834   0x0000000c   Code   RO         2372    i.__set_errno       mc_w.l(errno.o)
    0x0801c840   0x0801c840   0x00000184   Code   RO         2302    i._fp_digits        mc_w.l(printfa.o)
    0x0801c9c4   0x0801c9c4   0x000006dc   Code   RO         2303    i._printf_core      mc_w.l(printfa.o)
    0x0801d0a0   0x0801d0a0   0x00000024   Code   RO         2304    i._printf_post_padding  mc_w.l(printfa.o)
    0x0801d0c4   0x0801d0c4   0x0000002e   Code   RO         2305    i._printf_pre_padding  mc_w.l(printfa.o)
    0x0801d0f2   0x0801d0f2   0x0000000a   Code   RO         2307    i._sputc            mc_w.l(printfa.o)
    0x0801d0fc   0x0801d0fc   0x00000028   Data   RO          345    .constdata          memp.o
    0x0801d124   0x0801d124   0x00000050   Data   RO          477    .constdata          tcp.o
    0x0801d174   0x0801d174   0x00000008   Data   RO          589    .constdata          ip_addr.o
    0x0801d17c   0x0801d17c   0x0000000c   Data   RO          743    .constdata          etharp.o
    0x0801d188   0x0801d188   0x00000010   Data   RO          897    .constdata          stm32f4xx_hal_rcc.o
    0x0801d198   0x0801d198   0x00000008   Data   RO         1150    .constdata          stm32f4xx_hal_dma.o
    0x0801d1a0   0x0801d1a0   0x00000008   Data   RO         1585    .constdata          httpd_cgi_ssi.o
    0x0801d1a8   0x0801d1a8   0x00000030   Data   RO         1633    .constdata          httpd.o
    0x0801d1d8   0x0801d1d8   0x0002af80   Data   RO         1666    .constdata          fs.o
    0x08048158   0x08048158   0x00001644   Data   RO         1835    .constdata          process2.o
    0x0804979c   0x0804979c   0x00005914   Data   RO         1968    .constdata          tm_stm32f4_fonts.o
    0x0804f0b0   0x0804f0b0   0x00000081   Data   RO         2394    .constdata          mc_w.l(ctype_o.o)
    0x0804f131   0x0804f131   0x00000003   PAD
    0x0804f134   0x0804f134   0x00000004   Data   RO         2395    .constdata          mc_w.l(ctype_o.o)
    0x0804f138   0x0804f138   0x00000075   Data   RO          478    .conststring        tcp.o
    0x0804f1ad   0x0804f1ad   0x00000003   PAD
    0x0804f1b0   0x0804f1b0   0x0000000e   Data   RO         1586    .conststring        httpd_cgi_ssi.o
    0x0804f1be   0x0804f1be   0x00000002   PAD
    0x0804f1c0   0x0804f1c0   0x00000440   Data   RO         1634    .conststring        httpd.o
    0x0804f600   0x0804f600   0x00000199   Data   RO         1836    .conststring        process2.o
    0x0804f799   0x0804f799   0x00000003   PAD
    0x0804f79c   0x0804f79c   0x0000072b   Data   RO         1873    .conststring        rc5_ir_emul_receiver.o
    0x0804fec7   0x0804fec7   0x00000001   PAD
    0x0804fec8   0x0804fec8   0x00000c01   Data   RO         1998    .conststring        img.o
    0x08050ac9   0x08050ac9   0x00000003   PAD
    0x08050acc   0x08050acc   0x00000020   Data   RO         2426    Region$$Table       anon$$obj.o


    Execution Region RW_IRAM1 (Exec base: 0x20000000, Load base: 0x08050aec, Size: 0x0001bd28, Max: 0x00020000, ABSOLUTE, COMPRESSED[0x00000394])

    Exec Addr    Load Addr    Size         Type   Attr      Idx    E Section Name        Object

    0x20000000   COMPRESSED   0x00000014   Data   RW            5    .data               system_stm32f4xx.o
    0x20000014   COMPRESSED   0x00000020   Data   RW          185    .data               tcp_in.o
    0x20000034   COMPRESSED   0x0000000c   Data   RW          283    .data               lwip_timers.o
    0x20000040   COMPRESSED   0x00000004   Data   RW          389    .data               dhcp.o
    0x20000044   COMPRESSED   0x00000008   Data   RW          404    .data               udp.o
    0x2000004c   COMPRESSED   0x0000000c   Data   RW          434    .data               mem.o
    0x20000058   COMPRESSED   0x00000009   Data   RW          455    .data               netif.o
    0x20000061   COMPRESSED   0x00000003   PAD
    0x20000064   COMPRESSED   0x00000024   Data   RW          479    .data               tcp.o
    0x20000088   COMPRESSED   0x00000004   Data   RW          513    .data               raw.o
    0x2000008c   COMPRESSED   0x00000006   Data   RW          626    .data               ip_frag.o
    0x20000092   COMPRESSED   0x00000002   PAD
    0x20000094   COMPRESSED   0x00000012   Data   RW          646    .data               ip.o
    0x200000a6   COMPRESSED   0x00000001   Data   RW          744    .data               etharp.o
    0x200000a7   COMPRESSED   0x00000001   PAD
    0x200000a8   COMPRESSED   0x00000004   Data   RW          975    .data               stm32f4xx_hal.o
    0x200000ac   COMPRESSED   0x00000004   Data   RW         1355    .data               ethernetif.o
    0x200000b0   COMPRESSED   0x0000002c   Data   RW         1499    .data               stm32f4xx_it.o
    0x200000dc   COMPRESSED   0x00000010   Data   RW         1587    .data               httpd_cgi_ssi.o
    0x200000ec   COMPRESSED   0x00000120   Data   RW         1635    .data               httpd.o
    0x2000020c   COMPRESSED   0x00000007   Data   RW         1717    .data               stm324xg_eval_eeprom.o
    0x20000213   COMPRESSED   0x00000003   Data   RW         1745    .data               init_l.o
    0x20000216   COMPRESSED   0x00000002   PAD
    0x20000218   COMPRESSED   0x00000024   Data   RW         1773    .data               lab.o
    0x2000023c   COMPRESSED   0x00000228   Data   RW         1837    .data               process2.o
    0x20000464   COMPRESSED   0x000002a8   Data   RW         1874    .data               rc5_ir_emul_receiver.o
    0x2000070c   COMPRESSED   0x0000000b   Data   RW         1938    .data               lcd_g.o
    0x20000717   COMPRESSED   0x00000001   PAD
    0x20000718   COMPRESSED   0x00000030   Data   RW         1969    .data               tm_stm32f4_fonts.o
    0x20000748   COMPRESSED   0x00000018   Data   RW         1999    .data               img.o
    0x20000760   COMPRESSED   0x00000004   Data   RW         2373    .data               mc_w.l(errno.o)
    0x20000764        -       0x00000014   Zero   RW          184    .bss                tcp_in.o
    0x20000778        -       0x0000482b   Zero   RW          344    .bss                memp.o
    0x20004fa3   COMPRESSED   0x00000001   PAD
    0x20004fa4        -       0x00000032   Zero   RW          388    .bss                dhcp.o
    0x20004fd6        -       0x00002814   Zero   RW          433    .bss                mem.o
    0x200077ea        -       0x00000010   Zero   RW          588    .bss                ip_addr.o
    0x200077fa   COMPRESSED   0x00000002   PAD
    0x200077fc        -       0x000000c8   Zero   RW          742    .bss                etharp.o
    0x200078c4        -       0x000030e8   Zero   RW         1354    .bss                ethernetif.o
    0x2000a9ac        -       0x00000038   Zero   RW         1445    .bss                main.o
    0x2000a9e4        -       0x00000840   Zero   RW         1632    .bss                httpd.o
    0x2000b224        -       0x000000f0   Zero   RW         1665    .bss                fs.o
    0x2000b314        -       0x00000068   Zero   RW         1744    .bss                init_l.o
    0x2000b37c        -       0x00000da4   Zero   RW         1772    .bss                lab.o
    0x2000c120        -       0x00000048   Zero   RW         1804    .bss                onewire.o
    0x2000c168        -       0x0000f764   Zero   RW         1834    .bss                process2.o
    0x2001b8cc        -       0x00000058   Zero   RW         1872    .bss                rc5_ir_emul_receiver.o
    0x2001b924   COMPRESSED   0x00000004   PAD
    0x2001b928        -       0x00000400   Zero   RW         1315    STACK               startup_stm32f407xx.o


==============================================================================

Image component sizes


      Code (inc. data)   RO Data    RW Data    ZI Data      Debug   Object Name

        68         10          0          0          0       7241   app_ethernet.o
        62          0          0          0          0       1366   def.o
      4692         70          0          4         50      13502   dhcp.o
      2536         24         12          1        200      10459   etharp.o
      1064         50          0          4      12520      13379   ethernetif.o
       264          8     176000          0        240       5258   fs.o
      5468        396       1136        288       2112      19008   httpd.o
        52         22         22         16          0       5984   httpd_cgi_ssi.o
       560          8          0          0          0       2962   icmp.o
         0          0       3073         24          0        844   img.o
         0          0          0          0          0       3948   inet.o
       562          0          0          0          0       3385   inet_chksum.o
        28          0          0          0          0        624   init.o
      2820        206          0          3        104       4855   init_l.o
       856         28          0         18          0       7027   ip.o
       696         12          8          0         16      10159   ip_addr.o
      1720         18          0          6          0       7068   ip_frag.o
      1248         74          0         36       3492       5319   lab.o
      3212         80          0         11          0      11899   lcd_g.o
       628         40          0         12          0      19534   lwip_timers.o
       356         38          0          0         56       3222   main.o
       844         18          0         12      10260       4338   mem.o
       172         18         40          0      18475       4530   memp.o
       752         22          0          9          0       7377   netif.o
      1436         44          0          0         72       7560   onewire.o
      1920          0          0          0          0       9565   pbuf.o
     11068       1652       6109        552      63332      19974   process2.o
       448         12          0          4          0       3849   raw.o
      1248        114       1835        680         88      31912   rc5_ir_emul_receiver.o
        36          8        392          0       1024        848   startup_stm32f407xx.o
       344          4          0          0          0       3952   stm324xg_eval.o
       576          4          0          7          0       3530   stm324xg_eval_eeprom.o
       404         24          0          4          0       5055   stm32f4xx_hal.o
      3032         72          0          0          0       8459   stm32f4xx_hal_adc.o
      2244         50          0          0          0       6318   stm32f4xx_hal_adc_ex.o
       796         20          0          0          0      32435   stm32f4xx_hal_cortex.o
      1560         16          8          0          0       5264   stm32f4xx_hal_dma.o
      3752         58          0          0          0      10843   stm32f4xx_hal_eth.o
         0          0          0          0          0     473876   stm32f4xx_hal_flash_ex.o
       964         50          0          0          0       3907   stm32f4xx_hal_gpio.o
     12692        164          0          0          0      31900   stm32f4xx_hal_i2c.o
       240          0          0          0          0       2339   stm32f4xx_hal_iwdg.o
       108         10          0          0          0       1058   stm32f4xx_hal_msp.o
       524         20          0          0          0       3819   stm32f4xx_hal_pwr.o
      2276         66         16          0          0       5614   stm32f4xx_hal_rcc.o
      2984         20          0          0          0       8481   stm32f4xx_hal_rtc.o
      3486         18          0          0          0      13205   stm32f4xx_hal_rtc_ex.o
      4210         60          0          0          0      14892   stm32f4xx_hal_spi.o
     10232        152          0          0          0      32726   stm32f4xx_hal_tim.o
      3456         24          0          0          0      12466   stm32f4xx_hal_tim_ex.o
      1020        118          0         44          0       3407   stm32f4xx_it.o
       288         32          0         20          0     457793   system_stm32f4xx.o
      3680        140        197         36          0      22547   tcp.o
      4928        232          0         32         20      29458   tcp_in.o
      3300          8          0          0          0       9963   tcp_out.o
       336         26          0          0          0       5754   telnet.o
         0          0      22804         48          0       1665   tm_stm32f4_fonts.o
      1240         20          0          8          0      15373   udp.o

    ----------------------------------------------------------------------
    113496       4380     211696       1888     112068    1473095   Object Totals
         0          0         32          0          0          0   (incl. Generated)
         8          0         12          9          7          0   (incl. Padding)

    ----------------------------------------------------------------------

      Code (inc. data)   RO Data    RW Data    ZI Data      Debug   Library Member Name

       122          0          0          0          0        148   sqrt.o
        86          0          0          0          0          0   __dczerorl2.o
        28          0          0          0          0         68   _chval.o
       158          0          0          0          0         92   _strtoul.o
        26          0          0          0          0         80   atoi.o
         8          4        133          0          0         68   ctype_o.o
         0          0          0          0          0          0   entry.o
         0          0          0          0          0          0   entry10a.o
         0          0          0          0          0          0   entry11a.o
         8          4          0          0          0          0   entry2.o
         4          0          0          0          0          0   entry5.o
         0          0          0          0          0          0   entry7b.o
         0          0          0          0          0          0   entry8b.o
         8          4          0          0          0          0   entry9a.o
        20         10          0          4          0        136   errno.o
        30          0          0          0          0          0   handlers.o
        36          8          0          0          0         68   init.o
         0          0          0          0          0          0   iusefp.o
        98          0          0          0          0         84   ldiv.o
        30          0          0          0          0         68   llshl.o
        36          0          0          0          0         68   llsshr.o
        32          0          0          0          0         68   llushr.o
        26          0          0          0          0         80   memcmp.o
        36          0          0          0          0         68   memcpya.o
        36          0          0          0          0        108   memseta.o
      2276         86          0          0          0        520   printfa.o
        20          0          0          0          0         68   strchr.o
        28          0          0          0          0         76   strcmp.o
        18          0          0          0          0         68   strcpy.o
        34          0          0          0          0         80   strcspn.o
        14          0          0          0          0         68   strlen.o
        30          0          0          0          0         80   strncmp.o
        36          0          0          0          0         80   strstr.o
       112          0          0          0          0         88   strtol.o
        44          0          0          0          0         80   uidiv.o
        98          0          0          0          0         92   uldiv.o
        48          0          0          0          0         68   cdcmple.o
        48          0          0          0          0         68   cdrcmple.o
        56          0          0          0          0         88   d2f.o
       334          0          0          0          0        148   dadd.o
       222          0          0          0          0        100   ddiv.o
       186          0          0          0          0        176   depilogue.o
        50          0          0          0          0         76   dfixui.o
        48          0          0          0          0         68   dfixul.o
        26          0          0          0          0         76   dfltui.o
        24          0          0          0          0         76   dfltul.o
       228          0          0          0          0         96   dmul.o
       162          0          0          0          0        100   dsqrt.o
        38          0          0          0          0         68   f2d.o
       110          0          0          0          0        168   fepilogue.o
        28          0          0          0          0         84   ffltul.o

    ----------------------------------------------------------------------
      5148        116        136          4          0       3964   Library Totals
         2          0          3          0          0          0   (incl. Padding)

    ----------------------------------------------------------------------

      Code (inc. data)   RO Data    RW Data    ZI Data      Debug   Library Name

       122          0          0          0          0        148   m_wm.l
      3416        116        133          4          0       2356   mc_w.l
      1608          0          0          0          0       1460   mf_w.l

    ----------------------------------------------------------------------
      5148        116        136          4          0       3964   Library Totals

    ----------------------------------------------------------------------

==============================================================================


      Code (inc. data)   RO Data    RW Data    ZI Data      Debug   

    118644       4496     211832       1892     112068    1462911   Grand Totals
    118644       4496     211832        916     112068    1462911   ELF Image Totals (compressed)
    118644       4496     211832        916          0          0   ROM Totals

==============================================================================

    Total RO  Size (Code + RO Data)               330476 ( 322.73kB)
    Total RW  Size (RW Data + ZI Data)            113960 ( 111.29kB)
    Total ROM Size (Code + RO Data + RW Data)     331392 ( 323.63kB)

==============================================================================

